:100000000C94FF3A0C94273B0C94273B0C94273B11
:100010000C94273B0C94273B0C94273B0C94273BD8
:100020000C94273B0C94E7B80C94F2B80C94273B43
:100030000C94273B0C940FBF0C94273B0C94273B4C
:100040000C94FDB80C94273B0C94273B0C94273B55
:100050000C946FD10C94273B0C94273B0C94273BBA
:100060000C944B5A0C94273B0C94273B0C94273B45
:100070000C945FD00C9496D00C94273B0C94273BA7
:100080000C94273B0C94273B0C94273B783D7C3DFC
:10009000803D843D883DC73D9C3DA03DA43DAC3D99
:1000A000B03D353D4C3D503D543D583D5C3D603D7F
:1000B000643D683D6C3D703D743D483DB83DC33D79
:1000C0009C4CAC4CB14CBB4CC94CD04CD64CEA4CC3
:1000D000ED4CC470C770CF70CC70D270D570D87032
:1000E000DB70E070E370E870EB70EE70F170F4704C
:1000F000FC70FF70047107710C7111711671BAA256
:10010000FDA3C0A2CAA2D4A2E5A2F6A203A3FDA3A6
:1001100014A321A378A3B3A3CBA3DCA3ECA305A8CA
:100120004CCDB2D44EB93836A9020C50B99186885C
:10013000083CA6AAAA2ABE000000803F4F4B000D33
:100140000A00720A00496E717569727920456E6401
:10015000000D0A00496E71756972792052657375D8
:100160006C74733A0D0A002E004552524F520D0A1C
:10017000004F4B0D0A000D004154423F00415453C3
:10018000310041544E3D00415452310041545230EF
:100190000041544F300041544F31004154463F001C
:1001A0004154443D004154443000415448004154BE
:1001B0004100415400415445310041545130004107
:1001C00054453000415451310041544C35004154A4
:1001D0004C340041544C330041544C320041544C97
:1001E000310041544C300041544C2A0041545A30A3
:1001F000004154503D0054696D65206F75742C4664
:1002000061696C20746F20636F6E6E65637421008A
:10021000434F4E4E45435400444953434F4E4E4581
:100220004354000D0A0042544D32323220496E6967
:1002300074204F4B0042544D323232206E6F742086
:10024000666F756E642100425420696E697469613D
:100250006C6973696572656E2E2E007365617263D9
:1002600068206572726F7200666F756E64002E2E64
:100270002E2E002E2E2E002E2E002E003131353245
:1002800030300035373630302000333834303020CD
:1002900000313932303020003936303020200034FF
:1002A0003830302020003234303020200073656137
:1002B00072636820776974683A00736574204563D7
:1002C000686F206F6666004572726F722073657486
:1002D000204563686F0073657420426175647261C4
:1002E0007465204572726F72007365742042617587
:1002F0006472617465206F6B004572726F72312099
:100300007365742042617564726174652E2E0042BB
:100310005420736574206E65772042617564726144
:1003200074652E2E00504B54004576616C756174D7
:10033000696F6E20283836384D487A2920200052BF
:100340006164696F74726F6E69782057692E3233F9
:1003500032445453004143544956452100555342B9
:10036000202D3E2057692E32333200205553422033
:1003700042726964676520202020202000506F723F
:10038000742032303030004950203136392E323529
:10039000342E312E310050757474793A2074656CA6
:1003A0006E657400504B542076657262696E6465A8
:1003B0006E005043206D6974204164686F6320575C
:1003C000696669005769466C79204B6F6E6669678C
:1003D0007572696572656E004B6162656C20616E55
:1003E0007363686C69657373656E2E202000504BD3
:1003F000542065696E2067656B7265757A746573E4
:10040000202020005A7769736368656E204D4B2D5C
:1004100055534220756E642020004D4B2D5553429C
:1004200020616E20504320616E7363686C2E200043
:100430004643203E204D4B2D555342203E204254F2
:100440004D2D3232320042544D2D323232204B6F1C
:100450006E6669677572696572656E0041435449DD
:1004600056452100576C616E202D3E2057692E3273
:10047000333200574C414E2052616E676565787487
:10048000656E642E0052452D49443A200041435484
:100490004956452100426C7565746F6F7468202D54
:1004A0003E2057692E323332002042542052616E72
:1004B0006765657874656E64657200426175647223
:1004C0006174653A20004F4B002121436865636BDE
:1004D00020506172616D6574657221212000313692
:1004E000392E3235342E3030312E30303100323525
:1004F000352E3235352E3030302E3030300031361A
:10050000392E3235342E3030312E30303100313208
:1005100033343536373800504B54003030303000EB
:10052000303030302D30302D3030303030300050E1
:100530004B540030303030005374616E646172642B
:1005400077657274652067657365747A7400776582
:100550007264656E206175660020454550524F4DAE
:1005600020506172616D657465722020202000202A
:100570002020577269746520454550524F4D202008
:100580002020004F4B00636865636B207468652012
:1005900073657474696E6773210020202020202009
:1005A00056657273696F6E2020202020200045451B
:1005B00050726F6D55706461746520746F206E6544
:1005C00077003136392E3235342E3030312E3030FE
:1005D00031003235352E3235352E3030302E303038
:1005E00030003136392E3235342E3030312E303025
:1005F00031003132333400504B54006D002E002E48
:10060000006B6D2F68002E00636D002020006F6B63
:1006100000200044006E6F0032440033440020008C
:100620002D00780058004F00416C742020202020BD
:10063000203A20004C61742020202020203A200005
:100640004C6F6E6720202020203A20005370656593
:1006500064202020203A200050444F5020202020A9
:10066000203A20004163637572616379203A20006B
:100670005361742020202020203A200046697820F1
:1006800054797065203A20004E7572206D6974208F
:100690004E43202100332E372E3363583300536FDF
:1006A0006674776172653A005769466C7950617477
:1006B00063680031312E3230313200486172647724
:1006C00061726520504B5420332E397800576946AB
:1006D0006C7950617463680030392E3230313100EA
:1006E000486172647761726520504B5420332E3913
:1006F0006D000000000000007815141578002055EA
:100700005455780038454445380030494849300050
:100710003C4140413C003841402178007E15151590
:100720000A0022170F172200008482FF82841C1403
:100730001C00000000070507000010385410101EB0
:10074000180C180000001010101010101010107C61
:100750001010081008000000081400001408100809
:10076000040408100810202010080008142241007A
:1007700000412214080004027F02040010207F20A0
:100780001000103854101010101010543810101899
:100790001C1C181008183838180800081C3E7F0068
:1007A000007F3E1C080006090909060010201008F9
:1007B000040200000000000000002F0000000007FD
:1007C00000070000147F147F1400242A6B2A1200F3
:1007D00023130864620036495522500000050300C7
:1007E0000000001C224100000041221C00001408EF
:1007F0003E08140008083E080800005030000000C1
:1008000008080808080000606000000020100804C4
:1008100002003E5149453E0000427F4000004261D7
:10082000514946002141454B31001814127F1000F8
:100830002745454539003C4A4949300003017109C3
:100840000700364949493600064949291E00003645
:100850003600000000563600000008142241000057
:100860001414141414000041221408000201510948
:100870000600324979413E007E1111117E007F4908
:10088000494936003E41414122007F4141221C003E
:100890007F49494941007F09090901003E41494911
:1008A0007A007F0808087F0000417F410000204057
:1008B000413F01007F08142241007F40404040003A
:1008C0007F020C027F007F0408107F003E414141FF
:1008D0003E007F09090906003E4151215E007F0963
:1008E0001929460046494949310001017F010100AB
:1008F0003F4040403F001F2040201F003F40384005
:100900003F00631408146300070870080700615172
:10091000494543007F4141000000020408102000C7
:100920000041417F000004020102040040404040B9
:1009300040000001020400002054545478007F4815
:1009400044443800384444442000384444487F003C
:10095000385454541800087E090102000C525252B7
:100960003E007F080404780000447D4000002040E1
:10097000443D00007F102844000000417F400000FB
:100980007C04180478007C0804047800384444444B
:1009900038007C1414140800081414187C007C0817
:1009A00004040800485454542000043F44402000EC
:1009B0003C4040207C001C2040201C003C40384033
:1009C0003C004428102844000C5050503C00446423
:1009D000544C440000083641000000007F00000035
:1009E00000413608000008082A1C0800081C2A08D4
:1009F00008006E6F7420617661696C61626C6521BC
:100A000000746869732066756E6374696F6E20691F
:100A100073002A2A204F5554204F462052414D2022
:100A20002A2A003131353230300035373630300047
:100A300033383430300031393230300039363030EC
:100A4000003438303000323430300020202E202066
:100A50002E2020202000201A202020201B202020B3
:100A60002020457869740020203031323334353607
:100A70003738394142434445460D0A00537563688F
:100A800065204D696B726F6B6F7074657200736572
:100A900061726368204D696B726F6B6F7074004F89
:100AA000534420446174656E004F53442044617484
:100AB0006100504B54205370657A69616C00504B53
:100AC00054207370656369616C00504B5420436F10
:100AD0006E6E65637400504B5420536574757000DE
:100AE000504B5420496E666F004A6F797374696386
:100AF0006B004D4B20446973706C6179004D4B2045
:100B0000506172616D65746572004D4B2044617473
:100B1000656E004D4B2044617461004F5344004D9D
:100B20004B2047505320496E666F004254202020CE
:100B300052616E6765657874656E642E00574C412E
:100B40004E2052616E6765657874656E642E00553F
:100B5000534220202D3E20576932333200555342F4
:100B600020202D3E205356320042542020202D3E7E
:100B70002053563200504B5420436F6E6E656374A1
:100B8000004D4B204D6F746F727465737400547216
:100B900061636B696E6700504B54205370657A69CE
:100BA000616C002B112B112B11401156116C11820D
:100BB000119811AE11C411D611E811FA1104120ED8
:100BC0001218122212E8112C123C124C125C126DF7
:100BD0001282129712AB12BF12D412EA120013162D
:100BE000132C13421358136E1384139A13B013B0BB
:100BF00013C613DC13F21308141D143114441449E2
:100C0000144D145314561453145914601466146B71
:100C100014711477147E1491149F14B114BA14C370
:100C200014CC14D514DB14E414F814F8140D1511B5
:100C300015111516151D151D1523152B151D15330D
:100C40001539153F1545154B15511557155715579E
:100C5000155B156C157A158C159615A015AA15B48B
:100C600015BE15C815D715E415F215071619162C5B
:100C7000163F163F16511661166116701686169CA1
:100C800016B216C816DE16F41609171D172B1738DC
:100C90001745175217681774178A179D17B017C290
:100CA00017D317DD17EF17051818182D1843185507
:100CB0001869187F1889189B18AE18BA18C818DB5D
:100CC00018E718FB180F1923193619461955196713
:100CD0001979198B199D19B319C919DF19EF19025F
:100CE0001A171A271A371A491A491A491A5F1A7510
:100CF0001A8B1AA11AB71ACD1AE31AF91A0F1B2563
:100D00001B251B251B3B1B4B1B4B1B591B6F1B85A3
:100D10001B9B1BAD1BBC1BCD1BE31BF91B0E1C0E31
:100D20001C0E1C241C3A1C501C661C7C1C921CA80B
:100D30001CBE1CD41CEA1C001D081D141D1A1D20FD
:100D40001D261D261D261D2F1D2F1D2F1D371D3F46
:100D50001D471D4F1D591D631D6D1D7E1D8C1D9E44
:100D60001DA81DB11DBA1DC61DD21DDE1DEA1DF632
:100D70001D021E0E1E1A1E261E3C1E521E681E79C5
:100D80001E8A1E9B1EA61EB11EB81EC71ED71EE4BD
:100D90001EF11EFD1E0A1F181F181F261F261F26C4
:100DA0001F351F431F431F501F501F501F5A1F5AEC
:100DB0001F5A1F691F691F691F781F781F781F87B7
:100DC0001F871F871F961F961F961FA61FB81FCA33
:100DD0001FDC1FF21F012011201C20262038203D7F
:100DE00020422047204C20512056206C206C20822D
:100DF000209820A920BB20C620D020E220F4200685
:100E00002118212E212E214421522160216E216E94
:100E1000216E217E219421A821BD21D021DD21F345
:100E200021F32101220E2210221022122214221656
:100E3000221822182218221A221A221A221C221CD4
:100E4000221C221F221F221F222222252225222885
:100E5000223E224F2265227522812290229A22A4CC
:100E600022AD22C322D922EF22F622FD220823132B
:100E7000231C23262330233A2346235C236C237F21
:100E8000238F239A23A823B823C623D723E823F547
:100E900023012417242D24432456246324732489F6
:100EA000249F24B424CA24E024F6240C25222538C7
:100EB000254E2564257A258F25A425B925CF25CF54
:100EC00025E525FB25FB2511262226332643265121
:100ED0002651265F266D267B2689269726A526B3D2
:100EE00026C126C126CF26DD26EB26F926072715A3
:100EF00027232731273F274C274C274C275427549B
:100F00002754275C276B277A2789279D27B027C07E
:100F100027CB27D627E127EC27EC27F72702280D38
:100F2000281828232823282E282E282E2838283829
:100F30002838284228422842284728472847284C52
:100F4000284C284C2851285D28692875288128813B
:100F5000288D288D288D28992899289928A328AD8F
:100F600028B728C128C128C128CB28D528D528DFF3
:100F700028E928F328FD280729072911291B2925F5
:100F8000292F29452945295B296A296A297A29882F
:100F90002988299629A629B629C629D629D629E637
:100FA00029F629062A162A242A322A402A502A50AB
:100FB0002A602A6F2A6F2A802A802A802A8F2A8F05
:100FC0002A8F2AA22AA22AA22AB22AC32AD42AE52E
:100FD0002AE52AF62A072B182B292B392B4A2B5BBB
:100FE0002B6C2B7D2B7D2B8E2BA42BA42BB92BC7ED
:100FF0002BC72BD52BEB2BEB2B012C122C122C23DC
:101000002C232C232C392C392C392C4F2C4F2C4FA2
:101010002C582C5F2C662C6D2C752C7C2C842C8BE6
:101020002C932C9B2CAE2CAE2CC12CD42CE72CFA60
:101030002C0D2D0D2D202D332D462D592D6C2D6C65
:101040002D7F2D922DA52DB82DCB2DDE2DF12DF13F
:101050002DF12D042E0F2E1A2E252E382E4B2E5EFE
:101060002E712E842E972EAA2EBD2ED02EE32EF674
:101070002E092F162F232F302F3D2F3D2F4A2F5B68
:101080002F692F792F8C2F9F2FB22FB92FB92FC0F7
:101090002FC72FC72FCE2FE42FE42FFA2F0D300D9F
:1010A0003020302D302D303A304C304C305D306DAA
:1010B000306D307B308B308B309A30AB30AB30BA08
:1010C00030C830C830D430DD30E530ED30FE30FE91
:1010D000300E311E312E313E314E315E316E317E59
:1010E000318E319E31AE31BE31CE31CE31CE31D6A0
:1010F00031D631D631E131E131E131EA31EA31EA5B
:1011000031F431F431F431FD31FD31FD3105320579
:101110003205321032103210321532153215321AB1
:10112000321A321A321F321F321F32202020666FCD
:10113000726D6174206861726469736B20433F0053
:10114000201A20202020201B20202020456E6465AE
:101150002020204F4B00201A20202020201B202060
:101160002020656E64202020204F4B00201A202074
:101170002020201B2020202045696E646520204F00
:101180004B00201820202020201920202020456EF0
:1011900064652020204F4B0020182020202020199B
:1011A00020202020656E64202020204F4B00201836
:1011B0002020202020192020202045696E646520F1
:1011C000204F4B00201820202020201920202020F4
:1011D000456E646520002018202020202019202042
:1011E0002020656E64202000201820202020201957
:1011F0002020202045696E646500456E64652020CE
:10120000204F4B00656E64202020204F4B00456925
:101210006E646520204F4B00456E646520496E6604
:101220006F00656E642020696E666F005461737490
:101230006520312053656B756E6465004B65657084
:101240002074686520627574746F6E00486F7564F1
:10125000206465206B6E6F70202020006C616E67CB
:10126000206665737468616C74656E2E00707265BB
:101270007373656420666F722031207365636F6ECF
:10128000640031207365636F6E646520696E676505
:101290006472756B742E002066FC72204643203207
:1012A0002E3031662D322E3032620020666F722071
:1012B000464320322E3031662D322E3032620020ED
:1012C000566F6F7220464320322E3031662D322EFB
:1012D000303262002020204C65747A746520506F93
:1012E000736974696F6E202020002020206C617368
:1012F00074202020706F736974696F6E2020200045
:101300002020204C61617473746520706F73697460
:10131000696520202000204272656974656E6772DD
:1013200020204CE46E67656E67722000206C61744B
:10133000697475646520206C6F6E67697475646587
:1013400020006272656564746567722E206C656E3C
:1013500067746567722E20006CF6736368656E2093
:101360002020202020202077656974657200646544
:101370006C657465202020202020202020206578A6
:101380006974200077697373656E20202020202007
:101390002020207665726465720020202020476F2F
:1013A0006F676C652045696E67616265202020006B
:1013B00020202020476F6F676C6520496E70757420
:1013C00020202020200020202020202067656CF68F
:1013D00073636874202020202020200020202020FB
:1013E000202064656C657465642020202020202006
:1013F000200020202020202067657769737420203A
:1014000020202020202020007375636865204D690E
:101410006B726F6B6F707465722E2E2E0073656128
:10142000726368696E67204B6F707465722E2E2E22
:10143000007A6F656B20696B726F6B6F7074657289
:101440002E2E2E00456E646500656E640045696E43
:101450006465004F4B006F6B004665686C657200F9
:101460006572726F7200666F757400616B74697675
:101470000061637469760061637469656600464360
:10148000206E6963687420676566756E64656E2199
:10149000004643206E6F7420666F756E64210046AF
:1014A00043206E696574206765766F6E64656E2192
:1014B0000065727761727465740065787065637435
:1014C0006564007665727761636874006765667548
:1014D0006E64656E00666F756E64006765766F6E2C
:1014E00064656E00766F6C6C206B6F6D70617469F3
:1014F00062656C206E75720066756C6C20636F6D32
:1015000070617469626C65206F6E6C79006D6974CE
:101510000077697468004645484C45520045525270
:101520004F52005741524E554E47005741524E4977
:101530004E470045696E2020004F6E20202000415C
:10154000616E2020004175732020004F66662020C8
:101550000055697420200045534300504B542061CE
:101560007573736368616C74656E3F00736875743E
:10157000646F776E20504B543F00504B5420756978
:1015800074736368616B656C656E3F004A6120200F
:10159000204E65696E00796573202020206E6F00F3
:1015A0004A61202020204E6565004E65696E20202E
:1015B000204A61006E6F20202020796573004E65FF
:1015C00065202020204A6100446174656E206CF61D
:1015D000736368656E3F0064656C65746520646163
:1015E00074613F00446174656E2077697373656E42
:1015F0003F0056657262696E646520504B54206DE1
:1016000069742050432100436F6E6E6563742050EF
:101610004B5420746F2050430056657262696E64AB
:1016200020504B54206D6574205043004472FC637D
:101630006B6520275374617274272066FC7200501A
:1016400072657373202753746172742720666F72FA
:10165000006D696E2E20322053656B756E64656E69
:10166000006D696E2E2032207365636F6E647300A7
:101670002020202020202020202020456E6465206E
:10168000537461727400202020202020202020200C
:1016900020456E6420205374617274002020202045
:1016A00020202020202045696E64652053746172DB
:1016B00074002050432D517569636B2D566572621D
:1016C000696E64756E6720002050432D5175696303
:1016D0006B2D436F6E6E656374696F6E20002053CF
:1016E0006E656C6C652050432D76657262696E6420
:1016F000696E670056657262696E64652064617325
:1017000020504B54206D697400436F6E6E65637496
:1017100020504B542077697468204D4B00566572F9
:1017200062696E6420504B5420200064656D204D2A
:101730004B20FC6265723A002020206F7665722093
:101740002020203A002020206D65742020202020B9
:101750003A0064656D204D4B20FC6265723A202092
:101760004B6162656C2C20006F7665723A204B618C
:1017700062656C004D4B207669613A206B61626551
:101780006C202020202020202000657320697374A5
:10179000206B65696E2057692E323332007468659C
:1017A0007265206973206E6F2057692E32333200C4
:1017B0006572206973206765656E20576932333220
:1017C00020004D6F64756C2065696E676562617598
:1017D000742E006275696C7420696E2E006D6F64E2
:1017E000756C6520696E6765626F7577642E00574A
:1017F000656E6E20646F63682C2064616E6E20627B
:1018000069747465006966207965732C2074686555
:101810006E206669727374007A6F206A612C20648E
:10182000616E206175622065657273740064617316
:10183000204D6F64756C207A756572737420696DC4
:101840002020006163746976617465206D6F647532
:101850006C20696E006465206D6F64756C65206135
:101860006B7469766572656E0053657475706D652D
:101870006EFC20616B746976696572656E2E00532B
:10188000657475706D656E7500696E20686574208D
:1018900053657475704D656E752E00536965206DC6
:1018A000FC7373656E2064617320504B5400596F54
:1018B00075206861766520746F0055206D6F6574C2
:1018C00020646520504B54006A65747A74206E65FC
:1018D00075207374617274656E2100726573746132
:1018E000727420504B54006E75206F706E69657570
:1018F00077207374617274656E210045732069737B
:1019000074206B65696E2042544D2D323232005482
:1019100068657265206973206E6F2042544D2D32C8
:101920003232004572206973206765656E2042542B
:101930004D2D323232004D6F64756C2065696E67D3
:101940006562617574004D6F64756C206275696CB9
:101950007420696E006D6F64756C6520696E6765D3
:10196000626F7577642E00204D4B2D5553422046F3
:10197000756E6B74696F6E2000204D4B2D55534270
:101980002046756E6374696F6E2000204D4B2D5597
:1019900053422046756E63746965202000204254CE
:1019A000202D2D3E204B6162656C20616E204643E8
:1019B000202000204254202D2D3E204B6162656C7A
:1019C00020746F204643202000204254202D2D3EBD
:1019D000206B6162656C206E61617220464300502D
:1019E00043206D697420425420766572622E006334
:1019F0006F6E6E656374205043207769746820426F
:101A0000540050432076696120425420766572620A
:101A10006F6E64656E2E00504B542D4B6162656C89
:101A200020616E20464300504B542D4B6162656C23
:101A300020746F20464300504B542D6B6162656CDF
:101A4000206E61617220464300204254202D2D3EBD
:101A50002057692E323332202020202020200057AA
:101A6000692E32333220616E204643202020202010
:101A7000202020200057692E32333220746F2046F8
:101A8000432020202020202020200057693233329C
:101A9000206E6161722046432020202020202020DB
:101AA0000020555342202D2D3E204B6162656C2055
:101AB000616E204643200020555342202D2D3E20AC
:101AC0006361626C6520746F204643200055534269
:101AD000202D2D3E206B6162656C206E616172204D
:101AE0004643005043206D6974205553422076656B
:101AF0007262696E64656E2000636F6E6E656374FA
:101B000020504320776974682055534220200056A6
:101B1000657262696E64205043206D657420555370
:101B2000422020200020555342202D2D3E20576971
:101B30002E323332202020202020004D4B2D546F98
:101B40006F6C207374617274656E0073746172746B
:101B5000204D4B2D546F6F6C002057692E3233325D
:101B6000204B6F6E6669677572696572656E0020DD
:101B700057692E32333220436F6E66696775726122
:101B800074696F6E0020576932333220436F6E667E
:101B9000696775726174696520200050726F6772A1
:101BA000616D6D207374617274656E2E0073746163
:101BB00072742070726F6772616D2000737461724D
:101BC000742070726F6772616D6D612E0042544DAA
:101BD0002D323232204B6F6E66696775726965729D
:101BE000656E0042544D2D32323220636F6E66694D
:101BF0006775726174696F6E0042544D2D323232D6
:101C000020636F6E6669677572617469650046432B
:101C1000203E204D4B2D555342203E2042544D2D09
:101C2000323232004D4B2D55534220616E205043CD
:101C300020616E7363686C2E2000636F6E6E656347
:101C40007420504320746F204D4B2D55534220007B
:101C500056657262696E64205043206D6574204D34
:101C60004B2D555342005A7769736368656E204D5A
:101C70004B2D55534220756E64202000636F6E6EAD
:101C80006563742063726F73736564206361626C53
:101C9000650074757373656E204D4B2D555342204E
:101CA000656E20504B542000504B542065696E20C7
:101CB00067656B7265757A746573202020006265B4
:101CC000747765656E204D4B2D55534220616E64CF
:101CD0002020200065656E2067656B7275697374DE
:101CE00065206B6162656C2020004B6162656C2031
:101CF000616E7363686C69657373656E2E20200076
:101D0000504B54205356320061616E736C75697488
:101D1000656E2E004B6162656C006361626C6500EC
:101D20004B6162656C00536C617665202020004E2B
:101D30006F726D616C200052657665727365006923
:101D40006E7665727365006765696E7665720045CB
:101D50006E64652020204F4B00456E6420202020BB
:101D60004F4B0045696E642020204F4B00204545B5
:101D700050726F6D207769726B6C696368002052D6
:101D800065616C792064656C6574650020456570DB
:101D9000726F6D207765726B656C696A6B00206C81
:101DA000F6736368656E3F0020454570726F6D3F46
:101DB000002077697373656E3F00646575747363A3
:101DC0006820202020006765726D616E2020202031
:101DD0002000647569747320202020202000656E27
:101DE000676C6973636820202000656E676C697397
:101DF000682020202000656E67656C7320202020FD
:101E00002000686F6C6CE46E6469736368006475CD
:101E1000746368202020202020006E656465726C49
:101E2000616E64732000416E7A656967652045695B
:101E30006E7374656C6C756E67656E0020446973B3
:101E4000706C6179205365747570202020202020EB
:101E50002000446973706C617920696E7374656CDD
:101E60006C696E67656E2000496E666F73206265EF
:101E7000692053746172743A00496E666F20617410
:101E800020737461727475702000496E666F2062F1
:101E9000696A206F70737461727400537072616349
:101EA0006865203A20004C616E67756167653A206D
:101EB000005461616C3A20004C696368742061755C
:101EC00073206E616368004C69676874206F666692
:101ED000206166746572004C69636874207569746A
:101EE000206E61004C43442048656C6C69676B2E22
:101EF00000204272696768746E6573730020496ED2
:101F000074656E736974656974004C4344204B6F4B
:101F10006E74726173743A004C434420636F6E7444
:101F2000726173743A004C4344204E6F726D2F49B6
:101F30006E763A20005243204665686C657270697F
:101F40006570005243204572726F72626565700061
:101F5000446562756720504B540057692054582FD0
:101F60005258204368616E3A005769204E65745795
:101F70002E204772702E3A005769204E6574572EF6
:101F8000204D6F64653A0057692054582054696D9C
:101F9000656F75743A0057692055415254204D546D
:101FA000552020203A0057692E3233322065696E61
:101FB0006765626175743A0057692E323332206268
:101FC00075696C7420696E203A005769323332208B
:101FD000696E6765626F7577643A20004973742093
:101FE00065696E2057692E3233322D4D6F64756CE2
:101FF00020004973205769323332206D6F64756C4D
:102000000049732065722065656E2057693233324E
:102010000065696E6765626175743F006275696C21
:102020007420696E3F006D6F64756C6520696E6722
:1020300065626F7577643F004A612020007965739F
:1020400020004A612020004E65696E006E6F2020DE
:10205000004E656520002042544D323232204569E1
:102060006E7374656C6C756E67656E0020204254EB
:102070004D2D3232322073657474696E677320207F
:1020800020004973742065696E2042544D2D323210
:10209000322D4D6F64756C0049732042544D2D32C2
:1020A0003232204D6F64756C004973206572206573
:1020B000656E2042544D2D3232320065696E67657F
:1020C000626175743F006275696C7420696E3F00CF
:1020D0006D6F64756C6520696E6765626F75776496
:1020E0003F0042544D3232322065696E676562614D
:1020F00075743A0042544D323232206275696C7404
:1021000020696E203A0042544D32323220696E67A7
:1021100065626F7577643A0020504B5420416B6BB9
:10212000752045696E7374656C6C756E6700205020
:102130004B542041636375205365747570202020D3
:1021400020202000504B5420416B6B757479703AFD
:102150002000504B5420416363757479703A20001D
:10216000504B542041636375747970653A00416B3C
:102170006B752055204F66667365743A20004F6674
:1021800066736574207665727374656C6C656E2019
:102190006269730061646A757374206F6666736543
:1021A0007420756E74696C004F6666736574206187
:1021B00066726567656C656E20746F74006469652E
:1021C000205370616E6E756E67207061737374005A
:1021D000766F6C746167652066697473006465204E
:1021E0007370616E6E696E67206A756973742069B9
:1021F000732E004C6F77426174205761726E2056C7
:10220000004C6F7742617420616C61726D00560002
:1022100046004800420041004C0052004E69005206
:102220006F004B6F00436F004645484C45523A20C3
:10223000446174656E7665726C75737420004552E6
:10224000524F523A2044617461206C6F737400568F
:10225000657262696E64696E672076657262726F1C
:102260006B656E21004C65747A74652062656B61E4
:102270006E6E7465004C617374206B6E6F776E20A8
:10228000004C61617473742062656B656E646500F7
:10229000506F736974696F6E2000706F7369746931
:1022A0006F6E2000706F7369746965200020456946
:1022B0006E7374656C6C756E67656E2020202020CF
:1022C0002020002053657474696E67202020202030
:1022D00020202020202020200020496E7374656C6F
:1022E0006C696E67656E202020202020202000E48D
:1022F0006E6465726E006368616E67650076657214
:10230000616E646572656E00616B74697669657291
:10231000656E0061637469766174650061637469F8
:10232000766572656E00616B7469766965727400BA
:10233000616374697661746564006765616374697B
:102340007665657264002053657474696E672078E1
:102350002073706569636865726E3F002073746FE7
:1023600072652073657474696E673F0020736574CD
:1023700074696E6773206F70736C61616E3F0047A4
:102380006573706569636865727420756E64007347
:10239000746F72656420616E64006F706765736C42
:1023A0006167656E20656E004B6F706965726520B0
:1023B00053657474696E6700636F70792073657418
:1023C00074696E6773006B6F706965657220736501
:1023D0007474696E67730020766F6E2020782020F9
:1023E0006E616368202079002066726F6D2078200E
:1023F000746F2079002076616E2078206E612079DC
:1024000000766F6E2020206E6163682020456E6428
:10241000652020204F4B0066726F6D2020746F2066
:10242000202020656E64202020204F4B0076616EB6
:102430002020206E612020202065696E64652020A8
:102440004F4B005769726B6C696368206B6F7069E2
:102450006572656E3F007265616C6C7920636F70A8
:10246000793F0065636874206B6F7069656572659C
:102470006E3F004B6F706965727420756E642061E9
:102480006B7469766965727400636F706965642046
:10249000616E6420616374697661746564200047CD
:1024A000656B6F706965EB726420656E20616374A3
:1024B00069656600E46E646572652045696E7374D3
:1024C000656C6C756E67656E200020202063686106
:1024D0006E67652073657474696E677320202000D1
:1024E000696E7374656C6C696E67656E2077696A76
:1024F0007A6967656E002057E4686C6520506172E8
:10250000616D657465722020202020002073656C49
:1025100065637420706172616D65746572732020EB
:10252000200053656C65637465657220706172612B
:102530006D657465727320002057E4686C652053E4
:102540006569746520202020202020202000202084
:1025500020202073656C656374207061676520209E
:1025600020202000202053656C656374656572200F
:10257000706167696E61202020002057E4686C65F7
:102580002053657474696E673A2020202020002053
:1025900073656C6563742073657474696E6720205D
:1025A000202020002053656C65637465657220737C
:1025B000657474696E6720200020204750532045C1
:1025C000696E7374656C6C756E67656E2020002093
:1025D0002020204750532073657474696E67732000
:1025E0002020202000676577E4686C7465732047BD
:1025F000505320476572E47420200073656C656356
:1026000074656420475053206465766963652020B3
:102610000047505320456D70662E616B7469763F9C
:102620003A007265636569766520475053206F6E86
:102630003F3A00475053206F6E74762E2061616ED2
:102640003F3A006D61782048F66865202020203AE6
:10265000006D617820616C7469747564653A006D11
:102660006178204765736368772E203A006D617842
:102670002073706565642020203A006D61782073B6
:102680006E656C686569643A006D617820456E74AA
:102690006665726E2E3A006D6178206469737461AC
:1026A0006E63653A006D61782061667374616E6473
:1026B0003A20006D696E205370616E6E756E673AD8
:1026C000006D696E20766F6C74616765203A006DED
:1026D0006178205A656974202020203A006D617865
:1026E0002074696D65202020203A006D6178207487
:1026F000696A64202020203A006D6178205374724A
:102700006F6D2020203A006D6178206375727265CC
:102710006E74203A006D6178207374726F6F6D2053
:10272000203A00456E742E4B6170617A69742E3ABE
:10273000005573656443617061636974793A004759
:102740006562722E6361706163693A004C6F6E67F7
:102750002E203A004C61742E20203A004E757220D3
:102760006D6974204E4320212020004F6E6C79202B
:1027700077697468204E43202100416C6C65656E5A
:10278000206D6574204E4321004B65696E652053B2
:10279000657474696E67732021212020004E6F20BC
:1027A00073657474696E67732072656164212100BA
:1027B0004765656E2073657474696E6773212000C8
:1027C00048F6686520206175732000416C74692E9D
:1027D000206F66662000416C74692E207569742034
:1027E0000048F6686520626567722E00416C746966
:1027F0002E4C696D697400566172696F2061757342
:102800002000566172696F206F6666200056617203
:10281000696F207569742000566172696F2048F6EF
:10282000686500566172696F20416C742E0020202B
:102830002020202020202000436172652046726500
:10284000650020202020004C454431004C45443296
:10285000004E61766920206175732020004E6176FC
:102860006920206F66662020004E61766920207501
:102870006974202000506F732E2068616C74656E3F
:1028800000506F732E20486F6C64202000436F6DE2
:10289000696E6720486F6D65002020202020202071
:1028A0002020004A757374696572656E0043616C1F
:1028B0006962726174650043616C69627265722E4F
:1028C0000053746172742020202000426574726984
:1028D000656220200052756E2020202020200046B6
:1028E0006C696567656E202000466C792020202089
:1028F000202000566C69656720202020004C616E06
:1029000064756E672020004C616E64696E672020DC
:1029100000416B6B75206C656572004C6F772042CF
:1029200061742E20004C6F7720426174742E002059
:10293000204F534420416E7A656967652053657462
:10294000757020200020204F53442073637265650A
:102950006E207365747570202020004F7574312FC0
:1029600032206E656769657274004F7574312F325D
:1029700020696E766572746564004F7574312F320C
:1029800020466F726D6174004F7574312F3220666E
:102990006F726D6174004E6176696461746120616B
:1029A0006E20535632004E61766964617461207402
:1029B0006F20535632004E61766964617461206FF6
:1029C0007020535632006D2E2053696E6B72617405
:1029D00065206D2F73006D2E66616C6C737065657C
:1029E00064206D2F7300566172696F6D6574657236
:1029F000204265657000766172696F6D65746572FD
:102A0000206265657000766172696F6D65746572CC
:102A10002070696570006D4168205761726E756E37
:102A200067203E006D4168207761726E696E672095
:102A30003E006D416820776161727363682E3E00CD
:102A40004F534420416E7A656967657661723A003A
:102A50004F53442073637265656E6D6F64653A0011
:102A60004D4B20566F6C742042616C6B656E004D4F
:102A70004B20766F6C7420626172677261706800BF
:102A8000426175642057693233322F42543A002034
:102A9000466F6C6C6F77204D6520536574757020A0
:102AA0002000202020202052656672657368202057
:102AB0003A00476573636877696E6469676B656937
:102AC000743A002020202053706565642020202067
:102AD00020203A00202020536E656C6865696420D0
:102AE0002020203A00546F6C6572616E7A2052612A
:102AF000646975733A00546F6C6572616E746965D0
:102B0000205261642E3A00546F6E61757367616282
:102B100065204572772E3A00736F756E6420657874
:102B200074656E73696F6E3A00736F756E642065BD
:102B30007874656E7369653A004861726477617292
:102B400065205069657065723A00686172647761EA
:102B50007265206265657020203A00686172647752
:102B6000617265207069657020203A004C6175744F
:102B70007374E4726B6520202020203A00766F6C1D
:102B8000756D652020202020202020203A007365CC
:102B90007269656C6C65204B616EE46C65205365F1
:102BA0007475700073657269616C206368616E6E24
:102BB000656C207365747570004C69706F204D658D
:102BC0007373756E673A004C69706F206368656354
:102BD0006B20203A004B616E616C20202020202069
:102BE00020202020202020202020004368616E6EBD
:102BF000656C202020202020202020202020202044
:102C000000536572766F73636872697474653A20F5
:102C10002000736572766F73746570732020203A9C
:102C20002020002020202020202020536572766F55
:102C300020312020202020200020202020202020A3
:102C400020536572766F20322020202020200052F1
:102C50006576657273653A004C696E6B733A006C09
:102C6000656674683A006C696E6B733A005265630E
:102C70006874733A0072696768743A0072656368D1
:102C800074733A004D697474653A006D6964646CDC
:102C9000653A006D696464656E3A0054657374202A
:102CA00050756C736CE46E6765202020200074659D
:102CB0007374206672616D65776964746820202082
:102CC0000020536572766F207A756D205465737499
:102CD000656E200020736572766F20746F207465B6
:102CE0007374202020200020736572766F20746535
:102CF0002074657374656E20200020202020202021
:102D0000506572696F6465202020202000202020FB
:102D10002020206672616D65202020202020200068
:102D20005465737420666F72746C617566656E6449
:102D30002020007465737420636F6E74696E75650E
:102D40007320202020007465737420636F6E746993
:102D50006E752020202020200045696E7A656C73F6
:102D600063687269747420202020200073696E6784
:102D70006C65207374657020202020202020004185
:102D80006E7A61686C2020202020202020202020C6
:102D900020007465737420636F756E74202020208A
:102DA0002020202000746573742061616E74616C52
:102DB0002020202020202000506175736520456E62
:102DC00064706F736974696F6E20007061757365EC
:102DD00020656E64706F736974696F6E2000706136
:102DE0007573652065696E64706F736974696520B9
:102DF0000050617573652070726F20496E632E20DC
:102E000020202000475053204D617573203A004721
:102E10005053206D6F7573653A00475053206D75A0
:102E20006973203A00475053204254204D61757316
:102E30002031202020202000475053204254204D94
:102E40006F757365203120202020004750532042A9
:102E500054204D75697320312020202020004750D8
:102E60005320506F732E20766F6D204D4B20202005
:102E70000047505320706F732E2066726F6D204D87
:102E80004B20200047505320706F732E2076616EC8
:102E9000204D4B20202000537469636B206D696EB8
:102EA0002E20576572743A202000737469636B207A
:102EB0006D696E2E2076616C75653A2000737469B9
:102EC000636B206D696E207761617264653A2000E2
:102ED000537469636B206D61782E20576572743A64
:102EE000202000737469636B206D61782E207661F9
:102EF0006C75653A2000737469636B206D6178208E
:102F00007761617264653A20005269636874756E16
:102F1000673A20202000646972656374696F6E3AB5
:102F20002020007269636874696E673A202020006F
:102F3000537469636B747970653A20200073746907
:102F4000636B747970653A2020004E657574726108
:102F50006C6973696572656E643A006E657574724A
:102F6000616C697A696E673A006E65757472616C3E
:102F700069736572656E643A004C69706F204D65C7
:102F80007373756E673A2020202020004C69706FA3
:102F9000206D6561737572656D656E743A20004CC5
:102FA00069706F206D6574696E673A20202020205B
:102FB0002000506F7469202000706F746920200019
:102FC00054617374657200737769746368002020BC
:102FD00020504B54205A65697420205365747570D5
:102FE00020202000202020504B542074696D652043
:102FF000736574757020202020005A6569747A6F9B
:103000006E652020285554432B2D293A0074696D94
:1030100065207A6F6E6520285554432B2D293A0080
:10302000536F6D6D65727A656974203A0073756DC2
:103030006D65722074696D653A004F53442D20759B
:103040006E6420424C2D446174656E004F53442DD4
:1030500020616E6420424C206461746100204D4BFD
:10306000204665686C65726C6973746500204D4B11
:10307000206572726F726C6973740020557365728B
:10308000204750532D446174656E0020557365725E
:10309000204750532D6461746100206C65747A740C
:1030A0006520506F736974696F6E00206C61737472
:1030B00020706F736974696F6E00202020414C4C42
:1030C0004520446174656E00202020414C4C2064F2
:1030D000617461006CF6736368656E3F0064656CD3
:1030E0006574653F0077697373656E3F007A656943
:1030F0006765204D4B2D53657474696E6700736866
:103100006F77204D4B2073657474696E6700576C40
:10311000616E2065696E6765626175743A00576C0F
:10312000616E206275696C7420696E203A00576C7C
:10313000616E20696E6765626F7577643A005750FB
:10314000412076657277656E64656E203A0075730E
:103150006520575041202020202020203A00757300
:103160006520575041202020202020203A0053691C
:103170006368657268656974202020203A00736571
:103180006375726974792020202020203A007365CD
:103190006375726974792020202020203A004B61E9
:1031A0006E616C2020202020202020203A006368BF
:1031B000616E6E656C202020202020203A0063681C
:1031C000616E6E656C202020202020203A0047652B
:1031D0006E6572616C004E617669676174696F6ECD
:1031E00000456C656374726963004D4B2D537461C7
:1031F0007475730055736572204750530033442033
:103200004C6167650053746174697374696373001A
:103210004F534430004F534431004F534432004C1D
:1032200061737472696E6700322E3031662D322EF2
:1032300030326200204552522100332E372E336344
:1032400058330020504B542076003A2046432D52EC
:10325000657620004552524F523A206E6F206461CD
:103260007461004E43004643004552524F523A208B
:103270006E6F206461746100202000416E616C6F8C
:1032800067204E616D65733A200052656164696E16
:10329000673A004665686C65723A204B65696E65F1
:1032A00020446174656E004E4300464300202000B8
:1032B0004643004643004E430020202020446973CB
:1032C000706C617920001D00200020001D00416C01
:1032D0006C001D001A201B0056616C75653A202099
:1032E0002030004D6F746F723A2020203100204250
:1032F0004C2D4374726C2054657374202020202060
:1033000020202000BF34C834DA34EE3402351635BC
:103310002B353D354C355C3570357D358A359635E8
:10332000A235AE35B735C735CE35D935E535F435A7
:10333000FD350A3618362636353640365336613670
:103340006E3679368D369936A936B836B936BA36EC
:10335000BB36BC36BD360E0F0E4E0E0F0E4F0E0F87
:103360000E530E0F0E570E0F0E4E0E0F0E4F0E0F6A
:103370000E530E0F0E570E0F0E4E0E0F0E4F0E0F5A
:103380000E530E0F0E57C936CC36CF36D236D53641
:10339000D836DB36DE36496E666F005547707300EF
:1033A0006C6F6E672070726573733A003A002A2A58
:1033B000204D4B2D4572726F72202020202A2A004A
:1033C0002D206572726F72202D004D4B2053657455
:1033D00074696E6700504B54204F5344000B4300F8
:1033E0006D617820424C202054656D703A006D610B
:1033F0007820424C2020437572723A006D4168007B
:1034000020202030006B6D6800730041006D416822
:10341000006D4168006D0055475053006D00486FC6
:103420006D653A00416C743A00206B6D6800202095
:10343000493A004469723A00416C743A00206D4187
:10344000005750006D73006D202D005A69656C00A7
:1034500020536174005043002020006D202D00484F
:103460006F6D65004B6D68006D0041006D41680037
:103470005600560053006D0048F66865004D430045
:10348000545200534C00524C0046520054440054D5
:103490005500532100475000465300454C00465903
:1034A000004D52005354004341004241006F32002E
:1034B0006F31004348004346005048004148004EE9
:1034C0006F204572726F72004643206E6F742063E6
:1034D0006F6D70617469626C65004D4B334D61674F
:1034E000206E6F7420636F6D706174692E006E6F53
:1034F00020464320636F6D6D756E69636174696FFB
:103500006E006E6F204D4B334D616720636F6D6DA4
:10351000756E69632E006E6F2047505320636F6D88
:103520006D756E69636174696F6E006261642063BA
:103530006F6D706173732076616C75650052432006
:103540005369676E616C206C6F737400464320731F
:103550007069207278206572726F72006E6F204EF3
:103560004320636F6D6D756E69636174696F6E0082
:103570004643204E69636B204779726F00464320B3
:10358000526F6C6C204779726F0046432059617707
:10359000204779726F004643204E69636B20414398
:1035A0004300464320526F6C6C2041434300464326
:1035B000205A2D4143430050726573737572652024
:1035C00073656E736F720046432049324300426C4C
:1035D000204D697373696E67004D69786572204587
:1035E00072726F7200436172656672656520457222
:1035F000726F7200475053206C6F7374004D616797
:103600006E6574204572726F72004D6F746F722018
:103610007265737461727400424C204C696D6974F8
:103620006174696F6E00576179706F696E74207292
:10363000616E6765004E6F2053442D4361726400D4
:103640005344204C6F6767696E672061626F7274C4
:10365000656400466C79696E672072616E676521EA
:10366000004D617820416C746974756465004E6F1B
:10367000204750532046697800636F6D7061737303
:10368000206E6F742063616C6962722E00424C2060
:1036900073656C6674657374006E6F206578742E44
:1036A00020636F6D7061737300636F6D706173730E
:1036B0002073656E736F72000000000000504B5461
:1036C000205258206C6F7374004E45004520005303
:1036D00045005320005357005720004E57004E20FE
:1036E000004F534420446174656E004F534420647E
:1036F00061746100424C2020446174656E00424C4C
:10370000202064617461004D4B20204665686C6523
:10371000726C69737465004D4B20206572726F7214
:10372000736C697374004750532042656E75747AE8
:1037300065726C69737465004750532075736572C8
:103740006C69737400475053206C65747A746520FB
:10375000506F732E00475053206C61737420506F6C
:10376000732E004CD65343484520616C6C65204451
:103770006174656E0044454C45544520616C6C2075
:1037800064617461004F534420446174656E004469
:10379000656C00253230530020436F64652025306E
:1037A000327500253032753A253032753A2530327F
:1037B000752020253032752E253032752E25303477
:1037C0007500204D4B204572726F72730025332EA9
:1037D000366C6425332E366C6400253764206D47C3
:1037E00025352E3164206D4200253032752E25306E
:1037F00032752E253034752020253032753A25302B
:1038000032753A2530327500205573657220475065
:1038100053002020256354656D702E2538752025B2
:103820006343002020256343757272656E742534EE
:103830002E31752041002531643A2563437572723B
:10384000656E7425342E317520410020424C204491
:10385000617461002563424C2531642054656D70AC
:103860002E2025357520256343002563424C2531E4
:10387000642043757272656E7425322E3175204155
:1038800000256343757272656E7425362E3164208F
:103890004100256343757272656E7425362E31645E
:1038A00020410020424C2053746174697374696331
:1038B000002563526F6C6C2531316420256300252F
:1038C00063526F6C6C253131642025630025634E93
:1038D00069636B253131642025630025634E69637C
:1038E0006B2531316420256300256352432D5175CA
:1038F000616C69747925356400256352432D5175D7
:10390000616C697479253564002563566F6C746148
:10391000676525362E31642056002563424C2531DB
:10392000642054656D702E20253575202563430075
:103930002563424C25316420437572722E25342E46
:103940003175204100256343757272656E742536AA
:103950002E3164204100256343757272656E7425B3
:10396000362E3164204100204361706163697479AF
:10397000253764206D4168002563566572742E53A7
:103980007065656425332E3164206B6D6800256396
:1039900047726E642E537065656425332E31642042
:1039A0006B6D6800256344697374616E63652537C8
:1039B00075206D002563416C7469747564652537E5
:1039C00064206D00204C61737420466C79202025A2
:1039D0003032753A25303275206D696E00204F53B4
:1039E000442053746174697374696300456E643A6A
:1039F000202020253032753A2530327520202530A0
:103A000032752E253032752E00426567696E3A2078
:103A1000253032753A253032752020253032752E0A
:103A2000253032752E0020202020206E6F2064610A
:103A300074612E2E2E0020202020004B616EE46C3D
:103A4000652020202020202020004368616E6E65C4
:103A50006C20202020202020004B616E61616C20B2
:103A600020202020202020004B6F6E666967757231
:103A70006174696F6E20006D61696E2020202020C6
:103A8000202020202000436F6E6669677572617484
:103A90006965202000537469636B2020202020205A
:103AA00020202000737469636B20202020202020B8
:103AB000202000537469636B2020202020202020C8
:103AC00020004C6F6F70696E67202020202020201E
:103AD000004C6F6F70696E6720202020202020002E
:103AE0004C6F6F70696E67202020202020200048D6
:103AF000F668652020202020202020202000416C16
:103B000074697475646520202020202000486F6F40
:103B10006774652020202020202020004B616D65E7
:103B2000726120202020202020200043616D6572DA
:103B30006120202020202020200043616D657261DB
:103B40002020202020202020004E617669437472BE
:103B50006C202020202020004E6176694374726C16
:103B6000202020202020004E6176694374726C2052
:103B700020202020200041757367E46E67652020B7
:103B800020202020004F7574707574732020202031
:103B90002020200055697467616E67656E202020C3
:103BA000202000566572736368696564656E65738D
:103BB0002000446976657273202020202020202078
:103BC00000446976657273656E20202020202000F5
:103BD0004779726F202020202020202020200047BD
:103BE00079726F202020202020202020200047797B
:103BF000726F202020202020202020200042656E8F
:103C000075747A657220202020202000557365721B
:103C1000202020202020202020200047656272756F
:103C2000696B6572202020202000416368736B6FF0
:103C300070706C756E67202000436F75706C20414A
:103C400078657320202020004B6F7070656C696E62
:103C5000672041737320004D697865722D53657438
:103C6000757020202000436F6E666967204D69786B
:103C70002020202000436F6E6669672E204D6978F2
:103C8000657220004561737920536574757020203A
:103C9000202000436F6E666967204561737920209C
:103CA0002000436F6E6669672E206561737920205E
:103CB0000047617320202020202020202020200089
:103CC0005468726F74746C65202020202020004797
:103CD0006173202020202020202020202000476900
:103CE00065722020202020202020202000476965A8
:103CF000722020202020202020202000476965728B
:103D000020202020202020202020004E69636B20CE
:103D1000202020202020202020004E69636B2020BE
:103D20002020202020202020004E69636B202020AE
:103D30002020202020202000526F6C6C202020208A
:103D400020202020202000526F6C6C20202020207A
:103D5000202020202000526F6C6C2020202020206A
:103D60002020202000506F74692031202020202046
:103D700020202000506F7469203120202020202036
:103D8000202000506F746920312020202020202026
:103D90002000506F74692032202020202020202015
:103DA00000506F7469203220202020202020200025
:103DB000506F7469203220202020202020200050C5
:103DC0006F74692033202020202020202000506F95
:103DD00074692033202020202020202000506F7480
:103DE000692033202020202020202000506F74697B
:103DF0002034202020202020202000506F746920B3
:103E000034202020202020202000506F746920348E
:103E1000202020202020202000506F746920352091
:103E20002020202020202000506F74692035202081
:103E300020202020202000506F7469203520202071
:103E4000202020202000506F746920362020202060
:103E50002020202000506F74692036202020202050
:103E600020202000506F7469203620202020202040
:103E7000202000506F74692037202020202020202F
:103E80002000506F7469203720202020202020201F
:103E900000506F746920372020202020202020002F
:103EA000506F7469203820202020202020200050CE
:103EB0006F74692038202020202020202000506F9F
:103EC000746920382020202020202020004D6F748D
:103ED0006F7220536963682E536368004D6F742EB0
:103EE0005361666574792053772E004D6F742E737D
:103EF00061662E736368616B2E004D6F746F722064
:103F00005377692E4D6F6465004D6F746F72205347
:103F100077692E4D6F6465004D6F746F7220537713
:103F2000692E4D6F6465004572772E205369672EA8
:103F30002050722E2000456E682E205369672E4354
:103F40006865636B00556974672E5369672E436813
:103F500065636B00456D7066E46E67657220547929
:103F600070200052656365697665722054797065CA
:103F700020004F6E7476616E672E20547970652034
:103F80000053706B20616C6C204576656E74730015
:103F900053706B20616C6C204576656E74730053B2
:103FA000707265656B20616C6C657320200048F64B
:103FB00068656E726567656C657220200043747277
:103FC0006C20416C74697475646520004374726C74
:103FD00020486F6F677465202020004750532020D1
:103FE0002020202020202020200047505320202067
:103FF0002020202020202020004750532020202057
:1040000020202020202020004B6F6D7061737320D2
:1040100020202020202000436F6D706173732020CA
:104020002020202020004B6F6D7061732020202005
:1040300020202020004B6F6D704665737420417501
:1040400073722E00436F6D704F7269656E742E46E9
:104050006978004B6F6D70617320766173742020F6
:1040600020004572772E205369672E2050722E2033
:104070000053656E732E52637653696756616C0008
:10408000457874526563205369676E61616C0041C5
:1040900063687328652E296B6F70706C2E004178F1
:1040A000697320436F7570696E672020004173202B
:1040B0006B6F7070656C696E672020004472656874
:1040C000726174656E626567722E00526F74526120
:1040D0007465206C696D69742E00526F745261743E
:1040E00065206C696D69742E0048656164696E674E
:1040F00020486F6C642020004E69636B2F526F6CF8
:104100006C2020202020004B6F6572732076617335
:104110007420202020004E69636B2F526F6C6C203E
:1041200050202020004E69636B2F526F6C6C205022
:10413000202020004E69636B2F526F6C6C20502042
:104140002020004E69636B2F526F6C6C204420203E
:1041500020004E69636B2F526F6C6C20442020202E
:10416000004E69636B2F526F6C6C2044202020003E
:104170004769657220502020202020202020004701
:1041800069657220502020202020202020004769CF
:1041900065722050202020202020202000457874A7
:1041A00065726E65204B6F6E74722E004578746573
:1041B000726E204374726C20202000457874657202
:1041C0006E20436F6E74726F6C004C6F6F70696E0F
:1041D00067206F62656E2020004C6F6F70696E679C
:1041E00020757020202020004C6F6F70696E672052
:1041F0006F6D686F6F67004C6F6F70696E672075C9
:104200006E74656E20004C6F6F70696E6720646F0E
:10421000776E2020004C6F6F70696E672062656E4C
:1042200065642E004C6F6F70696E67206C696E6BF1
:104230007320004C6F6F70696E67206C6566742028
:1042400020004C6F6F70696E67206C696E6B732015
:10425000004C6F6F70696E672072656368747300DD
:104260004C6F6F70696E6720726967687420004CCC
:104270006F6F70696E672072656368747300476161
:1042800073204C696D6974202020202000546872CE
:104290006F74746C65204C696D697400476173209C
:1042A0004C696D6965742020202000416E73707226
:1042B000656368736368772E2000526573702E20E3
:1042C0005468726573682E20004472656D70656C69
:1042D00077616172646520004879737465726573F3
:1042E0006520202020200048797374657265736909
:1042F00073202020200048797374657265736520EF
:104300002020202000556D6B656872702E204E694C
:10431000636B20005475726E6F766572204E696310
:104320006B20004E69636B206765696E76657274F9
:104330002E00556D6B656872702E20526F6C6C206C
:10434000005475726E6F76657220526F6C6C20002F
:10435000526F6C6C206765696E766572742E0048CA
:10436000F668656E726567656C756E672000416CF6
:10437000746974756465204374726C2000486F6FB3
:1043800067746520436F6E74726F6C004A3A4842DE
:1043900065672C4E3A566172696F00593A4C696DE7
:1043A000482C4E3A566172696F00593A4C696D4813
:1043B0002C4E3A566172696F00536368616C746584
:1043C0007220662E20482E007573652053772E20AC
:1043D000662E5365747000536368616B2E20486FBE
:1043E0006F6774652000616B7573742E205661725F
:1043F000696F20200061636F757374696320566173
:1044000072696F00416B6F6573742E20566172691B
:104410006F2000536F6C6C68F668652020202020A8
:104420002000536574706F696E7420202020202056
:1044300000476577656E73746520686F6F677400F9
:104440004D696E2E20476173202020202020006DB2
:10445000696E2E207468726F74746C6520004D69EB
:104460006E696D61616C2067617320200048F66899
:10447000652050202020202020202000416C7469DD
:104480007475646520502020202000486F6F677489
:10449000652050202020202020004C756674647216
:1044A00075636B2044202020004261726F6D65743B
:1044B00072696320442020004261726F6D657472DE
:1044C0002E2044202020005A2D414343202020202C
:1044D000202020202000414343205A20202020205B
:1044E0002020202000414343205A2020202020204B
:1044F000202020004D61782E2048F668652020207D
:104500002020004D61782E20416C746974756465BB
:1045100020004D61782E20686F6F67746520202021
:10452000005665727374E4726B756E672F522000CB
:104530006761696E2F72617465202020202000560B
:10454000657273742E2F726174652020200053638E
:104550006877656265676173202B2F2D00686F6F28
:104560007665722076617269612E2000686F6F76C1
:1045700065722076617269612E2000475053205A7F
:1045800020202020202020202000475053205A2087
:10459000202020202020202000475053205A202077
:1045A0002020202020202000537469636B204E655A
:1045B0007574722E205000737469636B206E65757C
:1045C00074722E205000537469636B206E6575748D
:1045D000722E2050004175746F20532F4C20436879
:1045E000616E2E004175746F20532F4C204368611B
:1045F0006E2E004175746F20532F4C204368616EFE
:104600002E004C616E646520476573636877692E80
:10461000006C616E64696E6720737065656420006C
:104620006C616E64696E6720737065656420004E0E
:1046300069636B20532E20416E73742E20006E69C7
:10464000636B2073657276206374726C006E6963AD
:104650006B2073657276206374726C004E69636BB5
:10466000204B6F6D70656E732E20006E69636B203A
:10467000636F6D70656E732E20006E69636B2063CF
:104680006F6D70656E732E2000436F6D70656E7375
:104690002E20206175732000436F6D70656E732E40
:1046A00020206F66662000436F6D70656E732E204C
:1046B000206F666620004E69636B20556D6B6568E0
:1046C00072656E20006E69636B20696E762E2064C1
:1046D00069722E006E69636B20696E762E72696353
:1046E000682E004E69636B20536572766F20726589
:1046F0006C006E69636B20736572766F2072656CF7
:10470000006E69636B20736572766F2072656C0052
:104710004E69636B20536572766F206D696E006E13
:1047200069636B20736572766F206D696E006E69C8
:10473000636B20736572766F206D696E004E6963DE
:104740006B20536572766F206D6178006E69636BC4
:1047500020736572766F206D6178006E69636B20DF
:10476000736572766F206D6178004E69636B2053BC
:104770006572762046696C74004E69636B205365E0
:1047800072762046696C74004E69636B20536572C3
:10479000762046696C7400526F6C6C20532E204159
:1047A0006E73742E2000726F6C6C207365727620AD
:1047B0006374726C00726F6C6C2073657276206328
:1047C00074726C00526F6C6C204B6F6D70656E7301
:1047D0002E2000726F6C6C20636F6D70656E732E8F
:1047E0002000726F6C6C20636F6D70656E732E208D
:1047F00000526F6C6C20556D6B656872656E2000A1
:10480000726F6C6C20696E762E206469722E007255
:104810006F6C6C206F6D6B6572656E202000526F3F
:104820006C6C20536572766F206D696E00726F6CD0
:104830006C20736572766F206D696E00726F6C6CA0
:1048400020736572766F206D696E00526F6C6C20FC
:10485000536572766F206D617800726F6C6C207397
:104860006572766F206D617800726F6C6C20736575
:1048700072766F206D617800526F6C6C2053657298
:10488000762046696C7400526F6C6C2053657276AA
:104890002046696C7400526F6C6C205365727620F0
:1048A00046696C7400416E73742E204765736368AB
:1048B000772E2000736572766F207265667265735D
:1048C000682000536572766F207265667265736842
:1048D00020004D616E75656C6C652047657363687B
:1048E000006D616E75656C6C2053706565642000A9
:1048F000536E656C682E68616E646265642E004359
:10490000616D205269636874756E67202000436191
:104910006D204F7269656E74202020200043616D08
:104920006572612072696368742E20005365727627
:104930006F20332020202020202000536572766FC6
:1049400020332020202020202000536572766F2005
:10495000332020202020202000536572766F2034E1
:104960002020202020202000536572766F203420E4
:1049700020202020202000536572766F20342020D4
:10498000202020202000536572766F2035202020C3
:104990002020202000536572766F203520202020B3
:1049A00020202000536572766F20352020202020A3
:1049B000202000475053202020202020202020208D
:1049C0002000656E61626C652047505320202020D6
:1049D00000656E61626C65204750532020202000E6
:1049E000475053204D6F6475732053742E20004739
:1049F0005053206D6F646520636F6E747200475072
:104A000053206D6F646520636F6E7472004750535E
:104A1000205665727374E4726B2E20004750532049
:104A20004761696E202020202020004750532076C7
:104A30006572737465726B2E200047505320537457
:104A40002E20536368772E200047505320737469DB
:104A5000636B2074687265004750532073742E2076
:104A60006472656D702E004D696E2E205361742E38
:104A70002020202020004D696E2E205361742E20AE
:104A800020202020004D696E2E205361742E20209E
:104A9000202020004750532D50202020202020206F
:104AA0002020004750532D5020202020202020205F
:104AB00020004750532D502020202020202020204F
:104AC000004750532D492020202020202020200066
:104AD0004750532D4920202020202020202000470F
:104AE00050532D49202020202020202020004750F6
:104AF000532D4420202020202020202000475053E8
:104B00002D44202020202020202020004750532DFD
:104B1000442020202020202020200050204C696D9F
:104B2000697420202020202020004C696D697420A9
:104B30002050202020202020004C696D69657420C1
:104B4000205020202020200049204C696D697420CD
:104B5000202020202020004C696D697420204920ED
:104B60002020202020004C696D6965742020492098
:104B7000202020200044204C696D697420202020D2
:104B8000202020004C696D697420204420202020C2
:104B90002020004C696D696574202044202020206D
:104BA00020004750532041636320202020202020F4
:104BB0000047505320416363202020202020200004
:104BC00047505320416363202020202020200047AD
:104BD00050532057696E646B6F72722E20004750DD
:104BE000532057696E6420436F72722E00475053F2
:104BF0002057696E6420436F72722E004272656D99
:104C0000737769726B756E672020005370656564F9
:104C100020636F6D70656E732E0052656D776572DF
:104C20006B696E672020202000475053206D61780B
:104C30002E205261642E2000475053206D61782E43
:104C400072616469757300475053206D61782E72EC
:104C50006164697573004750532057696E6B656CCA
:104C6000204C692E0047505320616E676C2E6C6992
:104C70006D69740047505320686F656B206C696DD7
:104C80002E20005048204C6F67696E2074696D6556
:104C900020005048206C6F67696E2074696D652034
:104CA000005048206C6F67696E2074696A64200048
:104CB00044796E616D6963205048202020200044B3
:104CC000796E616D6963205048202020200044796E
:104CD0006E616D69736368652050482000475053CA
:104CE000206D2E20526164206450480047505320AC
:104CF0006D2E205261642064504800475053206D4F
:104D00002E20526164206450480043482048F668D1
:104D1000652020202020202000434820416C746919
:104D20007475646520202000434820486F6F6774C5
:104D3000652020202020004C454431204269746DBC
:104D400061736B6520004F757431204269746D6129
:104D5000736B20200055697467312042697470615B
:104D600074722E00202020202054696D696E672007
:104D70002020004F7574312054696D696E672020C2
:104D8000200055697467312054696D696E67202071
:104D9000002020202020736F666F727420616E00E7
:104DA00041637469762020202020202020200044A8
:104DB00069726563742061616E20202020002020CC
:104DC0002020206E2E6D2E4D6F746F720041637423
:104DD0002E2077692E204D6F746F7200416B742EF8
:104DE000206D6F746F7220756974006D697420573F
:104DF000502D4576656E74202000636F6D622E2005
:104E000057502D4576656E7400636F6D622E205786
:104E1000502D4576656E74004175746F54722E2066
:104E20006D2F506F7469004175746F54722E206D30
:104E30002F706F7469004175746F54722E206D2F3E
:104E4000706F7469004C454432204269746D61731F
:104E50006B6520004F757432204269746D61736B0D
:104E60002020005569746732204269747061747241
:104E70002E00202020202054696D696E672020209C
:104E8000004F7574322054696D696E6720202000D0
:104E900055697467322054696D696E67202000205F
:104EA00020202020736F666F727420616E00416352
:104EB0007469762020202020202020200044697260
:104EC0006563742061616E20202020002020202056
:104ED000206E2E6D2E4D6F746F72004163742E2004
:104EE00077692E204D6F746F7200416B742E206DA8
:104EF0006F746F7220756974004F75743120566D30
:104F0000696E2E5761726E004F75743120756E6434
:104F10006572766F6C74005569746731206F6E64CA
:104F2000657273702E004F75743220566D696E2E47
:104F30005761726E004F75743220756E64657276BB
:104F40006F6C74005569746732206F6E646572739C
:104F5000702E004D696E2E20476173202020202086
:104F600020006D696E2E207468726F74746C6520F9
:104F7000004D696E696D61616C206761732020006E
:104F80004D61782E20476173202020202020006D65
:104F900061782E207468726F74746C6520004D61A6
:104FA00078696D61616C206761732020004B6F6DC3
:104FB000706173737769726B756E6700636F6D7084
:104FC00061737320656666656374004B6F6D706115
:104FD000732065666665637420004B6F6D70617346
:104FE000736F66667365742000636F6D70617373B1
:104FF000206F6666736574004B6F6D706173206F10
:10500000666673657420004469732E6465636C6919
:105010006E2E63616C004469732E6465636C696E07
:105020002E63616C004469732E6465636C696E2E37
:1050300063616C0043617265667265652053742E0E
:105040002020004361726566726565204374726C4E
:1050500020004361726566726565204374726C203E
:1050600000546561636861626C652043617265002C
:10507000546561636861626C6520436172650054C8
:105080006561636861626C65204361726500556E9D
:105090007465727370616E6E756E672000756E64F4
:1050A0006572766F6C746167652020004F6E646571
:1050B000727370616E6E696E6720004175746F6CFB
:1050C000616E642E20566F6C74006175746F6C6134
:1050D0006E6420766F6C7420006175746F6C616E05
:1050E0006420766F6C742000566F6C742052656675
:1050F0006572656E7A2000566F6C74205265666525
:1051000072656E7A20005265662E207370616E6E35
:10511000696E6720004E6F7420476173205A65697D
:1051200074202000456D6572672E5468722E546994
:105130006D65004E6F6F64206761732074696A64E7
:1051400020004E6F742047617320202020202020F3
:1051500000456D6572672E5468726F74746C6500DB
:105160004E6F6F642067617320202020202000464E
:1051700061696C732E2043482054696D6500466157
:10518000696C732E2043482054696D65004661693F
:105190006C732E2043482054696A64004661696C30
:1051A000732E204368616E6E656C004661696C7396
:1051B0002E204368616E6E656C004661696C732ECB
:1051C000204368616E6E656C006B2E53756D6D6566
:1051D00072206F2053656E006E20626565702061DD
:1051E000637420545820004765656E2062656570C1
:1051F000207A20545800566172696F206661696C8C
:1052000020416C7400566172696F206661696C2080
:10521000416C7400566172696F206661696C20414F
:105220006C7400436F6D70617373204572726F729E
:105230002000436F6D70617373204572726F72202E
:10524000004B6F6D706173204572726F7220200089
:105250006B2E5374617274206F2E53442D4B006E6D
:105260002073742E207774686F2053442000472EDB
:105270007374617274207A2E20534420006B2E5375
:1052800074617274206F2E47505320006E20737427
:105290002E207774686F2047505300472E73746137
:1052A0007274207A2E20475053004779726F205035
:1052B0002020202020202020004779726F205020BD
:1052C00020202020202020004779726F20502020AD
:1052D000202020202020004779726F2049202020A4
:1052E0002020202020004779726F20492020202094
:1052F00020202020004779726F2049202020202084
:10530000202020004779726F204420202020202078
:105310002020004779726F20442020202020202068
:1053200020004779726F2044202020202020202058
:105330000047696572205020202020202020200076
:105340004C616365742050202020202020200047DD
:1053500069657220502020202020202020004769ED
:10536000657220492020202020202020004C6163ED
:105370006574204920202020202020004769657284
:10538000204920202020202020200044796E616DBB
:1053900069736368652053742E0064796E616D696A
:1053A000632073746162692E0044796E616D697364
:1053B0002E20737461622E00447265687261746598
:1053C0006E6265672E2000526F7452617465206CA6
:1053D000696D69742E00546F6572656E74616C201E
:1053E0006C696D2E004143432F4779726F204661EF
:1053F0006B2E20004143432F4779726F2046616333
:105400007420004143432F4779726F2046616374D3
:1054100020004143432F4779726F204B6F6D702EF0
:1054200000436F6D70204143432F4779726F200016
:10543000436F6D70204143432F4779726F200048BE
:10544000617570747265676C6572204920004D61EA
:10545000696E2049202020202020202000486F6FE6
:105460006664726567656C2E204920004472696627
:105470006B6F6D70656E7361742E00647269667413
:1054800020436F6D70656E732E00447269667420E0
:10549000636F6D70656E732E004779726F20737441
:1054A00061622E20202020004779726F2073746182
:1054B00062696C697479004779726F2073746162F4
:1054C000696C69742E004D6F746F7220736D6F6F0D
:1054D00074682020004D6F746F7220736D6F6F744D
:1054E000682020004D6F746F7220736D6F6F746849
:1054F000202000506172616D65746572203120203A
:105500002000506172616D65746572203120202029
:1055100000506172616D6574657220312020200039
:10552000506172616D6574657220322020200050D8
:105530006172616D657465722032202020005061B7
:1055400072616D6574657220322020200050617296
:10555000616D657465722033202020005061726196
:105560006D65746572203320202000506172616D7A
:1055700065746572203320202000506172616D6572
:10558000746572203420202000506172616D657452
:105590006572203420202000506172616D65746551
:1055A00072203420202000506172616D6574657234
:1055B000203520202000506172616D657465722075
:1055C0003520202000506172616D65746572203550
:1055D00020202000506172616D6574657220362054
:1055E000202000506172616D657465722036202044
:1055F0002000506172616D65746572203620202034
:1056000000506172616D6574657220372020200042
:10561000506172616D6574657220372020200050E2
:105620006172616D657465722037202020005061C1
:1056300072616D657465722038202020005061729F
:10564000616D6574657220382020200050617261A0
:105650006D657465722038202020004163687328CE
:10566000652E296B6F70706C2E0028446529436F7E
:1056700075706C2041786573004173206B6F70709A
:10568000656C696E672020004769657220706F73D2
:105690002E204B6F707000526574726F6163206CC6
:1056A0006163657420004769657220706F732E20F6
:1056B0006B6F702E004E69636B2F526F6C6C204BBA
:1056C0006F707000526574726F20726F756C2F74FA
:1056D000616E004E69636B2F526F6C6C206B6F7044
:1056E0002E0047696572204B6F7272656B7475721C
:1056F00000436F7272656374206C6163657420008F
:105700004769657220636F72726563746965004FE3
:105710007269656E74696572756E672020004F72DC
:1057200069656E74696572756E672020004F7269D5
:10573000656E7461746965202020200048F66865F4
:105740006E726567656C756E672000416C74697474
:10575000756465204374726C2000486F6F677465D0
:1057600020436F6E74722E2000536F6C6C68F66865
:105770006520202020202000536574706F696E74AE
:1057800020202020202000476577656E73742E68E6
:105790006F6F67746500537469636B204E65757431
:1057A000722E205000737469636B206E657574727D
:1057B0002E205000537469636B206E657574722ED1
:1057C000205000475053202020202020202020203F
:1057D0002000656E61626C652047505320202020B8
:1057E00000456E61626C65204750532020202000E8
:1057F000475053204D6F6475732053742E2000471B
:105800005053206D6F646520636F6E747200475053
:1058100053206D6F646520636F6E74720044796EFF
:10582000616D6963205048202020200044796E611A
:105830006D6963205048202020200044796E616DFE
:105840006963205048202020200043482048F66803
:1058500065202020202020200043482048696768D8
:105860002020202020202000434820686F6F67748C
:1058700065202020202000436172656672656520E6
:1058800053742E2020004361726566726565204363
:1058900074726C20004361726566726565204374A2
:1058A000726C2000546561636861626C65204361BD
:1058B000726500546561636861626C652043617262
:1058C0006500546561636861626C6520436172655F
:1058D000004D6F746F7220536963682E53636800C4
:1058E0004D6F742E5361666574792053772E004D89
:1058F0006F742E7361662E736368616B2E004F7236
:1059000069656E74696572756E672020004F7269F3
:10591000656E746174696F6E202020004F72696536
:105920006E7461746965202020200000000110035E
:105930000101010000011004040404000001100131
:10594000030303000001100202020200030020050D
:1059500005050500030020060606060003002007D3
:1059600007070700030020080808080003002009B3
:10597000090909000300200A0A0A0A000300200B93
:105980000B0B0B000300200C0C0C0C0007001E641A
:105990000000000002000873000000000200047212
:1059A000000000000600062701010100020040730C
:1059B000000000010200010D000000010200200DA6
:1059C000010101010200080D010101010200100D99
:1059D0000000000102000472000000010200400DFE
:1059E000010101010200800D000000010200040D10
:1059F00000000002000014170A0806020000141834
:105A000010100A020100FF19060604020100FF61DE
:105A10000000000302000170000000030200027099
:105A20000000000302000470000000030200087080
:105A3000000000030100FF3B323232030000F73C5C
:105A40005A5A5A030000F73D323232030000F74140
:105A50004E4E4E030000F7424E4E4E040200010D22
:105A60000000000402000172000000040200020DA8
:105A700001010104020002720101010407001F106C
:105A8000000000040000F70E1E1E1E040100FF119E
:105A90000F0F0F040100FF0F1E1E1E040100FF1355
:105AA000000000040100FF68969696040000F712BB
:105AB0000F0F0F040000F714080808040100FF1579
:105AC000404040040000A0160000000407001C6CC9
:105AD000000000040000F76D090909050100FF2D11
:105AE000808080050100F72E32323205020080737B
:105AF00000000005020001710000000502000471B1
:105B0000000000050000F72F0F0F0F050000F73011
:105B1000E6E6E6050000196A000000050100FF3115
:105B2000808080050000F73255555505020002714E
:105B3000000000050000F733464646050000F73434
:105B4000DCDCDC050000196B0000000500020835F4
:105B5000040404050000F7363C3C3C050500F7371B
:105B6000000000050100FF387D7D7D050100FF3943
:105B70007D7D7D050100FF3A7D7D7D060200200DC3
:105B80000101010608002051000000060100FF523B
:105B9000646464060000F75B080808060000F75A12
:105BA000060606060100FF535A5A5A060100FF5422
:105BB0005A5A5A060100FF555A5A5A060100FF5612
:105BC0004B4B4B060100FF57555555060100FF583A
:105BD0004B4B4B060100FF59000000060100FF5C23
:105BE0005A5A5A060100FF5D2A2A2A060100FF5E62
:105BF000F5F5F5060100FF5F8C8C8C060000F76060
:105C0000050505060200207200000006020002736E
:105C1000000000060000F766000000070400FF4ACD
:105C20005F5F5F070100FF4B141414070200207030
:105C3000000000070200107001010107020020733C
:105C4000000000070100FF50000000070400FF4CA7
:105C5000F3F3F3070100FF4D141414070200407022
:105C60000000000702008070010101070400FF4EE0
:105C7000AAAAAA070400FF4FAAAAAA080000F71AB6
:105C8000080808080000F71BE6E6E6080100FF1D0B
:105C90004040400809003C6E3C3C3C080A003C6E19
:105CA0003C3C3C0807001F630000000802004072F3
:105CB000000000080000F724212121080000F76FF0
:105CC0002020200802000872000000080000F726CB
:105CD0005A5A5A080000F7252D2D2D080000F767A5
:105CE0000000000800000C690000000802001072AB
:105CF0000000000802000473000000080200807227
:105D00000000000802000173000000080200107388
:105D1000000000090100FF1E5A6464090100FF1F12
:105D2000787878090100FF200A0A0A090100FF219A
:105D30005A6464090100FF22787878090100FF4560
:105D4000464646090200800D000000090000F71CCD
:105D50001B1B1B090000F743202020090100FF281E
:105D6000101010090000F744000000090000102383
:105D7000060606090000F7650000000A0100FF2979
:105D80000000000A0100FF2A0000000A0100FF2BAA
:105D90000000000A0100FF2C0000000A0100FF467D
:105DA0000000000A0100FF470000000A0100FF4850
:105DB0000000000A0100FF490000000B0200400D36
:105DC0000000000B0100FF3E5A5A5A0B0100FF3F32
:105DD0003737370B0100FF404646460C0500176277
:105DE0000000000D0200010D0000000D0100FF1079
:105DF000FFFFFF0D0000A0160000000D0200200DA7
:105E00000101010D0100FF51FEFEFE0D0200207296
:105E10000000000D0000F7660000000D0100FF63A8
:105E20000000000D020040720000000D00000C6434
:105E30000000000D0500176200000050504D2020AA
:105E40002020202020202020202020005370656B5F
:105E50007472756D20202020202020200053706552
:105E60006B7472756D204869526573202000537001
:105E7000656B7472756D204C6F5265732020004AFB
:105E80006574692020202020202020202020200050
:105E90004143542044534C20202020202020202007
:105EA00000484F5454202020202020202020202053
:105EB000200046757475626120534255532020209E
:105EC00020200055736572202020202020202020D3
:105ED000202020001300120013005553520053429B
:105EE0005500486F5400414354004A657400537094
:105EF0004C00537048005370650050504D002050C6
:105F00004800204348004672656500204F6E004FF0
:105F10006666004D6178004D6964004D696E0057FA
:105F2000504500446973004F6666005300430020EB
:105F3000204E0020204A00205000200025001200A2
:105F40001300120020001200300031002019202020
:105F50002020301149202020456E64652020204FEC
:105F60004B005048202020202020202000434820A3
:105F7000202020202020200046726565202020203F
:105F8000202020005750204576656E742020005355
:105F90006572436820202020004368616E6E656C46
:105FA000202020200044697361626C656420200019
:105FB0005374642E00442C312D5331322F572F4609
:105FC0002F432F5028643A2029004F6E2020202094
:105FD00020202020004F6666202020202020200046
:105FE0005750204576656E742020005365724368D3
:105FF00020202020004368616E6E656C20202020E8
:106000000044697361626C65642020005374642EDF
:10601000004469732C312D5331322F572F4F2028D4
:10602000643A202029004F6666202020202020206E
:10603000004D6178696D756D2020004D6964646C58
:1060400065202020004D696E696D756D2020005718
:1060500050204576656E7420200053657243682099
:10606000202020004368616E6E656C202020200097
:106070005374642E00312D5331322F572F3C2F7C17
:106080002F3E2028643A202029001D0020002000F7
:106090001D002A002A00506F00506F202900537401
:1060A000642E0028302D3234372D50382928643A98
:1060B000506F2029005374642E00282020202D20AA
:1060C0002020292028643A20202029004B6F706965
:1060D00065727420756E6420416B746976696572AF
:1060E00074005769726B6C696368204B6F706965E7
:1060F00072656E3F00323030382054686F6D6173C6
:10610000204B616973657200323030392D32303185
:1061100030205065746572204D61636B0032303100
:10612000302053656261737469616E20426F6568E7
:106130006D00323031322067656261640032303187
:1061400032204D617274696E2052756E6B656C0001
:106150002020202020486172616C6420426F6E67AD
:106160006172747A0032303132204368722E2042DC
:1061700072616E64746E65720032303133204F6C20
:10618000697665722047656D6573690020437265A5
:10619000646974730000466F6E7420426967004F33
:1061A000534420537461746973746963004F53449A
:1061B0002033442D4C616765004F5344205573656F
:1061C00072475053004F5344204D4B5374617475C4
:1061D00073004F534420456C656374726963004FCC
:1061E0005344204E617669676174696F6E004F5346
:1061F00044204F6C642053637265656E73004932AE
:1062000043204D6F746F7274657374004A6F7973B5
:106210007469636B00574C414E205779466C790086
:10622000466F6C6C6F77204D6500547261636B69CB
:106230006E6700536F756E64004D4B204469737038
:106240006C6179004D4B2044656275672044617430
:1062500061004D4B20506172616D65746572004F35
:1062600053442D4461746100204D6F64756C6573F7
:1062700020696E7374616C6C656400253135532040
:106280002534530000202020204E4F2057415252E9
:10629000414E54590028432920474E552047504C21
:1062A000204C6963656E73650000332E372E3363AF
:1062B00058330020504B5420762538532025730046
:1062C00020504B542055706461746520202020209C
:1062D00020202020200020202020202055706461D4
:1062E00074653F2020202020202020005665726207
:1062F000696E64756E67204D4B00636F6E6E6563EB
:1063000074696F6E204D4B0041616E736C756974DA
:10631000696E67204D4B00504B5420616C6C676573
:106320006D65696E00504B5420676C6F62616C0044
:10633000504B5420616C67656D65656E0057692E22
:1063400032333200426C7565746F6F746800576C3D
:10635000616E004F534420416E7A65696765004F56
:1063600053442073637265656E004F53442073631A
:106370006865726D00475053204D6175730047503A
:1063800053206D6F75736500547261636B696E673E
:1063900020536572766F7300747261636B696E6708
:1063A00020736572766F73004A6F79737469636BDB
:1063B00000504B542055706461746500454550721F
:1063C0006F6D205265736574004F534420536372A0
:1063D00065656E7300504B5420536574757000539F
:1063E000707261636865006C616E677561676500F6
:1063F0005461616C005A6569747A6F6E65007469E6
:106400006D65207A6F6E6500536F6D6D65727A658C
:1064100069740073756D6D65722074696D65004CEB
:10642000434420617573206E6163682E2E2E004CEC
:106430004344206F6666206166746572004C434475
:1064400020756974206E612E2E2E004C4344204826
:10645000656C6C69676B656974004C4344206272BB
:10646000696768746E657373004C43442048656CBB
:1064700064657268656964004C4344204B6F6E74B8
:1064800072617374004C434420636F6E7472617365
:1064900074004C434420436F6E7472617374004CFB
:1064A0004344204E6F726D616C2F496E7665727336
:1064B000004C4344206E6F726D616C2F696E76657F
:1064C0007274004C4344204E6F726D61616C2F6793
:1064D00065696E7600486172647761726520426515
:1064E00065706572004861726477617265207069D9
:1064F0006570657200416B6B757479700041636300
:1065000075747970006163637520747970650041FA
:106510006B6B75204D657373756E670041636375B2
:106520004D6561737572650061636375206D657497
:10653000696E6700504B5420616C6C67656D6569CE
:106540006E0054582F5258204B616E616C005458A5
:106550002F5258204368616E6E656C004E6574570B
:106560002E20477275707065004E6574572E204757
:10657000726F7570004E6574572E204D6F64650004
:1065800054582054696D656F7574005458204D54EB
:106590005500426175647261746520576932333207
:1065A0002F425400496E697469616C697369657240
:1065B000656E00696E697469616C697A6500496E1F
:1065C000697469616C69736572656E004B6F6E66A4
:1065D00069672E206D697420504300636F6E666991
:1065E000672E207769746820504300436F6E666998
:1065F000672E206D65742050430057692E32333268
:10660000205365747570002052452D4944204E6F0B
:1066100074697A202020202020202020003A004D7C
:1066200041433A002042544D2D323232204D4143F5
:106630002D416472657373652000425420496E6970
:1066400074204572726F7200425420496E69742042
:106650006F6B0020426C7565746F6F7468205069B1
:106660006E202020202020200020426C7565746F51
:106670006F7468204E616D65202020202020004D21
:106680006F64756C2065696E6765626175743F0043
:106690006D6F64756C65206275696C7420696E3FFE
:1066A000004D6F64756C65206765696E7374616C0D
:1066B0002E3F004E616D65006E616D65004E61613B
:1066C0006D0050696E0070696E00426C7565746F84
:1066D0006F7468204D41430052452D494400426C7F
:1066E0007565746F6F7468205365747570005375A9
:1066F00063686520475053204D6175730073656171
:1067000072636820475053206D6F757365005A6F30
:10671000656B204750532D6D756973005A65696725
:106720006520476572E474656C697374650073680D
:106730006F77206465766963656C6973740053686C
:106740006F772061707061726161746C697374003D
:106750005A656967652047505320446576696365CB
:106760000073686F772047505320646576696365CE
:106770000053686F772047505320617070617261D9
:10678000617400475053204D617573205479700037
:10679000475053206D6F757365207479700054797C
:1067A0007065204750532D6D756973004750532015
:1067B0004D61757320616B7469763F0047505320BB
:1067C0006D6F7573652061637469763F0047505340
:1067D0002D6D75697320616B746965663F00475064
:1067E0005320446174656E004750532064617461A6
:1067F00000475053204D6F75736520536574757055
:10680000004F53442053637265656E73004F5344C9
:1068100020536574757000566F6C740020464548AF
:106820004C45522120312E205A65696368656E21DE
:106830002000201720202020201620202020201992
:10684000202020204F4B002020202020202020200E
:1068500020202020430020002500576932333200D9
:106860005769323332004C69496F6E004C69706F62
:1068700020005750412020004164686F6300343885
:10688000303020200031313532303000353736306D
:10689000302000333834303020003139323030206D
:1068A0000039363030202000323430302020004D86
:1068B000696B726F6B6F70740042542D4D6F7573FE
:1068C00065310062697474652077617274656E2E3B
:1068D0002E2E00475053207472656E6E656E006CEC
:1068E0006F73742042542064617461006D00202035
:1068F0002D2D2D00416C743A2000204C6174697478
:106900007564652020204C6F6E676974756465003E
:1069100048444F503A20004669783A200058457262
:10692000723A20005361743A20004F4B0045727256
:106930006F7220636F6E6E656374696E6721007499
:10694000727920746F20636F6E6E656374006B6F75
:106950006E66696775726965727421006B65696E30
:106960006520475053204D617573007375636865EA
:106970002042542044657669636500425420446592
:1069800076696365732073756368656E3F00616B3C
:106990007475656C6C657320425420446576696338
:1069A000653A200042542073656C65637420446529
:1069B000766963650073756368656E21004269746A
:1069C000746520657273742042542D446576696342
:1069D0006573004D41433A004465766963653A004A
:1069E00065696E67656261757421006B65696E200B
:1069F00042544D323232004F4B00194F1800207371
:106A0000657269656C6C6520506F74697320312DF7
:106A1000352000DC62657273696368740073756D9C
:106A20006D61727900537469636B2031007374690E
:106A3000636B203100537469636B20320073746997
:106A4000636B203200537469636B20330073746985
:106A5000636B203300537469636B20340073746973
:106A6000636B203400537469636B20350073746961
:106A7000636B203500504B54204C69706F6D65730B
:106A800073756E6700504B54204C69706F206D65B4
:106A900061737572652E00504B54204C69506F2005
:106AA0006D6574696E67004A6F79737469636B739F
:106AB000205365747570004D696E696D616C205767
:106AC000657274006D696E696D616C2076616C75BC
:106AD00065006D696E696D2E207761617264650075
:106AE0004D6178696D616C2057657274006D6178D5
:106AF000696D616C2076616C7565006D6178696D9A
:106B00002E20776161726465005479706500747934
:106B10007065005269636874756E670064697265B8
:106B20006374696F6E007269636874696E67004EA2
:106B300065757472616C69736965726564006E6510
:106B4000757472616C697A696E67006E65757472CE
:106B5000616C69736572656E64004A6F79737469FC
:106B6000636B004F4B00504B54204C69706F6D6548
:106B70007373756E672020200059004E00526576B1
:106B8000004E6F726D005461737400506F74690031
:106B900053204D696E204D61782054797020204437
:106BA000697220204E002020204A6F797374696337
:106BB0006B20536574757020202020005556F732E5
:106BC000EE1AAB0DDC066F03B801DC006E00370077
:106BD0001B000E00070003000200010053657276DF
:106BE0006F736368726974746500736572766F2081
:106BF000737465707300536572766F20310073652E
:106C000072766F203200536572766F2032007365A2
:106C100072766F203200536572766F7465737400FC
:106C2000736572766F7465737400547261636B6917
:106C30006E6720536572766F7300546573742050CD
:106C4000756C736CE46E67650074657374207075A1
:106C50006C73207769647468005465737420666F80
:106C600072746C66642E007465737420636F6E7446
:106C70002E00536572766F00736572766F005065F3
:106C800072696F6465006672616D65005365727646
:106C90006F746573740053746172742054657374F7
:106CA00000737461727420746573740045696E7A40
:106CB000656C736368726974740073696E676C6580
:106CC000207374657000416E7A61686C205465733E
:106CD00074006E756D626572206F662074657374E2
:106CE0000061616E74616C2074657374730050612F
:106CF00075736520456E64706F736974696F6E009B
:106D0000706175736520656E6420706F73007061CB
:106D10007573652065696E6420706F732E00506115
:106D20007573652070726F20496E632E00706175F7
:106D300073652070726F6320696E632E00536572F5
:106D4000766F7465737420436F6E742E005265768F
:106D5000657273650072657665727365004C696E65
:106D60006B73006C656674006C696E6B73005265C2
:106D7000636874730072696768740072656368742D
:106D800073004D69747465006D6964646C65006DB1
:106D9000696464656E00536572766F2041646A753C
:106DA000737400536572766F203200536572766F8C
:106DB000203100536572766F3A00010000000A002E
:106DC000000064000000E803000010270000A08617
:106DD000010040420F008096980000E1F50500CACE
:106DE0009A3B456E64650020547261636B696E67FF
:106DF000204D696B726F6B6F7074657200547261B5
:106E0000636B696E6720426C7565746F6F74682080
:106E10002020006C6F73742057692E323332206447
:106E200061746100475053206F6B2C207374617242
:106E300074206F6B20200020202020202020202084
:106E40002020202020202020200057686169742005
:106E5000666F72204750532046697820005768615A
:106E6000697420666F72204750532046697820006D
:106E700053204C6174697475646520204C6F6E6793
:106E80006974756465004665686C65722062656941
:106E90006D205472656E6E656E00737769746368F9
:106EA000206F6E204254204D6F757365212100457F
:106EB00072726F7220617420636F6E6E65637469A5
:106EC0006E6700475053207472656E6E656E006C7D
:106ED0006F737420425420646174610048444F50C1
:106EE0003A004669783A005361743A004D00480010
:106EF00053204C6174697475646520204C6F6E6713
:106F00006974756465004641494C00204F4B200070
:106F1000203F3F200054696C743A0050616E203A63
:106F2000006D00446973743A001E00426561723A54
:106F300000256325632531377320002563256325EC
:106F400031367325632000256325632531375320AF
:106F500000256325632531365325632000253553ED
:106F60000025345300202532307300202532305361
:106F7000002020253139730020202531395300208D
:106F8000202020206E6F7420706F737369626C65AF
:106F90002020202000204552524F525F4E4F49542E
:106FA000454D202000204552524F525F4D415849D7
:106FB00054454D2000204552524F525F4D41584D8F
:106FC000454E552000204552524F525F4E4F4D4581
:106FD0004E55202000130012001D0020002020200C
:106FE00020206E6F7420706F737369626C6520204F
:106FF00020200020202020004E6F206D6F72652021
:1070000052414D004572726F723A205363726F6C39
:107010006C426F780057692E323332204E414B005C
:10702000576932333220496E69744572726F72202B
:107030002000576932333220496E6974206F6B2EFD
:107040002E2E2E00576932333220496E69744572F4
:10705000726F722020002E002E002E002E002E00B7
:107060002E002E002E002E002E002E002E002E00B0
:107070002E002E002E002E002E002E00496E697468
:1070800020576932333220776169742E2E2E2E00FC
:1070900056657273696F6E3A004572726F72207333
:1070A00065742052414D2020202020004572726FCF
:1070B0007220736574204E562D52414D0057692E33
:1070C0003233322077726F6E67204261756472616D
:1070D00074650057692E32333220666F756E6420F6
:1070E0000057692E32333220537974617865727299
:1070F0006F72202020006E6F2057692E32333220AD
:10710000666F756E64007365617263682057692EDF
:10711000323332204D6F64756C003131353230308E
:1071200000203537363030002033383430300020FE
:1071300031393230300020203936303000202032D2
:1071400034303000207769746820202020202020EF
:107150002042617564006765742069700D004950B4
:107160003D004E4D3D0047573D00484F53543D00B4
:10717000444843503D00676574206D61630D004DC8
:10718000616320416464723D0067657420776C61BF
:107190006E0D00535349443D004368616E3D0067E6
:1071A0006574206F70740D00446576696365496489
:1071B0003D0067657420750D0042617564726174ED
:1071C000653D006765742074696D650D005A6F6ECA
:1071D000653D0073686F772074696D650D005570AB
:1071E00054696D653D0054696D653D0067657420A7
:1071F000646E730D00416464726573733D0073685F
:107200006F77207420740D005254433D004D6F641D
:10721000653D0067657420636F6D6D0D00466C758C
:10722000736854696D65723D004D617463684368AD
:1072300061723D00466C75736853697A653D0073F1
:10724000686F7720727373690D00525353493D285C
:107250002D00464C4147533D30780050524F544F1B
:107260003D00676574206164686F630D004265616D
:10727000636F6E3D0050726F62653D005265626FD4
:107280006F743D004A6F696E3D00526174653D0048
:107290005478506F7765723D005265706C6163651C
:1072A0003D007665720D005769466C7900414F4B81
:1072B0000D0A004552523A200055736520636F6EE7
:1072C0006669672077697468205043005769466C87
:1072D000792046696E644572726F720073656172DF
:1072E0006368203234303020426175640073656118
:1072F00072636820343830302042617564007365F1
:107300006172636820313932303020426175640027
:1073100073656172636820333834303020426175A0
:10732000640073656172636820313135323030201A
:10733000426175640073656172636820393630306C
:107340002042617564007365617263682057694605
:107350006C7900736574207561727420696E737442
:10736000616E74007365742075617274206261755A
:10737000640031313532303000353736303000334B
:107380003834303000313932303000393630300066
:107390003438303000323430300073657420697016
:1073A0002067617465776179007365742069702066
:1073B0006E65746D61736B0073657420697020680D
:1073C0006F7374002A5265626F6F742A007265626F
:1073D0006F6F740D0073657420697020616464724E
:1073E0006573730073657420776C616E206A6F69D2
:1073F0006E0073657420776C616E20686964652027
:10740000310073657420776C616E207068726173EF
:10741000650073657420776C616E206B657900730D
:10742000657420776C616E206368616E00736574AB
:1074300020697020646863700073657420776C61E4
:107440006E207373696400455849540D0A006578CD
:1074500069740D003C74696D656F75743E00414F31
:107460004B0D0A004552523A200053746F72696EF8
:107470006700736176650D004661696C20496E692D
:1074800074204164686F632000496E697420416410
:10749000686F63204E6574776F726B00462073656A
:1074A0007420636F6D6D2072656D00736574206369
:1074B0006F6D6D2072656D6F7465203000462074AD
:1074C00075726E206F6666206563686F0073657401
:1074D0002075206D2031004572726F7220536574E3
:1074E0004261756472617465005769466C79206EFB
:1074F0006F7420666F756E6400434D440D0A00245E
:10750000242400434D440D0A0024242400576C61B8
:107510006E20496E6974204572726F7200576C61FB
:107520006E20496E6974206F6B00576C616E204944
:107530006E69742000202020202020576C616E206E
:1075400053534944202020202020004D6F64756C47
:107550002065696E6765626175743F006D6F647563
:107560006C65206275696C7420696E3F004D6F64B4
:10757000756C65206765696E7374616C2E3F00538E
:10758000534944004B616E616C006368616E6E65C7
:107590006C0070617373776F726400496E6974690F
:1075A000616C6973696572656E00696E69746961A1
:1075B0006C697A6500496E697469616C697365729A
:1075C000656E004B6F6E6669672E206D6974205082
:1075D0004300636F6E6669672E2077697468205078
:1075E0004300436F6E6669672E206D6574205043BB
:1075F00000574C414E20205365747570000014BE36
:1076000088E10FB6F89480936000109260000FBE7E
:1076100011241FBEC0E0D0E4DEBFCDBF13E0A0E068
:10762000B1E0E8EEFCEE01E00BBF02C007900D9266
:10763000AC35B107D9F716E2ACE5B3E001C01D9255
:10764000A733B107E1F70E941A5B0C9472F60C9411
:107650000000E5EFFDE08191882319F08E32D9F723
:1076600006C08091F50D803211F0882331F485EF4A
:107670009DE065E273E00E9405F585EF9DE00C94C6
:1076800087E220E030E048E853E105C0FA01319795
:10769000F1F72F5F3F4F28173907C4F30895809102
:1076A000EF0D813019F410925D03089581E080930D
:1076B0005D03089523C00E9407D1BC01807022E0C1
:1076C0008030920789F022E08130920728F421E08F
:1076D0008030920779F4089524E08030920721F0F9
:1076E00028E08030920731F4809160038F5F8093AF
:1076F0006003089582E693E00E942A4482E693E0C4
:107700000E94FF438823B9F20895A1E0B0E0EBE8BE
:10771000FBE30C943EF2682E562E062D192F6E01B7
:107720000894C11CD11C28E8A22E23E1B22E94EFAC
:10773000892E91E0992E4FC0F80180810E9421D1BD
:10774000009709F44DC080911201882341F484EF21
:1077500091E0F4013197F1F70197D9F734C0813006
:1077600021F4C5010197F1F72EC0823061F58091B7
:107770005D03813041F522C09DDF81E090E081DF33
:107780000894E11CF11CFAECEF16F10431F082E6EA
:1077900093E00E94F643882379F782E693E0B601EE
:1077A0000E940A44F80180819981981791F00E9403
:1077B00021D10097A9F07A9419F40BC083E0782EB8
:1077C000EE24FF24DDCF76DF82E693E0B6010E944F
:1077D0000A440F5F1F4F802F8619851508F4ACCF20
:1077E0002196EFE00C945AF2CF93DF93C0E0D0E003
:1077F00004C060DF81E090E044DF2196C433D1050E
:10780000C1F782E693E063E272E00E945444DF91A4
:10781000CF9108951F93182F80E061E04DEA52E068
:1078200020E00E946352133011F1143028F411301B
:10783000A1F01230B8F407C0153019F11530E0F09E
:10784000163031F505C08EE061E046EA52E01DC019
:107850008EE061E04FE952E018C08EE061E048E957
:1078600052E013C08EE061E041E952E00EC08EE0CC
:1078700061E04AE852E009C08EE061E043E852E08E
:1078800004C08EE061E04CE752E020E00E946352C9
:107890001F910895FC0140E021912D3251F4228185
:1078A0002D3239F44450262F372FD90120E030E013
:1078B00005C04F5F483281F740E0F5CFFC01E20F91
:1078C000F31FE40FF11D50815D3209F44F5FFC019D
:1078D000E20FF31FE40FF11D50815D932F5F3F4FC7
:1078E0002E30310559F70895262F372FD90120E082
:1078F00030E040E0FC01E20FF31FE40FF11D508186
:107900005D3209F44F5FFC01E20FF31FE40FF11D3C
:1079100050815D932F5F3F4F2E30310559F7089509
:10792000CF93DF93E82FF92FDB0180E0EF01908107
:10793000903219F49181903231F0319698819D9373
:107940008F5F823199F780915E03680F711DFB0193
:107950001082DF91CF910895A0E0B1E0E2EBFCE36B
:107960000C9445F200E010E004C0A4DE81E090E059
:1079700088DE0F5F1F4F87E0023D180709F44FC0F4
:1079800082E693E062E471E08FD7882371F347C009
:1079900082E693E0B8013ED70F5F1F4F82E693E087
:1079A0006FE371E07ED7882399F3F8011082898113
:1079B0008823C9F1CE01019660E071E095DF40E0D7
:1079C000E42E41E0F42E35E0C32E3EE0D32E90E0CD
:1079D0008701892F66E0F70141917F0120E0C050C7
:1079E000DF4F9883C050D1400E94A352F80180819C
:1079F000F60181936F01C050DF4F9881C050D14094
:107A00009F5F9D3029F782E693E06CE371E04CD7ED
:107A1000882381F082E693E03DD781E00CC07E01AF
:107A20000894E11CF11C82E693E0E0D6882311F46F
:107A30008701B4CF80E0C050DF4FE8E00C9461F2E2
:107A4000A4E1B0E0E6E2FDE30C9443F2A82E7B0152
:107A5000E82FF0E0EA31F10508F0C1C1EA5BFF4F21
:107A60008E010F5F1F4F0C9472F2C80161EF71E03D
:107A70000E9405F58091F00D8D838091F10D8E832C
:107A80008091F20D8F838091F30D8887198684C0D1
:107A9000C8016CEE71E067C0C80167EE71E07AC0A2
:107AA000C80162EE71E076C0C8016DED71E072C090
:107AB000C80168ED71E06EC0C80163ED71E06AC095
:107AC000C8016EEC71E066C0C80169EC71E062C08B
:107AD000C80164EC71E05EC0C8016FEB71E05AC090
:107AE000C8016AEB71E056C0C80165EB71E052C095
:107AF000C80162EB71E04EC0C8016EEA71E04AC095
:107B0000C8016AEA71E046C0C80165EA71E042C096
:107B1000C80160EA71E00E9405F5F80101900020BB
:107B2000E9F731978E2D9F2DDC018CE00D900192AD
:107B30008150E1F7198A30C0C8016BE971E02AC0B1
:107B4000C80166E971E003C0C80161E971E00E9403
:107B500005F50CEA1DE022C0C8016CE871E003C025
:107B6000C80167E871E00E9405F508EB1BE016C04C
:107B7000C80162E871E00E9405F5C80165EF7DE08B
:107B80000E943FF509C0C8016DE771E003C0C8015C
:107B900068E771E00E9405F504E610E07E010894B4
:107BA000E11CF11CC70166E771E00E94FAF482DD76
:107BB00082E693E06FD6F70101900020E9F7BF015C
:107BC000615070406E197F09C7019FDD80915D0390
:107BD000882319F0EE24FF24F9C0B80180E090E07A
:107BE0000E94D5EF5B016C0120E030E44CE955E4E4
:107BF0000E94C4F0F62E172FE82E092F20E030E067
:107C000040E85FE30E9435EF87FD29C06F2D712F9B
:107C10008E2D902F20E03FEF4FE757E40E94C0F0F9
:107C20001816B4F4C601B50120E030E040E251E49A
:107C30000E94C4F00E94A9EF24EF31E005C0C90101
:107C40000197F1F76150704061157105C1F70CC0E3
:107C50006F2D712F8E2D902F0E94A9EF02C061E031
:107C600070E0CB010197F1F70E946AD182E693E0C0
:107C700011D69FC01FDDFA2DF53009F04BC0B801B9
:107C800080E090E00E94D5EF5B016C0120E030E4E1
:107C90004CE955E40E94C4F07B018C017F2D912FAB
:107CA00020E030E040E85FE30E9435EF87FD29C027
:107CB0006E2D7F2D802F912F20E03FEF4FE757E46F
:107CC0000E94C0F01816B4F4C601B50120E030E0FF
:107CD00040E251E40E94C4F00E94A9EF24EF31E099
:107CE00005C0C9010197F1F7615070406115710538
:107CF000C1F70CC06E2D7F2D802F912F0E94A9EF10
:107D000002C061E070E0CB010197F1F725DE282F7A
:107D100030E067C082E693E061E771E0C5D5882373
:107D200009F44AC0B80180E090E00E94D5EF5B0101
:107D30006C0120E030E44CE955E40E94C4F07B0182
:107D40008C017F2D912F20E030E040E85FE30E941E
:107D500035EF87FD29C06E2D7F2D802F912F20E0DC
:107D60003FEF4FE757E40E94C0F01816B4F4C60185
:107D7000B50120E030E040E251E40E94C4F00E94EE
:107D8000A9EF24EF31E005C0C9010197F1F7615077
:107D9000704061157105C1F70CC06E2D7F2D802FCD
:107DA000912F0E94A9EF02C061E070E0CB01019722
:107DB000F1F721E030E015C082E693E069E671E07A
:107DC00073D5882361F481E090E05BDC0894E11CCA
:107DD000F11C82EDE81687E0F80609F04BCF20E0B1
:107DE00030E0C9016496EAE00C945FF20F931F93B0
:107DF000CF93DF938C01C0E0D0E03CC05BDC82E637
:107E000093E068E172E050D5882349F0EDDC82E030
:107E10008093120180E060E070E012DE2FC082E605
:107E200093E060E172E040D5882359F088EE93E05A
:107E300024EF31E0F9013197F1F70197D9F781E0AB
:107E40000EC082E693E066EF71E02ED5219688237E
:107E500049F0CADC80E060E070E0F2DD82E080930F
:107E600012010EC081E090E00115110511F480E0CF
:107E700090E007DC0C171D0708F0C0CF80911201BD
:107E8000DF91CF911F910F910895A1E0B0E0EBE455
:107E9000FFE30C9445F280E090E0A8DF823059F1D6
:107EA000F4E0DF2EEBE2CE2E8E010F5F1F4F74EF5A
:107EB000E72E71E0F72EC982C80161E026DC80E17F
:107EC00097E2F7013197F1F70197D9F7DA9499F72B
:107ED00082E08093120160E070E0B2DD009789F0EB
:107EE00083E060E070E0ACDD009759F080E197E25C
:107EF0007DDF823031F482E693E0CCD421E030E0C3
:107F000002C020E030E0C9012196E8E00C9461F263
:107F1000CF93DF93EC0182E693E06AE673E040E002
:107F200052E056D4C7DB82E693E0B4D480E090E020
:107F30005DDF8130F1F080E060E070E081DD80E0C5
:107F400060E070E07DDD84E0BE017ADD009789F0BD
:107F500080E060E070E074DD81E060E070E070DDA2
:107F6000009739F080E29EE441DF21E030E081308B
:107F700011F020E030E0C901DF91CF9108951F9307
:107F8000182F82E080931201812F0E94E1D0812F6F
:107F900041DC0E946AD182E693E07CD410925D03BA
:107FA00080E062E04AE752E020E00E94635280E015
:107FB00060E070E045DD80E062E047E752E020E00D
:107FC0000E94635285E160E070E03ADD80E062E0AB
:107FD00043E752E020E00E94635286E160E070E0F7
:107FE0002FDD81E080935D0380E062E04EE652E0A9
:107FF00020E00E94635280E060E070E021DD0097A5
:1080000049F080E062E048E652E020E00E946352DE
:1080100081E008C080E062E04BE552E020E00E9491
:10802000635280E01F91089592E0909312011092A4
:108030005D03882319F186E160E070E001DD85E1F0
:1080400060E070E0FDDC80E060E070E0F9DC80E0A2
:1080500060E070E0F5DC009701F580E066E047EC59
:1080600052E020E00E94635280E395E724EF31E084
:10807000F9013197F1F70197D9F7089580E066E0AB
:108080004AEB52E020E00E94635284E160E070E03D
:10809000D7DC83E160E070E0D3CC08950F931F93A9
:1080A000182F809113011817A1F1112399F482E080
:1080B0008093120181E0B8DF89E060E070E0C0DC0D
:1080C000009701F11092130187E060E070E0B8DCE6
:1080D0003FD718C01130B1F402E00093120181E0E3
:1080E000A3DF88E060E070E0ABDC009759F010930C
:1080F00013018AE060E070E0A3DC26D780E094DF23
:108100000093120181E090911301191719F080E09A
:1081100001C081E01F910F910895AFEFB0E0E3E956
:10812000F0E40C9441F280E0B9DF882309F497C0B1
:1081300080E060E070E084DC86E060E070E080DC9D
:10814000009709F48CC0CC24DD2420E4A22E2CE975
:10815000B22E98E8892E93E1992EACDA0894C11CCE
:10816000D11CC4010197F1F782E693E03BD3AC0147
:1081700080E065E025E030E000E0EE240E945B57FF
:1081800088EEC81683E0D80671F480915E03982FBC
:108190009F5F90935E0361E047E651E020E00E941C
:1081A0006352CC24DD2482E693E029D3882369F44A
:1081B0000894A108B108A114B10479F682E693E00D
:1081C00064E571E071D3882341F2EE24FF246E014F
:1081D0000894C11CD11C84E0A82EB12CAC0EBD1E8D
:1081E00037C082E693E0B80115D30F5F1F4F82E6D8
:1081F00093E061E571E055D3882399F3F80110828B
:108200008981882329F1C60165E471E00E941BF58C
:10821000009731F082E693E03DD321E030E021C0C9
:108220008701000F111FC701A5E0880F991FAA95AC
:10823000E1F7080F191FB8016654744FC50170DBD0
:10824000B8016253744FC50125DB0894E11CF11C91
:1082500082E693E0CBD2882311F48601C8CF20E0D8
:1082600030E0C901C150DF4FECE00C945DF21F9388
:10827000CF93DF93182F10925E030E94C24E80E0CE
:1082800060E04FE053E020E00E94635282E0809380
:1082900012010E946AD182E693E0FCD281E0C4DE42
:1082A00080E060E070E0CCDB009789F480E061E082
:1082B00049EF52E020E00E94635288E092E524EF0B
:1082C00031E0F9013197F1F70197D9F776C0133012
:1082D00059F1143028F41130C9F01230F0F408C00C
:1082E000153081F1153038F1163009F045C007C05E
:1082F0008CE060E070E0A4DBEC0180E029C08DE060
:1083000060E070E09DDBEC0186E022C08EE060E082
:1083100070E096DBEC0181E01BC08FE060E070E074
:108320008FDBEC0182E014C080E160E070E088DB6C
:10833000EC0183E00DC081E160E070E081DBEC01E5
:1083400084E006C082E160E070E07ADBEC0185E069
:108350000E94E1D00E946AD182E693E09BD280E045
:1083600060E070E06DDB80E060E070E069DB00976A
:1083700029F011E0209719F010E001C011E080E031
:1083800053DE112351F480E062E049EE52E020E038
:108390000E94635221E030E012C080E062E046EDCE
:1083A00052E020E00E94635288E092E524EF31E041
:1083B000F9013197F1F70197D9F720E030E0C901D1
:1083C000DF91CF911F9108951F93CF93DF930E9468
:1083D000C24E80E060E047E452E020E00E94635239
:1083E00038D982E00E94624D10925D0382E693E0EC
:1083F0006AE673E040E052E0EBD18091F61BBFDD0E
:108400008823E1F482E0BBDD8823C1F481E0B7DD9D
:108410008823A1F483E0B3DD882381F484E0AFDD19
:10842000882361F485E0ABDD882341F486E0A7DD95
:10843000882321F4A4DD882309F46EC082E08093B0
:10844000120183E060E070E0FBDAEC018AE060E0BA
:1084500070E0F6DA009729F011E0209719F010E0AB
:1084600001C011E08BE060E070E0EADA009709F407
:1084700011E088E160E070E0E3DA009709F411E0D0
:1084800089E160E070E0DCDA009709F411E085E052
:1084900060E070E0D5DA009739F0112329F480917B
:1084A000500EE5DE009709F411E08091500E0E9415
:1084B000E1D01123F1F480E0B7DD81E08093130176
:1084C00080E064E046E252E020E00E94635288E8E7
:1084D00093E124EF31E0F9013197F1F70197D9F7F2
:1084E0002BD532D5DCD881E00E94624D21E030E00E
:1084F0000EC081E00E94624D80E29EE424EF31E0F4
:10850000F9013197F1F70197D9F720E030E0C9017F
:10851000DF91CF911F91089580E064E045E352E040
:1085200020E00E94635281E0809390051092EC0D50
:108530000E94624D8091500E0E94E1D0E6CF1F93C1
:1085400082E693E06AE673E040E052E041D188EED3
:1085500093E024EF31E0F9013197F1F70197D9F772
:10856000A9D882E693E096D18091EF0D813059F43D
:1085700012E01093120158DD80E090DD882331F085
:108580001093120103C082E0809312011F9108959D
:10859000A0E6B0E0EEECF2E40C944BF29E01235F17
:1085A0003F4F80E090E0AE014F5F5F4F0BC01192F4
:1085B000E217F307E1F701969F01245F3F4F8830F0
:1085C000910561F0FC01EE0FFF1FE80FF91FEE0FA0
:1085D000FF1FEE0FFF1FE40FF51FE9CFCE0101963D
:1085E0009CDD009779F1EEECFBE080E0908199232F
:1085F00009F591819923F1F492819923D9F493811A
:108600009923C1F494819923A9F49581992391F434
:108610009681992379F49781992361F49085992320
:1086200049F49185992331F49285992319F493851E
:10863000992331F08F5FB2969CE0EE3DF907B1F6D9
:1086400080935F03C05ADF4FE2E00C9467F2A1E031
:10865000B0E0EDE2F3E40C9442F26E010894C11C28
:10866000D11C99249394F4E2AF2EFBE0BF2E54C0AA
:1086700080915C03813009F45FC01CD882E693E0EE
:10868000B5D0882329F00894E108F10801091109FF
:1086900082E693E0ABD0882309F046C082E693E0FF
:1086A000B601B8D080915C038823B1F5898184320A
:1086B00061F480911101813041F410921101B09266
:1086C0001001A0920F011092DA0D80911101882300
:1086D000A1F4E0910F01F0911001898180838091D4
:1086E000DA0D8F5F8093DA0D89818A3031F481E071
:1086F0008093110180935C0320C080910F019091C1
:10870000100101969093100180930F018091DA0D72
:10871000863911F490921101E0E8EE2EEAE1FE2E86
:10872000E6E00E2F112DA4CFE114F104010511058F
:1087300009F09ECF80E001C081E02196EBE00C942F
:108740005EF2A0E0B0E0E7EAF3E40C9445F2EC015D
:108750006B018A0120E030E019C0C901800F911F30
:108760008E159F0578F58A819B81800F911F820F5E
:10877000931F6C817D810E94D7F1AE81BF81A80FCC
:10878000B91F8C918E17F1F42F5F3F4FF601E20F66
:10879000F31FE491E880F980EE23F9F68A819B814A
:1087A000800F911F820F931F6C817D810E94D7F1F2
:1087B0009B838A83E01AF10AE21AF30AF982E882BB
:1087C00081E001C080E0CDB7DEB7E8E00C9461F253
:1087D000FC0155834483778366831382128211825E
:1087E00010820895FC01808191810895FC0181E04F
:1087F000208131812115310509F080E00895FC01C7
:1088000081E044815581208131814217530709F06D
:1088100080E00895FC01808191810097C9F0A681D4
:10882000B78182819381A80FB91F8C91DB018C9352
:10883000828193810196648175810E94D7F193832F
:1088400082838081918101979183808381E0089563
:1088500080E008951F93FC01162F2481358140810B
:1088600051812417350799F082819381840F951FD8
:10887000B9010E94D7F1A681B781A80FB91F1C9337
:108880008081918101969183808381E001C080E0A5
:108890001F910895FC01118210821382128281E0DF
:1088A000089540E050E04DCFEF92FF920F931F9359
:1088B000CF93DF938C017B01C0E0D0E007C0C801FB
:1088C000B701AE013EDF882349F42196F80180818B
:1088D0009181C817D90798F380E001C081E0CDB736
:1088E000DEB7E6E00C9463F2429A289A469A459ADB
:1088F000823051F0833018F48823F9F008958530E0
:10890000C1F0863071F517C08091C9008F7E8093C9
:10891000C9008091C900877F8093C9008091C900F8
:108920008F778093C900529853985A985B984298D1
:10893000089545980895469808958091C9008F7EBE
:108940008093C9008091C900877F8093C90080917E
:10895000C9008F778093C900529853985A985B98B2
:10896000289808950E94C24E8091EC0D813009F044
:108970007BC082E390E00E94EA5DAC0180E060E0B1
:1089800022E00E94635283E390E00E94EA5DAC0122
:1089900080E061E020E00E94635284E390E00E9466
:1089A000EA5DAC0180E063E020E00E94635285E371
:1089B00090E00E94EA5DAC0180E064E020E00E946B
:1089C00063528BE390E00E94EA5DAC0180E065E0D9
:1089D00020E00E94635280E066E04BEB54E020E030
:1089E0000E9463528AE066E04091500E20E00E94AF
:1089F00056598CE190E00E94EA5DAC018CE067E0A2
:108A000020E00E94635282E00E94624D80E29EE478
:108A100024EF31E0F9013197F1F70197D9F780910F
:108A2000EF0D882311F481E039DB82E05DDF0E94E5
:108A30009B5A80E20E94F3BA8823C9F380EF0E9418
:108A4000F3BA84E190E00E94C4D08091500E0E945D
:108A5000E1D08091E90D813011F486E001C085E01C
:108A600043DF81E00C94624D80E390E00E94EA5D78
:108A7000AC0180E061E020E00E94635281E390E07D
:108A80000E94EA5DAC0180E061E020E00E94635258
:108A90008BE290E00E94EA5DAC0180E062E020E0C1
:108AA0000E9463528CE290E00E94EA5DAC0180E09B
:108AB00063E020E00E9463528DE290E00E94EA5D54
:108AC000AC0180E064E020E00E9463528FE090E01F
:108AD0000E94EA5DAC018CE067E020E00E946352F6
:108AE00080E20E94F3BA8823D9F380EF0C94F3BAA2
:108AF0001F93CF93DF930E94C24E80E060E049EA6B
:108B000054E022E00E9463520E949B5A81E062E09E
:108B100045E954E020E00E94635287E063E04DE8BD
:108B200054E020E00E94635285E065E045E854E0AF
:108B300020E00E946352C0E0DEE01CE04991812FFA
:108B400065E020E00E94A3521F5F1031B9F78FE06B
:108B500090E00E94EA5DAC018CE067E020E00E94BA
:108B6000635282E0AFD780E29EE424EF31E0F90166
:108B70003197F1F70197D9F78091EF0D882311F420
:108B800081E08CDA80E0B0DE0E949B5A80E20E9495
:108B9000F3BA8823C9F384E190E00E94C4D08091A5
:108BA000500E0E94E1D08091E90D813011F486E0F1
:108BB00001C085E099DE81E085D780EF0E94F3BA9D
:108BC000DF91CF911F9108950E94C24E80E060E036
:108BD00043E754E022E00E9463520E949B5A81E0E6
:108BE00062E044E654E020E00E94635287E063E0E4
:108BF0004CE554E020E00E9463528FE090E00E9438
:108C0000EA5DAC018CE067E020E00E94635283E003
:108C100059D780E069DE0E949B5A80E20E94F3BA35
:108C20008823C9F384E190E00E94C4D08091500E63
:108C30000E94E1D08091E90D813011F486E001C0FD
:108C400085E052DE81E03ED780EF0C94F3BA0E94BB
:108C5000C24E80E060E046E454E022E00E946352AD
:108C600080E061E040E354E022E00E94635280E053
:108C700063E04AE154E020E00E94635280E064E057
:108C800044E054E020E00E94635280E065E04EEE54
:108C900053E020E00E94635280E066E048ED53E03C
:108CA00020E00E9463528CE190E00E94EA5DAC01FA
:108CB0008CE067E020E00E94635282E003D782E00C
:108CC00013DE80E20E94F3BA8823D9F380EF0E947A
:108CD000F3BA8091E90D813011F486E001C085E09E
:108CE00003DE81E0EFC60E94C24E80E060E044EC0B
:108CF00053E022E00E94635280E061E042EB53E0E7
:108D000022E00E94635280E063E044EA53E020E006
:108D10000E94635280E064E046E953E020E00E9454
:108D2000635280E065E047E853E020E00E94635230
:108D300080E066E04DE753E020E00E9463528CE162
:108D400090E00E94EA5DAC018CE067E020E00E94C8
:108D5000635283E0B7D680E20E94F3BA8823D9F346
:108D600080EF0E94F3BA81E0ADC60E94C24E82E35A
:108D700090E00E94EA5DAC0180E060E022E00E94A9
:108D8000635288E390E00E94EA5DAC0180E061E01C
:108D900020E00E94635289E390E00E94EA5DAC010A
:108DA00080E063E020E00E94635285E390E00E944F
:108DB000EA5DAC0180E064E020E00E9463528BE356
:108DC00090E00E94EA5DAC0180E065E020E00E9456
:108DD00063528CE190E00E94EA5DAC018CE067E0B8
:108DE00020E00E94635282E07FDD0E949B5A80E275
:108DF0000E94F3BA8823C9F380EF0E94F3BA84E19A
:108E000090E00E94C4D08091500E0E94E1D08091E9
:108E1000E90D813011F486E001C085E065CDB2D75F
:108E200080E060E04BE653E022E00E94635284E081
:108E300063E04DE553E020E00E94635287E064E088
:108E400045E553E020E00E9463528FE090E00E94ED
:108E5000EA5DAC018CE067E020E00E94635280E0B4
:108E600043DD0E949B5A80E20E94F3BA8823C9F333
:108E70008091E90D813011F486E001C085E034DD98
:108E800080EF0C94F3BA7ED78CE390E00E94EA5D09
:108E9000AC0180E060E022E00E9463528AE390E04F
:108EA0000E94EA5DAC0180E061E022E00E94635232
:108EB00089E390E00E94EA5DAC0180E063E020E09D
:108EC0000E94635280E064E04FE353E020E00E94A0
:108ED000635280E065E049E253E020E00E94635283
:108EE0008DE390E00E94EA5DAC0180E066E020E066
:108EF0000E9463528CE190E00E94EA5DAC018CE03C
:108F000067E020E00E94635280E0EEDC5E9880E241
:108F10000E94F3BA8823D9F380EF0E94F3BA5E9AD5
:108F20008091E90D813011F486E001C085E0DCCC50
:108F300081E08093ED0D089581E08093EE0D08951A
:108F400081E08093B00E089581E08093EF0D089545
:108F50001092EF0D08956093380E7093390E809340
:108F60003A0E90933B0E20933C0E30933D0E40936F
:108F70003E0E50933F0E089587E00E94ED4F80E033
:108F800067E04FE655E020E00E9463528BED9DE0E4
:108F900060E070E047E657E00E943EF687E00C9400
:108FA00011500F931F93CF93DF93ECD680E060E0D6
:108FB00049E555E022E00E94635280E061E04EE422
:108FC00055E020E00E94635280E062E048E355E013
:108FD00020E00E94635289E88093DC0D1092DD0D41
:108FE00085E08093DE0D21E02093DF0D82E4809305
:108FF000E00D2093E10D80E18093E20D80E4809309
:10900000E30D2093E40D1092E50D84E18093E60DCD
:1090100084E68093E70D1092E80D1092E90D10920E
:10902000EA0D1092EB0D1092EC0D1092ED0D1092D6
:10903000EE0D2093EF0D1092400E1092410E2093F2
:10904000450E1092460E2093470E1092480E88E26D
:109050008093490E20934A0E20934B0E80E197E2B5
:1090600090934D0E80934C0E10924E0E10924F0E18
:1090700084E08093500E2093440E84E391E2909319
:10908000430E8093420E84EF91E09093520E8093B2
:10909000510E8EE190E09093540E8093530E85E034
:1090A00090E09093560E8093550E1092570E209399
:1090B000580E1092590E1092380E1092390E1092CE
:1090C0003A0E10923B0E10923C0E10923D0E1092F2
:1090D0003E0E10923F0E80EF9DE063E375E00E942C
:1090E00005F585EF9DE06FE275E00E9405F585E0EE
:1090F0009EE060E275E00E9405F580E09EE06BE195
:1091000075E00E9405F5E4E1FEE011928EE0E832A0
:10911000F807D9F780E381939EE0E633F907D9F7A2
:109120001092360E1092370E86E88093DB0D109267
:10913000680E10925A0E8DE290E090935C0E809330
:109140005B0E90935E0E80935D0E2FE730E03093C0
:10915000600E20935F0E1092610E9093630E8093C9
:10916000620E9093650E8093640E3093670E209389
:10917000660E84E180936B0E10926C0E81E08093FA
:109180006D0E8AE080936E0E10926F0E1092700E2C
:1091900088E28093710E1092720EAF01435C5F4FB4
:1091A0002DE73EE007E81EE0CCE8DEE0A1E9BEE006
:1091B00080E090E0BC01625E7F4FFA0161937193A1
:1091C000AF01BC01625F7E4FF901619371939F0112
:1091D000F80111928F0119921D9201968530910527
:1091E00049F711E01093960E1093970E1093980E76
:1091F0008AE99EE067E175E00E9405F585EA9EE058
:109200006EE075E00E9405F51092B00E1092990E76
:109210008FEF9FEFDC018093B10E9093B20EA0937D
:10922000B30EB093B40E1092B50E1092B60E10930A
:10923000B70E1093B80E89EB9EE06EEF74E00E94BB
:1092400005F589EC9EE06EEE74E00E9405F589ED6F
:109250009EE06EED74E00E9405F50E9480E30E949E
:1092600000690E94AB800E94126986DE80E066E0A1
:1092700049EC54E020E00E94635282E167E046EC52
:1092800054E020E00E946352789488EC90E060E81B
:1092900070E040E00E9429BB80E10E94F3BA88237D
:1092A000D9F32998DF91CF911F910F9108958BEDFC
:1092B0009DE060E070E047E657E00E942EF60E94D5
:1092C000293B8091DB0D863809F483C087578031B4
:1092D00008F067CE0E9480E30E9400690E94AB8084
:1092E0000E9412698091DB0D813830F481E0809317
:1092F000970E8093980E02C0813821F481E080930C
:10930000E40D02C0823881F41092990E1092B00ED2
:109310008AE99EE067EF75E00E9405F585EA9EE028
:1093200062EF75E00E9405F58091DB0D843860F4F2
:109330008FEF9FEFDC018093B10E9093B20EA0935C
:10934000B30EB093B40E02C08438D9F41092B50EA7
:109350001092B60E81E08093B70E8093B80E89EB21
:109360009EE062EE75E00E9405F589EC9EE062EDFC
:1093700075E00E9405F589ED9EE062EC75E00E94C3
:1093800005F586E88093DB0D7894FCD480E062E0FC
:109390004EEA55E020E00E94635280E063E04AE933
:1093A00055E020E00E94635280E065E046E855E029
:1093B00020E00E94635282E167E043E855E020E04C
:1093C0000E94635280E10E94F3BA8823D9F3D4DD6E
:1093D000F8940895FC01608160933E16718170934A
:1093E0003F16828180934016938190934116089591
:1093F0002F923F924F925F926F927F928F929F92A5
:10940000AF92BF92CF92DF92EF920F931F93DF93B1
:10941000CF930F92CDB7DEB780E80E94F3BA8823CE
:1094200029F480916F05823009F040C080916F056A
:109430008130C9F1A7D480E060E04CE756E020E03D
:109440000E94635280E061E040E756E020E00E9425
:10945000635280E062E044E656E020E00E946352FE
:1094600080E063E048E556E020E00E94635280E03F
:1094700064E04CE456E020E00E94635280E065E046
:1094800040E456E020E00E94635280E066E044E35E
:1094900056E020E00E94635280E067E048E256E038
:1094A00020E00E94635281E080936F0580916C05FB
:1094B000813009F067C080916D05803309F062C08A
:1094C00080916F05882309F05DC0A09046158BE45C
:1094D00095E110E03C0153C0103109F453C018303D
:1094E00010F09BE001C090E0F3014081892F612FD3
:1094F00050E023E030E000E0EE2499830E945B57C7
:10950000F30143819981892F8C5F612F50E022E024
:1095100030E00E945B57F301218130E0A9014370E4
:10952000507099814330510531F4892F895F612F43
:1095300046E256E01DC020FF06C0892F895F612FDB
:1095400044E256E015C0F3012281253030F0892F26
:10955000895F612F42E256E00BC0892F895F22307C
:1095600020F0612F40E256E003C0612F4EE156E04B
:1095700020E0A9D71F5F8CE090E0680E791E1A15D5
:1095800008F4AACF80916F05813009F068C18091FD
:109590006C05813009F07DC080916D05863009F041
:1095A00078C080914C15823049F0823060F085306F
:1095B00050F48BE060E04BE156E009C08BE060E0E6
:1095C00048E156E004C08BE060E045E156E020E071
:1095D0007AD780914D158370833029F481E160E062
:1095E00043E156E004C081E160E041E156E020E063
:1095F0006AD780914D1580FF05C08EE060E04EE097
:1096000056E004C08EE060E04BE056E020E05BD71F
:10961000409171158BE061E050E022E030E000E025
:10962000EE240E945B578AE595E1D4DE9B01AC01F4
:109630008BE062E0A90125E030E00E945B5781E108
:1096400062E048E056E020E03ED790916F158FEF42
:10965000989FC001112420916E15820F911D64E620
:1096600070E00E94D7F1AB015C018BE063E022E087
:1096700030E00E945B578DE063E046E056E020E07A
:1096800022D78EE063E0A50122E030E001E00E94F5
:109690005B5780916C05813011F580916D058231A9
:1096A000F1F486E595E196DE20E13EE040E050E011
:1096B0000E94ACF120EA36E841E050E00E94FEF161
:1096C0008BE064E0A90123E030E000E0EE240E949A
:1096D0005B578FE064E041E056E020E0F4D68091F3
:1096E0006C05813009F0BBC080916D05823009F0B6
:1096F000B6C086E495E16EDE5B016C0190E8692EF0
:1097000096E9792E98E9892E912CC601B501A4011C
:1097100093010E94FEF18AE065E0A90122E030E0B9
:1097200000E0EE240E945B578CE065E04FEF55E0CF
:1097300020E0C9D6C601B50128EE33E040E050E094
:109740000E94FEF1CA01B90120E137E240E050E099
:109750000E94FEF19B01AC018DE065E0A90124E0CF
:1097600030E001E00E945B57C601B5012AE030E01D
:1097700040E050E00E94FEF184E6282E312C412C7E
:10978000512CCA01B901A20191010E94FEF19B0175
:10979000AC0181E165E0A90122E030E00E945B5765
:1097A0008AE495E117DE5B016C01A40193010E943C
:1097B000FEF18AE066E0A90122E030E000E00E94CC
:1097C0005B578CE066E04DEF55E020E07CD6C601AB
:1097D000B50128EE33E040E050E00E94FEF1CA01FE
:1097E000B90120E137E240E050E00E94FEF19B0128
:1097F000AC018DE066E0A90124E030E001E00E94C8
:109800005B57C601B5012AE030E040E050E00E941D
:10981000FEF1CA01B901A20191010E94FEF19B0172
:10982000AC0181E166E0A90122E030E00E945B57D3
:1098300082E595E1CFDD28EE33E040E050E00E9484
:10984000FEF18BE067E0A90124E030E000E00E9437
:109850005B5780E167E04BEF55E020E034D60F9096
:10986000CF91DF911F910F91EF90DF90CF90BF903C
:10987000AF909F908F907F906F905F904F903F90B0
:109880002F90089590916A05980F90936A058091A2
:109890006B05890F80936B050895A2E0B0E0E3E5C6
:1098A000FCE40C9445F26ED282E080936F058091C7
:1098B0008105823099F480E063E048E856E020E0DA
:1098C00002D684E690E09093211C8093201C809126
:1098D000201C9091211C0097D1F7A0C08091820597
:1098E000813011F00E9499D40E94FCD488EC90E061
:1098F0009093211C8093201C1982CC24DD2420E02D
:109900007E010894E11CF11C08EC10E0C7012A83D9
:109910000E94BDD22A81882309F46DC01093211CB6
:109920000093201CE22FF0E0E930F10508F063C05D
:10993000E05AFF4F0C9472F28981853B09F05BC0BD
:1099400010926E0510926D0510926C0510926A05CA
:1099500010926B0521E04FC08981823609F04AC020
:1099600047C08981813009F045C08CDF89818093AF
:109970006C0523E040C08981803331F0863021F0CE
:10998000823111F08230B1F580936D057BDF24E0E8
:1099900032C089818B3F70F575DFD98025E02BC0FF
:1099A0008981882339F56EDF26E025C0DA94898124
:1099B000E0916E05F0E0EE5BFA4E80832A8362DF71
:1099C00080916E058F5F80936E052A81DD2099F46A
:1099D00027E011C0C98028E00EC080916A05C81632
:1099E00049F4998180916B05981721F401DD02C03B
:1099F00022E001C020E080E22A830E94F3BA2A819B
:109A0000882339F48091201C9091211C009709F043
:109A10007DCF80EF0E94F3BA0E9499D42296E8E0AD
:109A20000C9461F211B814B817B81AB880B18093C9
:109A3000571683B18093591686B18093561689B113
:109A40008093431617B84798379B02C081E001C046
:109A500082E0809358164098309B03C010925516B0
:109A600003C081E080935516409A0895809158165E
:109A7000813009F4479880915816823009F45F9834
:109A8000089580915816813009F4479A80915816AC
:109A9000823009F45F9A089580915816813009F454
:109AA0005F9A80915816823009F4479A0895809100
:109AB0005816813009F45F9880915816823009F465
:109AC0004798089590915516992319F098B1947F6D
:109AD00098B9823051F0833001F1813009F58091DD
:109AE0005516439A10927005089580915516882353
:109AF00011F0409A01C0439880917005882381F449
:109B000081E08093700580E395E724EF31E0F9016F
:109B10003197F1F70197D9F70895419A109270059E
:109B2000089580917005882399F4809155168823B3
:109B300011F082E0C7CF439881E08093700580E305
:109B400095E724EF31E0F9013197F1F70197D9F763
:109B5000089580915516882311F081E0B3CF439A80
:109B6000109270050895EF920F931F935BDF809121
:109B70005516882331F087B1836087B988B1847F17
:109B800088B982B1806F82B90C988091960E81302D
:109B900009F409988FEF84B988B1806988B987B1D1
:109BA0008C6E87B93C988091551643985E9A8AB11D
:109BB000806F8AB9299A0E94D7B811E010931F1CB0
:109BC00084E190E00E94ECD284E190E00E94C4D055
:109BD00081E00E94E16680E096D169DB84E10E9429
:109BE000EBBC78948091500E8093F61B0E94E1D0DC
:109BF0008091500E0E941DD38091DE0D843088F03C
:109C00001093DE0D81E090E060E070E043E050E012
:109C100020E50CE0EE24E3940E9416A48093DE0D70
:109C2000ABD981E070D180E991E060E870E040E07C
:109C30000E9429BB10928A050E94AD598091581646
:109C40008130B1F482E060E040EE56E020E03BD4A9
:109C500087E061E048ED56E020E035D4809155166C
:109C6000882331F086E062E04DEC56E020E02BD412
:109C7000809158168230A9F460E04BEB56E020E06A
:109C800022D487E061E043EB56E020E01CD48091D1
:109C90005516882331F086E062E048EA56E020E07D
:109CA00012D480E063E04EE956E020E00CD48AE074
:109CB00063E045E956E020E006D486E090E00E94AB
:109CC000EA5DAC0180E065E020E0FDD387E090E054
:109CD0000E94EA5DAC0180E066E020E0F4D380E41D
:109CE0009FE124EF31E0F9013197F1F70197D9F7BE
:109CF0000799299888EE93E024EF31E0F901319734
:109D0000F1F70197D9F780E991E060E870E040E071
:109D10000E9429BB80EF0E94F3BA34D01ADF8091F1
:109D2000EB0D813041F48091ED0D882321F4809179
:109D3000500E0E94DEE526D08091EC0D813031F48A
:109D40008091EE0D882311F40E94E4410E944F3B64
:109D500019D08091EB0D813031F48091E90D882389
:109D600011F485E001C086E00E9474440BD01F917D
:109D70000F91EF9008952C988EBD0DB407FEFDCF86
:109D80002C9A08951F93CF93DF932BE536E1C901F9
:109D900060E070E040E054E00E9438F510EB2B9852
:109DA000812FE9DF80E1E7DF80917105E4DF2B9A05
:109DB000C0E8D0E080E0DFDF2197E1F71F5F183BCC
:109DC00071F71092351B1092361BDF91CF911F91C6
:109DD0000895A1E0B0E0EFEEFEE40C9449F28C01AE
:109DE0002B989C01220F232F221F330B3195822F9A
:109DF00080556983C0DF80917105102F1F77180F80
:109E0000812F82958F70805FB6DF812F8F70B3DFD7
:109E10002B9A6981862FAFDF2196E4E00C9465F2DE
:109E2000CF93DF93C0E0D0E0FE01E552F94E808190
:109E3000FE01E55AF94E80836081CE01CADF21968A
:109E400083E0C038D80781F7FE01E55AF94E108249
:109E5000CE0160E0BEDF219684E0C030D807A1F7D4
:109E6000DF91CF910895282F87FD35C0603498F594
:109E7000862F86958695869590E09695982F8827CB
:109E800097958795820F911D677021E030E001C0A2
:109E9000220F6A95EAF79370413061F0413018F073
:109EA0004230A1F40DC0FC01E55AF94E30812095F5
:109EB00032230BC0FC01E55AF94E3081322B05C02C
:109EC000FC01E55AF94E308132273083FC01E55A16
:109ED000F94E60817ECF089588E893E10197F1F70C
:109EE00008950F931F93CF93DF938C01C0E0D0E0D0
:109EF00002C0F2DF2196C017D107D8F3DF91CF91CE
:109F00001F910F9108951F93182F1092351B1092D7
:109F1000361B8CE58CBD81E08DBD2C9A2A988AE099
:109F200090E0DFDF2A9A2C982B9880E424DF113010
:109F300089F480917105882321F481EA1CDF80EC8B
:109F400003C080EA18DF88EC16DF8091E50D8823D6
:109F500039F404C081EA0FDF80EC0DDF86EA01C02E
:109F600087EA09DF82EA07DF8FE205DF88EF03DF98
:109F700080E001DF87E2FFDE113029F481E8FBDEBB
:109F80008091E60D03C081E8F6DE86E1F4DE8CEA1E
:109F9000F2DE80E0F0DE8FEAEEDE8091570E88235D
:109FA000C9F41130A1F46091E70D70E0882777FDC6
:109FB0008095982F0E94D7EF23E333E343E250E4E8
:109FC0000E94C4F00E94A9EF6093B30003C08FEF1A
:109FD0008093B300D7DE1F9108950F931F93CF9303
:109FE000DF93082F10E01695102F0027179507957F
:109FF0001370C0E0D0E0CE01800F911FFC01E55A44
:10A00000F94E2081DE01A45AB54E2C936081E1DE29
:10A010002196CE37D10579F7DF91CF911F910F911E
:10A0200008950F931F93CF93DF93082F10E0169599
:10A03000102F0027179507951370C0E0D0E0CE01D0
:10A04000800F911FFE01E45AF54E2081FC01E55A74
:10A05000F94E20836081BDDE2196CE37D10579F798
:10A06000DF91CF911F910F9108958091361B8F5FE3
:10A070008093361B883020F0D3DE87E08093361B38
:10A080000895A5E0B0E0E7E4F0E50C943BF2602E23
:10A09000082F10E0C62EDD24242E3324D101A01B6E
:10A0A000B10B422F50E05A8349837A01EC18FD0826
:10A0B000B7FD08C0E1E08E2E912C109731F4882472
:10A0C000992403C088248A94982CF7FC09C071E075
:10A0D000472E512CE114F10431F44424552403C0DB
:10A0E00044244A94542C9D01B7FF03C03095219518
:10A0F0003F4FF7FE04C0F094E194F108F394462D2D
:10A100002C833D83B0DE2C813D81E216F3063CF5C5
:10A11000C90162E070E00E94EBF1AA24BB24A61AF8
:10A12000B70A982D782C700E16C0AE0CBF1C080D07
:10A13000191D1A141B0424F4C40CD51CA21AB30A4A
:10A14000872D6C2D462D2C833D839B838CDE9B813C
:10A15000790E3D812C810215130539F726C0C70100
:10A1600062E070E00E94EBF1AA24BB24A61AB70AB1
:10A17000342C742C7C0C14C0A20EB31EC40CD51C41
:10A180001A141B0424F4080D191DAE18BF08802FE3
:10A19000672D462D2C833D8366DE730C3D812C811B
:10A1A00089819A81C816D90639F72596E2E10C947F
:10A1B00057F2A0E0B0E0EFEDF0E50C9444F2182F78
:10A1C000B02E87FD1FE7603408F06FE3E42EFF2414
:10A1D000C62EDD24C20ED11CE10EF11C21E8E216D0
:10A1E000F10418F0A0E8EA2EF12C31E4C316D104F2
:10A1F00018F0F0E4CF2ED12CC62FD0E007C0812F6D
:10A200006C2F4E2D2C2F0B2D3CDF2196CC16DD060E
:10A21000B0F7CDB7DEB7E9E00C9460F2A1E0B0E0B2
:10A22000E4E1F1E50C9441F2C82EB62E322FD02E87
:10A230004F3DE1F0403E38F4463D81F04C3D91F019
:10A24000443CA9F407C0463F59F04C3F69F0443EF6
:10A2500071F402C041E00BC042E009C043E007C016
:10A2600044E005C045E003C046E001C04EE1142FC4
:10A270001F77FC2CFF0CFC0CFF0CFD0C6B2D660FEC
:10A28000660F660FAE2CA60EEE2009F051C03230DC
:10A2900011F0343039F48F2D45E027E001E03983A7
:10A2A00088DF3981AB2CBB24B694BA2CAA24B7948E
:10A2B000A79446E02C2D249FC0011124A80EB91E9E
:10A2C0008D2D992787FD9095A80EB91E8FEF93E0ED
:10A2D000A822B922149FA00111248A010E50194FFF
:10A2E00088EFE82E86E0F82EE40EF51EF801949132
:10A2F000323011F0343039F4F501E55AF94E8081ED
:10A300008927808304C0F501E55AF94E9083F50151
:10A31000E55AF94E6081C50139835BDD0F5F1F4F40
:10A320000894A11CB11C39810E151F05F9F63AC01D
:10A3300006E0109F80011124B2EF8B2EB6E09B2E19
:10A34000800E911E0850194FF401B490EA2CCC24D1
:10A35000C394DD248C2D8B2139F0323059F041E04B
:10A3600050E0343061F406C0323039F041E050E062
:10A37000343029F040E050E002C041E050E08F2D41
:10A380006E2D398370DD3981D394E394FD2DF8303F
:10A3900011F0CC0CDFCF0894811C911CF394801633
:10A3A000910691F62196ECE00C945DF2AF92BF928B
:10A3B000DF92EF92FF920F931F93CF93DF93D62EEE
:10A3C000F42E122FA82EE5015E01B92EE50119C069
:10A3D0004A30B1F04D3019F41092351B12C0809103
:10A3E000351B6091361B2D2D0F2DE12E17DF80912F
:10A3F000351B8F5F8093351B863118F01092351B0B
:10A4000034DE4991442321F7DF91CF911F910F91C1
:10A41000FF90EF90DF90BF90AF900895EF920F9371
:10A42000FA01402F8093351B6093361BCF01622FBA
:10A430002E2DBCDF0F91EF9008958093351B609314
:10A44000361BCA01622F40E020E0B0CFA0E0B0E0B0
:10A45000ECE2F2E50C9446F2EC01D62EF42E122F2B
:10A460001AC04A30B1F04D3019F41092351B12C0A9
:10A470008091351B6091361B2D2D0F2DE12ECEDEE8
:10A480008091351B8F5F8093351B863118F01092B9
:10A49000351BEBDD2196FE014491442311F7CDB726
:10A4A000DEB7E7E00C9462F2EF920F93FA01402FCF
:10A4B0008093351B6093361BCF01622F2E2DC6DF94
:10A4C0000F91EF9008958093351B6093361BCA015E
:10A4D000622F40E020E0BACF40E020E0B7CF8F927B
:10A4E0009F92BF92CF92DF92EF92FF920F931F93B2
:10A4F000CF93DF93182FF62EB22EC02EDE2C842E93
:10A50000E4014E01952EE40107C0812F6F2D2B2D04
:10A510000C2DED2C83DE1F5F49914423B1F7DF91B1
:10A52000CF911F910F91FF90EF90DF90CF90BF9050
:10A530009F908F900895EF920F9300E0EE24CFDF6D
:10A540000F91EF900895EF920F9300E0EE2466DEF6
:10A550000F91EF9008951F93CF93DF93EC01162F87
:10A5600017C04A3019F04D3019F40FC07EDD0FC00E
:10A570008091351B6091361B212FE5DF8091351BC3
:10A580008F5F8093351B863110F01092351B21961A
:10A59000FE014491442329F7DF91CF911F91089543
:10A5A0008093351B6093361BCA01622FD4CF0F9363
:10A5B0001F938093351B6093361B282F30E0240FA8
:10A5C000311D263131051CF005E1081B01C0042FA7
:10A5D000080F182F07C0812F6091361B40E220E042
:10A5E000B2DF1F5F1017B8F31F910F910895A0E01D
:10A5F000B0E0EDEFF2E50C9446F2F82EE02E87FF86
:10A6000002C03FE7F32E162F603408F01FE3E42F5B
:10A61000F0E0C12FD0E0C20FD11DEF0DF11DE138E8
:10A62000F10510F0E0E8F0E0DE2E8F2D612F4E2FC7
:10A63000212F0E2D26DDC134D10510F0C0E4D0E06D
:10A640008D2D612F4D2D2C2F0E2D1BDD8D2D9E015F
:10A650006C2F4F2D16DD8F2D6C2F4F2D212F11DDDF
:10A66000CDB7DEB7E7E00C9462F2A0E0B0E0EBE338
:10A67000F3E50C943BF2C82ED62E7A01922EC1E05F
:10A68000D0E0C41BD50B00271127041B150B000FAE
:10A69000111F6E2D6D0D422FE6DB6D2D6E198C2D69
:10A6A000492DE1DB8E2D8C0D6D2D492DDCDB8C2DA4
:10A6B0008E196D2D492DD7DB43E0242E312CAA2491
:10A6C000BB2443C0D7FD07C00894E108F1080E5F22
:10A6D0001F4FC00FD11F0894A11CB11CC20DD31D68
:10A6E0005A2C5C0C6E2C6D0C852D662D492DBBDB18
:10A6F0004C2C4A18842D662D492DB5DB6D2C6E1817
:10A70000852D662D492DAFDB842D662D492DABDBC4
:10A710005E2C5C0C6A2C6D0C852D662D492DA3DBFF
:10A720008C2D8E19782E662D492D9DDB9D2D9A1925
:10A73000892E852D692F492D96DB872D682D492D72
:10A7400092DB82E090E0280E391EAE14BF040CF4B8
:10A75000B9CFCDB7DEB7E2E10C9457F2A0E0B0E09C
:10A76000E4EBF3E50C943BF2B82E162F6A01A22E0F
:10A77000C1E0D0E0C41BD50BEE24FF24E41AF50A97
:10A78000EE0CFF1C642F610F212F241B4B2D0A2D73
:10A7900078DC4B2D4C198C2D8B0D612F212F71DC0A
:10A7A000460163E0262E312C6624772437C0D7FD7E
:10A7B00009C008948108910882E090E0E80EF91E33
:10A7C000CE0DDF1D0894611C711CC20DD31DC62C5B
:10A7D000562C5B0C4B2C4618282D210F852D622FF3
:10A7E000442D0A2D4EDC212F2819852D622F442D52
:10A7F00048DC582C5B0C9B2D9819D92E262D210F47
:10A80000852D622F492F3DDC212F2619852D622FA2
:10A810004D2D37DC82E090E0280E391E6814790453
:10A8200034F2CDB7DEB7E2E10C9457F2A1E0B0E02C
:10A83000ECE1F4E50C943CF2882EF62E342ED22E68
:10A840009E2CB80180E090E00E94D5EF2BED3FE018
:10A8500049E450E40E94C4F020E030E044E353E4D3
:10A860000E943CEF162FA72E082FE92E0E9439EFE9
:10A870002B013C016D2D70E080E090E00E94D5EF4F
:10A880009B01AC01C301B2010E94C4F00E9427F1F8
:10A890002B013C01612F7A2D802F9E2D0E9447F1C4
:10A8A0005B016C01632D70E080E090E00E94D5EFC9
:10A8B0009B01AC01C601B5010E94C4F00E9427F1C2
:10A8C0000E94A9EF462F480DC301B20149830E949F
:10A8D000A9EF2F2D261B882D6F2D4981092DD1DB46
:10A8E0002196E1E10C9458F2AEE0B0E0EAE7F4E53D
:10A8F0000C943BF2182FF62E6A015901449F9001E7
:10A90000459F300D549F300D11243A832983AA9C12
:10A91000C001AB9C900DBA9C900D11249C838B833D
:10A92000A29E4001A39E900CB29E900C1124BC01EB
:10A9300068197909882777FD8095982F0E94D7EFAD
:10A940002B013C01E981FA81BF01882777FD8095C1
:10A95000982F0E94D7EF20E030E040E85EE30E94AD
:10A96000C4F09B01AC01C301B2010E94D1EE0E9470
:10A9700027F10E94A4EF3B019401220F331F3A8775
:10A9800029876A2D6F0D812F402F6DDA6F2D6A197F
:10A99000812F402F68DA8C2D810F6F2D402F63DAC5
:10A9A000812F8C196F2D402F5EDA89819A819095C5
:10A9B00081959F4F880F991F9E838D83EB81FC812A
:10A9C000EE0FFF1FF887EF836F012B813C81C20ED2
:10A9D000D31E44245524882499247E866D86298597
:10A9E0003A853DC08D859E8597FD0BC00894A108D2
:10A9F000B108ED81FE812E0F3F1F821B930B9E87B6
:10AA00008D870894411C511C8F819885880E991E52
:10AA1000ED85FE85EC0DFD1DFE87ED87E42CE10E36
:10AA20007A2C7F0C8E2D672D402F2B873C871BDACD
:10AA3000FF2DFA196F2E8E2D6F2F402F14DAE12E75
:10AA4000E4188E2D672D402F0EDA8E2D662D402FA7
:10AA50000ADA8F819885C80ED91E3C852B8582160F
:10AA600093060CF4BFCF3A872987B201882777FD78
:10AA70008095982F0E94D7EF20E030E040E05FE320
:10AA80000E94D1EEE62EC72E782E692E150108946D
:10AA900021083108EB81FC81BF01882777FD809573
:10AAA000982F0E94D7EFF3012E2D3C2D4F2F5E2FB4
:10AAB0000E94C4F0F3012E2D3C2D4F2F5E2F0E94DB
:10AAC000C4F05B016C01229CC001239C900D329C60
:10AAD000900D112429813A81829FB001839F700DCE
:10AAE000929F700D1124882777FD8095982F0E94E2
:10AAF000D7EF9B01AC01C601B5010E94D1EE5B010D
:10AB00006C018B819C81E981FA818E9FB0018F9FBE
:10AB1000700D9E9F700D1124882777FD8095982FCA
:10AB20000E94D7EF9B01AC01C601B5010E94D0EE97
:10AB30000E9427F10E94A4EF51012D813E813095A2
:10AB400021953F4FC980DA808D819E81C81AD90A2C
:10AB5000E985FA85CE1ADF0A7A836983190136C03E
:10AB600029813A81121613065CF00894411C511C8D
:10AB70008F819885880E991E280D391D3A83298367
:10AB8000E981FA81EC0DFD1DFA83E983E42CE10EE5
:10AB90007A2C7F0C8E2D672D402F4B8664D9FF2D8C
:10ABA000FA196F2E8E2D6F2F402F5DD99B85E12EC8
:10ABB000E91A8E2D672D402F56D98E2D662D402FE8
:10ABC00052D90894A108B108C20CD31CC501019642
:10ABD000181619062CF22E96E2E10C9457F20F93F8
:10ABE000FA01022F4D5F5F4F9F017EDE0F910895A6
:10ABF000EF920F931F93942FF901E02E4D5F292FB1
:10AC00008F0114DE1F910F91EF9008958A3010F498
:10AC1000805D0895895C0895A1E0B0E0E2E1F6E589
:10AC20000C9448F2F82E042F122F6093361B8F5F7E
:10AC30008093351B842F82958F706983E7DF482FBF
:10AC40008F2D6981212F7FDC802F8F70DFDF482FD0
:10AC50008091351B6091361B212F75DC2196E5E034
:10AC60000C9464F2FF920F931F93082F162FF0900D
:10AC7000351B8F2D8F5F8093351B802F82958F70B2
:10AC8000C5DF482F8F2D6091361B212F5CDCF090A3
:10AC9000351B8F2D8F5F8093351B802F8F70B6DF14
:10ACA000482F8F2D6091361B212F4DDC8091351B55
:10ACB000982F9F5F9093351B6091361B40E2212FA8
:10ACC00042DC1F910F91FF900895A0E0B0E0EBE609
:10ACD000F6E50C9447F2FE0170964CEDE42E4AE145
:10ACE000F42E80E0B70140E52E853F858F010E945C
:10ACF000BFDF89858093351B8A858093361BC7010A
:10AD00006B854C852D8552DB2096E6E00C9463F232
:10AD1000A0E0B0E0EEE8F6E50C9447F2FE01709694
:10AD20005CEDE52E5AE1F52E81E0B70140E52E8578
:10AD30003F858F010E94BFDF89858093351B8A85FF
:10AD40008093361BC7016B854C852D852FDB2096A4
:10AD5000E6E00C9463F2EF92FF920F931F93CF9370
:10AD6000DF93082FC3E0D0E020E014E6EAE0EE2E07
:10AD7000802F612F0E94CBF1F82E882321F422230B
:10AD800011F4113069F48091351B982F9F5F9093D7
:10AD9000351B4F2D405D6091361B20E0D4DB21E058
:10ADA000812F6E2D0E94CBF1219731F0F19E102D55
:10ADB0001124011B182FDCCFCDB7DEB7E6E00C94D1
:10ADC00063F28093351B6093361B842FC4CFA0E0C1
:10ADD000B0E0EDEEF6E50C9446F2D82ECB017A0108
:10ADE00035E23093371B222331F020E32093381BC8
:10ADF000C9E3DBE102C0C8E3DBE16EE27BE14AE0EC
:10AE000050E00E949EF50EE21BE1F80101C089931B
:10AE100081918823E1F71E141F0484F48EE2899344
:10AE2000C7016EE27BE14AE050E00E949EF501C05E
:10AE30008993F80181918F018823D1F7D8821982F3
:10AE4000CDB7DEB7E7E00C9462F2AF92CF92EF920B
:10AE5000FF920F931F93CF93DF93182FF62EEA01E3
:10AE6000B901202F85E740E050E0B1DF8DB79EB7F4
:10AE700009979EBF8DBFEDB7FEB73196ADB7BEB790
:10AE800011961C93F182E282C382A48287E39BE144
:10AE900096838583D087C78318DF8DB79EB70996C1
:10AEA0009EBF8DBFDF91CF911F910F91FF90EF90CB
:10AEB000CF90AF900895AF92CF92EF920F93CC24A2
:10AEC000AA24C3DF0F91EF90CF90AF900895AF9277
:10AED000CF92EF92FF920F931F93CF93DF93182F90
:10AEE000F62EEA01B901202F84E640E050E06FDF42
:10AEF0008DB79EB709979EBF8DBFEDB7FEB7319650
:10AF0000ADB7BEB711961C93F182E282C382A482D0
:10AF100087E39BE196838583D087C783D6DE8DB791
:10AF20009EB709969EBF8DBFDF91CF911F910F9164
:10AF3000FF90EF90CF90AF900895AF92CF92EF92A5
:10AF40000F93CC24AA24C3DF0F91EF90CF90AF9042
:10AF50000895AF92CF92EF92FF920F931F93CF93EA
:10AF6000DF93182FF62EEA01B901202F61507040AF
:10AF700085E741E050E02BDF8DB79EB709979EBF74
:10AF80008DBFEDB7FEB73196ADB7BEB711961C9326
:10AF9000F182E282C382A48287E39BE19683858368
:10AFA000D087C78392DE8DB79EB709969EBF8DBFAF
:10AFB000DF91CF911F910F91FF90EF90CF90AF90C5
:10AFC0000895AF92CF92EF920F93CC24AA24C1DFC1
:10AFD0000F91EF90CF90AF900895CF92EF92FF92A4
:10AFE0000F931F93CF93DF93182FF62EEA01B90129
:10AFF000202F6150704085E742E050E0E8DE80910C
:10B0000080052DB73EB7295030403EBF2DBFEDB76C
:10B01000FEB73196ADB7BEB711961C93F18282830D
:10B02000E382C48287E39BE196838583D087C783CD
:10B030004CDE2DB73EB7275F3F4F3EBF2DBFDF91A0
:10B04000CF911F910F91FF90EF90CF900895CF92E5
:10B05000EF920F93EE24CC24C0DF0F91EF90CF90AE
:10B060000895AF92CF92EF92FF920F931F93CF93D9
:10B07000DF93182FF62EEA01B901202F615070409E
:10B0800084E641E050E0A3DE8DB79EB709979EBFEE
:10B090008DBFEDB7FEB73196ADB7BEB711961C9315
:10B0A000F182E282C382A48287E39BE19683858357
:10B0B000D087C7830ADE8DB79EB709969EBF8DBF26
:10B0C000DF91CF911F910F91FF90EF90CF90AF90B4
:10B0D0000895AF92CF92EF920F93CC24AA24C1DFB0
:10B0E0000F91EF90CF90AF900895CF92DF92EF92B3
:10B0F0000F931F93CF93DF93182F362F6A01CCE362
:10B10000D0E0CA01BE010E94D7F18DB79EB70B9760
:10B110009EBF8DBFADB7BEB71196EDB7FEB7118319
:10B1200011963C93119712962C93129713960C93A9
:10B1300013971496EC92149784E191E016969C93E1
:10B140008E93159718967C936E9317976C9FC001FA
:10B150006D9F900D7C9F900D1124F601E81BF90B5B
:10B160001A96FC93EE931997B0DD8DB79EB70B96A8
:10B170009EBF8DBFDF91CF911F910F91EF90DF9018
:10B18000CF900895EF920F9320E000E0EE24ADDF22
:10B190000F91EF900895A0E1B0E0E1EDF8E50C9497
:10B1A0003FF2D82EB62EE986FA860B871C872D87AC
:10B1B0003E874F87588BF82CCE010196BE01675F02
:10B1C0007F4F0E949FE269807A808B809C808DB740
:10B1D0009EB70D979EBF8DBF0DB71EB70F5F1F4F58
:10B1E000EDB7FEB7D182F801B182C282A382F482A8
:10B1F0008EE191E096838583C401B30120E13EE0B6
:10B2000040E050E00E94FEF1F80127831086FCE345
:10B21000CF2ED12CE12CF12CC401B301A701960152
:10B220000E94FEF1662ECA01B901A70196010E9493
:10B23000FEF1F801618712866386148646DD8DB7BC
:10B240009EB70D969EBF8DBF6096EEE00C945BF2AC
:10B25000CF92EF920F93CF93DF93EDB7FEB73B976B
:10B26000FEBFEDBFCDB7DEB72196818369830A8328
:10B27000EB82CC828CE391E09E838D83CA01B9017D
:10B2800024E630E040E050E00E9420F22F8338872F
:10B2900049875A871ADD8DB79EB70B969EBF8DBF23
:10B2A000DF91CF910F91EF90CF9008954330D1F07F
:10B2B000443028F4413081F0423088F407C04530F2
:10B2C000B9F0453090F04630B1F403C046E45AE09E
:10B2D0000EC041E45AE00BC04CE35AE008C046E31C
:10B2E0005AE005C040E35AE002C04AE25AE0EBC827
:10B2F00043E25AE0E8C808950F930E94C24E88E0E6
:10B3000068E04FE620E301E072D982E062E042E1CA
:10B310005AE022E0D8D882E064E041E05AE020E040
:10B32000D2D882E065E042EF59E020E0CCD880E15D
:10B330000E94F3BA882379F480E20E94F3BA88234A
:10B3400051F480E40E94F3BA882329F480E80E9433
:10B35000F3BA882361F30F91089509981198ECE7E7
:10B36000F0E080E480838081807E816080838FEE46
:10B3700080937A000895EF92FF920F931F93CF93DB
:10B38000DF93F8946091420E7091430E80E090E05C
:10B390000E94D5EF2091720530917305409174059C
:10B3A000509175050E94D1EE2FE832EC45E75FE33E
:10B3B0000E94C4F07B018C01762F272F3F2D402F58
:10B3C000512FCA01B9010E94A4EFCB0160E470E0E3
:10B3D0000E94EBF1EC0190937B0580937A056E2D32
:10B3E0007F2D802F912F20E030E040E85CE30E9429
:10B3F000C4F0262F372F482F592F209372053093F2
:10B4000073054093740550937505C032D10574F0EF
:10B4100020E030E040E85FE30E94D1EE60937205E7
:10B420007093730580937405909375056091720510
:10B4300070917305809174059091750520E030E05E
:10B4400040EF50E40E943CEF262F372F482F592F12
:10B4500020937605309377054093780550937905CE
:10B460000E94A9EF70937F0560937E0510927D0581
:10B4700010927C0580E090E0DC018093720590934F
:10B480007305A0937405B09375057894CDB7DEB7B6
:10B49000E6E00C9463F21F920F920FB60F920BB678
:10B4A0000F9211242F933F934F935F936F937F934A
:10B4B0008F939F93AF93BF93EF93FF936091780027
:10B4C0007091790080E090E00E94D5EF9B01AC0183
:10B4D0006091720570917305809174059091750566
:10B4E0000E94D1EE6093720570937305809374058A
:10B4F0009093750580917C0590917D0501969093C0
:10B500007D0580937C0520E1803092070CF033DFCD
:10B51000FF91EF91BF91AF919F918F917F916F912B
:10B520005F914F913F912F910F900BBE0F900FBEE7
:10B530000F901F9018950F93CF93DF9387E662E0EB
:10B5400041E023E001E053D880917E0590917F0592
:10B5500021E08034920738F489E662E043E123E099
:10B5600000E00E94D9508091440E813051F588E668
:10B5700060E047E127E001E03AD880917E059091B4
:10B580007F0531E0843A930718F4C0E0D0E002C0B0
:10B59000C3E1D0E09C01215431402336310538F419
:10B5A0008054914065E070E00E94D7F1EB018C2F50
:10B5B00043E14C1B855962E023E000E00E94D95032
:10B5C00002C0C0E0D0E08091440E882331F588E6C7
:10B5D00060E046E127E001E00AD880917E05909185
:10B5E0007F0531E08A39930710F0C2E1D0E09C0179
:10B5F000215431402935310538F48054914065E0BB
:10B6000070E00E94D7F1EB018C2F42E14C1B855971
:10B6100062E023E000E00E94D950209739F08AE6EA
:10B6200062E04C2F23E001E00E94D950DF91CF91DE
:10B630000F910895CF92EF920F930E94B34D109205
:10B640008105109282058091380E9091390EA0915B
:10B650003A0EB0913B0E181619061A061B060CF08E
:10B660008AC080913C0E90913D0EA0913E0EB0910B
:10B670003F0E181619061A061B060CF07CC00E9415
:10B68000C24E89E090E0A6D2AC0180E060E022E00A
:10B690000E9463528CE090E09DD2AC0180E061E0BA
:10B6A00022E00E9463528AE090E094D2AC0180E0F4
:10B6B00062E022E00E9463528BE090E08BD2AC010A
:10B6C00080E067E020E00E94635220913C0E3091C0
:10B6D0003D0E40913E0E50913F0E81E064E000E04F
:10B6E000EE24CC24B5DD2091380E3091390E4091F6
:10B6F0003A0E50913B0E8CE064E0AADD80E80E9497
:10B70000F3BA882361F160E070E0CB0120E030E023
:10B71000A9010E94AB4780E060E240E820E100E040
:10B720000E94D9508DE090E055D2AC0180E065E0F8
:10B7300020E00E94635280E066E045E10E94D7521B
:10B7400080E067E045E10E94D75280E197E224EF74
:10B7500031E0F9013197F1F70197D9F70CC080E199
:10B760000E94F3BA882351F280E060E240E820E2D0
:10B7700000E00E94D950D8D2FCD1FECFEF92FF92C8
:10B780000F931F930E94DBD585E79BE00E940FD6A5
:10B7900081E00E9440D68091EC0D882371F0809169
:10B7A000EB0D882351F088E261E048E755E42BE295
:10B7B0003BE0890179010E94B5D780915516882315
:10B7C00051F08CE261E044EE55E42DE33BE0890169
:10B7D00079010E94B5D78091EB0D882351F089E261
:10B7E00061E04FE057E42FE43BE0890179010E94DA
:10B7F000B5D78AE261E045EB56E42DE53BE08901EF
:10B8000079010E94B5D78091EC0D882351F08BE22D
:10B8100061E042EB54E429E63BE0890179010E94B2
:10B82000B5D780E00E9435DB0E9402D61F910F91B0
:10B83000FF90EF900895EF92FF920F931F930E9455
:10B84000DBD587E99BE00E940FD681E00E9440D6BD
:10B850008CE361E044E55CE521E83BE089017901A6
:10B860000E94B5D78091EC0D882351F08DE361E003
:10B8700041E350ED2EE83BE0890179010E94B5D704
:10B880008EE361E049E653EB29EE3AE08901790164
:10B890000E94B5D780E00E9435DB0E9402D61F913E
:10B8A0000F91FF90EF90089580918105882319F4FE
:10B8B00081E00E948D6580918105813019F482E0DC
:10B8C0000E948D6580918105823011F40C948D6504
:10B8D0000895EF92FF920F931F9381E061E048ED8E
:10B8E00050E82BE13BE0890179010E94B5D782E065
:10B8F00062E043E85BE82FE93AE009EA1AE0780100
:10B900000E94B5D783E061E04EEE53E622EF3AE0C5
:10B91000890179010E94B5D780918305882351F46C
:10B9200084E062E049EE59E92DEF3AE089017901BE
:10B930000E94B5D785E061E042E352E62AE03BE0B1
:10B9400003E11BE078010E94B5D786E061E04DE499
:10B950005CE42FE13BE0890179010E94B5D78BE0DF
:10B9600062E04BE15CE522EB3AE00EEB1AE0780195
:10B970000E94B5D788E062E04EEB5BE52AEC3AE046
:10B98000890179010E94B5D789E062E040E050E08A
:10B9900026ED3AE0890179010E94B5D78AE061E09D
:10B9A00049E95CE920EE3AE0890179010E94B5D7C6
:10B9B0001F910F91FF90EF900895EF92FF920F93D8
:10B9C0001F938EE361E049E653EB29EE3AE08901EB
:10B9D00079010E94B5D783E061E04EEE53E622EF95
:10B9E0003AE0890179010E94B5D7809183058823C7
:10B9F00051F484E062E049EE59E92DEF3AE0890123
:10BA000079010E94B5D785E061E042E352E62AE081
:10BA10003BE003E11BE078010E94B5D78BE062E0D8
:10BA20004BE15CE522EB3AE00EEB1AE078010E9474
:10BA3000B5D788E062E04EEB5BE52AEC3AE089019D
:10BA400079010E94B5D789E062E040E050E026ED40
:10BA50003AE0890179010E94B5D78AE061E049E9BD
:10BA60005CE920EE3AE0890179010E94B5D71F9187
:10BA70000F91FF90EF900895EF92FF920F931F9315
:10BA80005EE8E52E5AE0F52E87E061E040E050E008
:10BA90002CE73AE087010E94B5D749EAE42E4AE054
:10BAA000F42E82E062E043E85BE82FE93AE08701A8
:10BAB0000E94B5D73EEBE32E3AE0F32E8BE062E036
:10BAC0004BE15CE522EB3AE087010E94B5D72AEC16
:10BAD000E22E2AE0F22E88E062E04EEB5BE5970171
:10BAE00087010E94B5D796EDE92E9AE0F92E89E0FC
:10BAF00062E040E050E0970187010E94B5D780EEF8
:10BB0000E82E8AE0F82E8AE061E049E95CE99701D5
:10BB100087010E94B5D71F910F91FF90EF90089574
:10BB20000E94DBD58CE491E00E9428D681E00E943F
:10BB300040D68BE190E04ED0BC0185E04BE55CE95E
:10BB40000E9456D688E660E070E04EEB5BE50E940E
:10BB500056D680918105882309F48EDF8091810576
:10BB6000813009F4B6DE80918105823009F425CF59
:10BB700008951F931091EC0D0E946AD1EEDB80EFC7
:10BB80000E94F3BA81E591E063E471E04CE050E09B
:10BB90000E9468F581E00E940CD6C2DF80E00E941E
:10BBA00035DB0E94D0D6873039F4BED0882341F0EF
:10BBB0000E9402D6B5DF04C0893011F40E9442B160
:10BBC0008091EC0D181751F30E9402D6A9DF109155
:10BBD000EC0DE4CF2091DE0D222361F4FC01EE0F89
:10BBE000FF1FE80FF91FEE0FFF1FED55F44F2591D2
:10BBF00034911BC0213061F4FC01EE0FFF1FE80FF0
:10BC0000F91FEE0FFF1FEB55F44F259134910DC036
:10BC1000223069F4FC01EE0FFF1FE80FF91FEE0F51
:10BC2000FF1FE955F44F25913491C9010895E3EAC6
:10BC3000FBE025913491C9010895A1E0B0E0E3E271
:10BC4000FEE50C943FF289838B01742E0E94C2D4CE
:10BC500081E5809380051092180A3FE0932E21E73A
:10BC6000622E882483945E010894A11CB11C91E08B
:10BC7000C92ED12C84E1E82EF12C24C08DB79EB7BB
:10BC800007979EBF8DBFEDB7FEB73196ADB7BEB774
:10BC900011966C9281828282B482A382D682C582FE
:10BCA0000E944AD3F092211CE092201C8DB79EB7CF
:10BCB00007969EBF8DBF8091201C9091211C0097FC
:10BCC000D1F79A948091180A882311F49920B1F63B
:10BCD0001982992069F00E943ED4E0911A0AF091ED
:10BCE0001B0A81918983D8011196FC93EE9317C0AA
:10BCF0007720A9F082E790E06DDFAC0180E062E0A0
:10BD000020E00E94635284E690E09093211C80938F
:10BD1000201C8091201C9091211C0097D1F78981D3
:10BD20002196EEE00C945BF2A2E0B0E0EAE9FEE5D9
:10BD30000C943BF21A8219828BE10E9443D38BE16F
:10BD40000E9443D385E50E9443D38AEA0E9443D3ED
:10BD500080E00E9443D386E5809380051092180A04
:10BD6000FF2401E016E783C00E94519C882319F448
:10BD7000002309F441C00E94C24E80E060E045E625
:10BD800027E001E00E94D95080E060E043E452E304
:10BD900022E00E94635286E060E04AE352E322E040
:10BDA0000E94635288E090E015DFAC0183E061E01F
:10BDB00020E00BEFE2E0EE2E0E9454528EE090E085
:10BDC00009DFAC0180E063E020E000E074E0E72EF2
:10BDD0000E9454528FE090E0FDDEAC018CE067E001
:10BDE00020E00E94635280E067E24EE728E001E035
:10BDF0000E94F75232E0F32E9EDB00D00F92EDB797
:10BE0000FEB73196ADB7BEB711961C931182128260
:10BE10000E944AD38EE090E09093211C8093201CD6
:10BE20000F900F900F908091201C9091211C0097F3
:10BE3000D1F782E069E24F2D24E001E00E94D95061
:10BE4000B2E0FB0E2F2D2D3740F082E069E24BE788
:10BE500024E000E00E94D950FF2480E20E94F3BA5F
:10BE6000882321F01092810580E081C100E080915B
:10BE7000180A882309F478CF8091180A882351F092
:10BE80000E943ED480911A0A90911B0A90934C1BF9
:10BE900080934B1B8091931C823611F482E005C085
:10BEA0008091931C833629F481E0809381058093EF
:10BEB000820581E0809383058FEFBE016F5F7F4F26
:10BEC00040E0BBDE882339F0E981FA811081113628
:10BED00009F437C101C010E084EF91E024EF31E0B4
:10BEE000F9013197F1F70197D9F781E08093830544
:10BEF00082EC91E060E470E040E00E9429BB01E048
:10BF00007724739422E6A22E21E0B22E92E0F92E3D
:10BF100089E6882E81E0982EBAE4CB2EB2E3DB2EA0
:10BF2000A1E64A2E512CF8E72F2EF1E03F2EE6E055
:10BF30006E2E002309F4E5C00E94C24E80E060E04E
:10BF40004FE727E001E00E94D950112389F488E1EE
:10BF500090E040DEADB7BEB71997BEBFADBFEDB73D
:10BF6000FEB7319611966C921182F282BEEF10C02C
:10BF700089E190E02FDEADB7BEB71997BEBFADBF68
:10BF8000EDB7FEB7319611966C921182F282BBEF3B
:10BF9000B3831482B682A582908787830E946556F8
:10BFA0002DB73EB7275F3F4F3EBF2DBF84E190E0E6
:10BFB00011DEADB7BEB71D97BEBFADBFEDB7FEB7C3
:10BFC000319611961C92718212821382F4829682AB
:10BFD000858290878783D286C186548643860E9455
:10BFE00065562DB73EB7235F3F4F3EBF2DBF112390
:10BFF00011F185E190E0EEDDADB7BEB71D97BEBF94
:10C00000ADBFEDB7FEB7319611961C92F182128248
:10C010001382F4829682858290878783D286C18636
:10C02000138714860E9465562DB73EB7235F3F4F96
:10C030003EBF2DBF2AC085E190E0CCDDADB7BEB7D5
:10C040001B97BEBFADBFEDB7FEB7319611961C92E0
:10C05000F18212821382F48222E731E03683258353
:10C0600090878783D286C1860E9465568DB79EB71A
:10C070000B969EBF8DBF80E162E044E352E322E075
:10C0800000E072E0E72E0E94545280E06DE14FE73D
:10C0900027E101E00E94F75286E190E09BDDAC01D0
:10C0A00081E064E020E000E0EE240E94545287E149
:10C0B00090E090DDADB7BEB71B97BEBFADBFEDB78B
:10C0C000FEB7319611967C92B5E0B183128213824D
:10C0D000F482368225829087878328E232E3328792
:10C0E00021870E9465568DB79EB70B969EBF8DBF68
:10C0F00080E190E06FDDAC0183E167E020E00E9429
:10C100006352A0E9B1E0B093211CA093201CEE245F
:10C1100000E008C00E94519C882311F001E002C099
:10C12000EE24E39480E10E94F3BA882331F48091F5
:10C13000201C9091211C009769F7EE2009F4F9CE9C
:10C1400002C010928305109280051092180A82E3B3
:10C1500090E09093211C8093201C8091201C909152
:10C16000211C0097D1F780EF0E94F3BA81E022965C
:10C17000E2E10C9457F2A1E0B0E0E1ECF0E60C94BF
:10C180003EF2E0918205F0E0ED57FA4F808189831D
:10C190000E94C24E80E062E04AE852E320E00E9442
:10C1A000635281E064E04BE752E320E00E94635277
:10C1B00084E090E00FDDAC018CE067E020E00E94BD
:10C1C000635283E167E048E752E320E00E94635254
:10C1D00081E48093800580ED97E024EF31E0F90160
:10C1E0003197F1F70197D9F71092180A84E190E09E
:10C1F0009093211C8093201C11E000E0B1E6FB2EFF
:10C20000552453945E010894A11CB11CA1E08A2E10
:10C21000912CF4E1CF2ED12CE4EF6E2EE1E07E2EB6
:10C22000C1C08DB79EB707979EBF8DBFEDB7FEB754
:10C230003196ADB7BEB71196FC9211825282B4828C
:10C24000A382968285820E944AD38DB79EB70796B5
:10C250009EBF8DBF11E006C080E20E94F3BA11E0DC
:10C26000811110E08091180A882341F48091201CEC
:10C270009091211C009711F0112371F78091201CDF
:10C280009091211C009709F467C00E943ED4498117
:10C29000E0911A0AF0911B0A8081481709F04EC0FC
:10C2A0008FE064E050E022E030E000E0EE240E9405
:10C2B0005B572091820530E02150304075E0220F1D
:10C2C000331F7A95E1F78981280F311DC90164E098
:10C2D000880F991F6A95E1F7820F931FA0914F1B5A
:10C2E000B091501BE0911A0AF0911B0AA80FB91FD8
:10C2F000319680E101900D928150E1F780918205A5
:10C3000090E00197298155E0880F991F5A95E1F730
:10C31000820F911D9C0144E0220F331F4A95E1F7E3
:10C32000280F391FE0914F1BF091501BE20FF31FB4
:10C33000108A89818F5F898300E007C088EE93E0CF
:10C34000F3013197F1F70197D9F7D092211CC092F0
:10C35000201C1092180A26C01123D9F00F5FD0922A
:10C36000211CC092201C0233E0F080E062E049E62C
:10C3700052E320E00E94635284E690E09093211CF7
:10C380008093201C8091201C9091211C0097D1F754
:10C3900012C080E20E94F3BA11E0882319F010E085
:10C3A00001C011E08981803220F4112309F039CFD6
:10C3B0000AC0112341F0E0918205F0E0ED57FA4FF9
:10C3C0008981808311E0812F2196EFE00C945AF24D
:10C3D000FF920F931F93CF93DF93F82E0E94C24ECC
:10C3E00007E02F2D209F80011124C0E0D0E06C2FAA
:10C3F0009F2D943041F4C43030F080E06C2F45E143
:10C400000E94D75220C02091820530E02150304058
:10C4100055E0220F331F5A95E1F7200F311F2C0FE3
:10C420003D1FC90144E0880F991F4A95E1F7820F2B
:10C43000931F40914F1B5091501B480F591F80E094
:10C4400020E00E941D522196C730D10581F6CDB75C
:10C45000DEB7E5E00C9464F280914F1B9091501B85
:10C460000C9412F3A3E0B0E0E8E3F2E60C943BF2A4
:10C470000E94C24E80E494E00E9478F29093501B98
:10C4800080934F1B009719F40E947C59A3C1E82F99
:10C49000F92F80E494E0DF019C011D92215030408F
:10C4A000E1F710928405109285050E94C2D488ECB1
:10C4B00090E09093211C8093201CE0918205F0E095
:10C4C000ED57FA4F8081803220F455DE882309F43D
:10C4D00080C18091201C9091211C009709F479C1A2
:10C4E00084E4809380051092180A08EC10E0109301
:10C4F000211C0093201C8AE089838DB79EB7079783
:10C500009EBF8DBFEDB7FEB7319684E6ADB7BEB71F
:10C5100011968C93118281E082835E010894A11CA4
:10C52000B11CB482A38281E090E0968385830E944F
:10C530004AD31093231C0093221CEDB7FEB7379605
:10C54000FEBFEDBF80E044DF10E0B8ECCB2ED12C75
:10C55000AAE09A2EF4E66F2E552453948A2C7B2C55
:10C56000E1E0AE2EB12C74E4472E8091180A8823A6
:10C5700009F467C00E943ED420911A0A30911B0A28
:10C580003B832A8383E090E025DBAC0180E067E019
:10C5900020E00E946352412F4F5F85E067E00E94D8
:10C5A000E15680918205823011F483E001C083E17D
:10C5B00067E046E652E320E00E94635280918205E4
:10C5C000823011F483E101C083E067E043E652E387
:10C5D00020E00E94635287E0189F10011124FF247D
:10C5E00016C0220D331D2F5F3F4F220F331F8A814C
:10C5F0009B81280F391FD9014D915C918FE06F2DE0
:10C6000026E030E000E0EE240E949D57F3942F2DA9
:10C6100030E0143019F484E090E002C087E090E04C
:10C6200028173907F4F21092180A8CEA9DE0E4EF1B
:10C63000F1E03197F1F70197D1F7D092211CC09228
:10C64000201C8091221C9091231C0097E1F4998278
:10C65000EDB7FEB73797FEBFEDBF3196ADB7BEB7AA
:10C6600011966C921182528283827482B682A58264
:10C670000E944AD3D092231CC092221CEDB7FEB771
:10C680003796FEBFEDBF80E80E94F3BA882329F0F9
:10C690001150153058F014E009C080E40E94F3BA3C
:10C6A000882331F01F5F153008F010E0812F90DEF5
:10C6B00080918105813009F040C080E10E94F3BA89
:10C6C0008823D9F180918205813019F40E94C2D467
:10C6D00002C00E9499D4E0918205F0E0ED57FA4F34
:10C6E0008081803220F447DD882309F472C04092B3
:10C6F00080051092180AD092211CC092201C9982A9
:10C700002DB73EB7275030403EBF2DBFEDB7FEB727
:10C710003196ADB7BEB711966C9211825282838268
:10C720007482B682A5820E944AD3EDB7FEB73796CF
:10C73000FEBFEDBF80E04CDE10E080E20E94F3BA65
:10C74000882339F48091201C9091211C009709F0D6
:10C750000CCF19822DB73EB7275030403EBF2DBFBA
:10C76000EDB7FEB7319684E6ADB7BEB711968C93A0
:10C77000118281E08283CE0101969483838381E0DC
:10C7800090E0968385830E944AD310928005109290
:10C79000180A8091201C9091211CEDB7FEB73796A6
:10C7A000FEBFEDBF0097A9F40E94C24E80E062E098
:10C7B00044E552E320E00E94635284E690E09093C7
:10C7C000211C8093201C8091201C9091211C00979B
:10C7D000D1F742DE2396E2E10C9457F2A1E0B0E0FB
:10C7E000E4EFF3E60C943BF288E48093800510922A
:10C7F000180A84EF91E09093211C8093201C8CEF09
:10C80000898311E0FF2478E6572E6E010894C11C3D
:10C81000D11C61E0A62EB12C44244A9454EF852EFD
:10C8200051E0952E44EF642E41E0742E3EEF332EFE
:10C830002DEF222E112309F454C00E94C24E80E035
:10C8400060E04FE728E001E00E94D95086E660E012
:10C8500048E128E000E00E94D95080E06BE04FE71B
:10C8600029E201E00E94F75280E060E049EB52E3E8
:10C8700022E00E94635283E090E0ACD9AC0180E0FA
:10C8800067E020E00E94635280918205813059F474
:10C8900060E046EB52E322E00E94635283E167E0EE
:10C8A00043EB52E31BC080918105823061F481E04B
:10C8B00060E040EB52E322E00E94635283E167E0D4
:10C8C0004DEA52E30BC081E060E04AEA52E322E025
:10C8D0000E94635283E167E047EA52E320E00E944E
:10C8E00063520E949B5A8DB79EB707979EBF8DBF1C
:10C8F000EDB7FEB73196ADB7BEB711965C92118217
:10C9000081E08283D482C382B682A5820E944AD308
:10C9100049828DB79EB707969EBF8DBF80E991E093
:10C92000F4013197F1F70197D9F78091180A88231C
:10C9300009F454C00E943ED480918105882361F49B
:10C940008091931C815680938105813009F082E0AB
:10C950008093820511E001C010E0F090A91C1092B4
:10C96000A91C80E062E045E95CE120E005E0EE24FE
:10C97000EA940E940E52F092A91CF090BD1C1092F5
:10C98000BD1C80E063E049EA5CE120E0EE240E9407
:10C990000E52F092BD1CF090D11C1092D11C80E080
:10C9A00064E04DEB5CE120E0EE24E3940E940E5243
:10C9B000F092D11C1092E51C80E065E041ED5CE155
:10C9C00020E092E0E92E0E940E521092180A709216
:10C9D000211C6092201CFF24F39401C010E00E94EF
:10C9E000519C811111E080E80E94F3BA882331F450
:10C9F00080E862E00E941DBB882311F0398222C0CA
:10CA000080E40E94F3BA882331F480E462E00E945B
:10CA10001DBB882311F0298215C0809181058130CA
:10CA200089F480E10E94F3BA882361F08091820545
:10CA3000813019F40E94C2D402C00E9499D49CEFA4
:10CA4000998311E080E20E94F3BA882339F480913F
:10CA5000201C9091211C009709F0ECCE80EF0E94E1
:10CA6000F3BA109280051092180A8091201C9091C0
:10CA7000211C0097B9F4FF2011F00E94C24E80E003
:10CA800062E043E952E320E00E94635284E690E0D2
:10CA90009093211C8093201C8091201C9091211C3C
:10CAA0000097D1F70E9499D42196E2E10C9457F2B5
:10CAB000A8E7BDE190E1FD0111929A95E9F788237D
:10CAC00039F4CD0170E040E150E00E9438F505C036
:10CAD000E82FF0E0E958F24E60838DB79EB70797D4
:10CAE0009EBF8DBFEDB7FEB7319684E7ADB7BEB739
:10CAF00011968C9381E08183828388E79DE1948302
:10CB0000838380E190E0968385830E944AD3EDB7CA
:10CB1000FEB73796FEBFEDBF0895EF920F931F93B8
:10CB2000CF93DF93182F0E94C24E81E08093521B57
:10CB30008093541B1092531B0E94C24E8EEE92E3C0
:10CB400062E00E946C5282E062E043EE52E320E039
:10CB50000E94635282E063E048ED52E320E00E94CD
:10CB6000635288E068E240E026E001E00E94D9508C
:10CB700083E090E02FD8AC0180E067E020E00E94E5
:10CB8000635282E167E044ED52E320E00E94635289
:10CB900080E062E042ED52E320E00E9463521230F6
:10CBA00051F480918105813031F48091820581308A
:10CBB00011F40E94C2D4CFEFD0E08091521B8823A1
:10CBC00069F580E40E94F3BA882331F480E463E0DD
:10CBD0000E941DBB882311F14091531B4E3FF0F47E
:10CBE0004F5F4093531B89E063E050E023E030E067
:10CBF00000E0EE240E945B57123081F48091531BB9
:10CC000020E7829FC0011124BE010E94EBF1462F54
:10CC100088E068E226E001E00E94D9508091521B32
:10CC2000882309F040C080E80E94F3BA882331F4D9
:10CC300080E863E00E941DBB8823A9F18091531B0B
:10CC4000882389F1123079F420E7829FC0011124F2
:10CC5000BE010E94EBF1862F885F68E240E026E08B
:10CC600000E00E94D9504091531B41504093531B08
:10CC700089E063E050E023E030E000E0EE240E9431
:10CC80005B57123081F48091531B20E7829FC001D3
:10CC90001124BE010E94EBF1462F88E068E226E0F5
:10CCA00001E00E94D9508091521B8130D9F480E478
:10CCB0000E94F3BA882331F480E461E00E941DBB36
:10CCC000882381F04091541B403160F44F5F4093C2
:10CCD000541B89E062E050E023E030E000E0EE2405
:10CCE0000E945B578091521B813041F580E80E9481
:10CCF000F3BA882331F480E861E00E941DBB8823E9
:10CD0000E9F04091541B4423C9F041504093541B17
:10CD1000442349F089E062E050E023E030E000E0A5
:10CD2000EE240E945B578091541B882339F489E0DC
:10CD300062E04EEC52E320E00E94635280E10E94E8
:10CD4000F3BA882329F18091521B882389F462E089
:10CD50004CEC52E320E00E94635280E063E04AEC36
:10CD600052E320E00E94635281E08093521B10C086
:10CD700080E062E048EC52E320E00E94635280E0F1
:10CD800063E046EC52E320E00E9463521092521B93
:10CD90008091541B6091531B8BDE80E20E94F3BA9A
:10CDA000882309F40ACF80EF0E94F3BA123019F4F5
:10CDB00080E060E07DDEDF91CF911F910F91EF90D9
:10CDC0000895089510927D1B10927E1B08951F9365
:10CDD000CF93DF93EA0110917E1B1F30B0F58823BB
:10CDE000E1F021E030E002C0220F331F8A95E2F724
:10CDF000C901AA2797FDA095BA2F2091B10E3091B5
:10CE0000B20E4091B30E5091B40E82239323A4230B
:10CE1000B5230097A105B105C1F0E12FF0E0DF01D6
:10CE2000AA0FBB1FAA0FBB1FA358B44E13967C9327
:10CE30006E931297EE0FFF1FEE0FFF1FEF57F44E8A
:10CE4000D183C0831F5F10937E1BDF91CF911F9111
:10CE5000089510927D1B90917E1B891710F480938A
:10CE60007D1B089580917D1B8F5F80937D1B90912A
:10CE70007E1B891710F010927D1B81E08093BC1BF4
:10CE8000089580917D1B882311F480917E1B815031
:10CE900080937D1B81E08093BC1B0895E0917D1BF6
:10CEA000F0E0EE0FFF1FEE0FFF1FEF57F44E019063
:10CEB000F081E02D09950895FC0110821182128203
:10CEC000138220E021C0822F90E0DC01AA0FBB1F5B
:10CED000A80FB91FAA0FBB1FAA53BD4E3C91418199
:10CEE000431710F431832083DC01AA0FBB1FA80F66
:10CEF000B91FAA0FBB1FA753BD4E8C9193819817E2
:10CF000010F4838322832F5F8091C3122817D8F2F5
:10CF10000895EF920F93DF93CF9300D000D0CDB759
:10CF2000DEB7CE010196C8DF87E890E00E94EA5D97
:10CF3000AC0180E060E020E00E9463526091A312A7
:10CF40007091A412882777FD8095982F0E94D7EFC3
:10CF500020E030E040EA51E40E943CEF0E94A4EF60
:10CF60009B01AC018EE060E0A90124E030E000E02C
:10CF7000EE240E949D5782E160E04DE620E002E051
:10CF80000E940E5188E890E00E94EA5DAC0180E0CA
:10CF900061E020E00E9463522091A9123091AA1210
:10CFA00040E050E0CA01B901E3E0660F771F881F37
:10CFB000991FEA95D1F7620F731F841F951F2AEFFF
:10CFC00030E040E050E00E94FEF18FE061E0A90116
:10CFD00023E030E000E00E945B5782E161E045E041
:10CFE00054E320E002E00E94545289E890E00E945D
:10CFF000EA5DAC0180E062E020E00E946352809133
:10D00000AF129091B0126AE070E00E94D7F1AB01CC
:10D010008EE062E024E030E000E00E945B5782E1B5
:10D0200062E04DE620E002E00E940E518AE890E0C6
:10D030000E94EA5DAC0180E063E020E00E94635260
:10D040004091C1124F3F41F48EE063E040E054E371
:10D0500020E00E94635209C08EE063E050E023E0CC
:10D0600030E000E0EE240E94E15782E163E046E513
:10D0700020E002E0EE240E940E518DE890E00E9434
:10D08000EA5DAC0180E064E020E00E9463524091E0
:10D09000BB125091BC128EE064E024E030E000E06E
:10D0A0000E945B5782E164E04CEF53E320E002E032
:10D0B0000E9454528CE890E00E94EA5DAC0180E04E
:10D0C00065E020E00E9463524091B3125091B41287
:10D0D0008DE065E024E030E000E00E94E15782E16D
:10D0E00065E041E420E002E00E940E5180E066E04D
:10D0F0004EEE53E320E00E946352498150E04F5FBF
:10D100005F4F86E066E021E030E000E00E945B5780
:10D110004A818EE066E050E023E030E00E94E15773
:10D1200082E166E041E420E002E00E940E5180E0EE
:10D1300067E040EE53E320E00E9463524B8150E0F1
:10D140004F5F5F4F86E067E021E030E000E00E9443
:10D150005B574C818EE067E050E024E030E00E94B5
:10D160005B5782E167E04DED53E320E002E00E946F
:10D1700054522496DEBFCDBFCF91DF910F91EF9037
:10D180000895A1E0B0E0E7ECF8E60C9448F2F82E40
:10D19000FF0CFF0CFF0C9FE39F19692F685080E084
:10D1A0004FE723E000E099830E94D9509981192F1D
:10D1B00014502F2D2C5F80E0612F4FE701E00E947B
:10D1C000D95080E0612F40E00E94334F8FE7612FFC
:10D1D00040E00E94334F9981935081E0612F40E0FD
:10D1E000292F00E099830E9441508EE7612F4FE77D
:10D1F0009981292F0E9441502196E5E00C9464F218
:10D2000089E6EBE8F2E1DF011D928A95E9F78FEFFD
:10D210008093C1128093B8128EE78093BE128093E0
:10D22000C012089584E591E0EEEEF3E1DF019C0188
:10D230001D9221503040E1F70895A2E0B0E0E3E212
:10D24000F9E60C944BF2813089F58A830E9499D4D7
:10D2500019822DB73EB7275030403EBF2DBFEDB7E6
:10D26000FEB7319694E6ADB7BEB711969C93118286
:10D270008A818283CE0101969483838381E090E04A
:10D28000968385830E944AD383E090E09093211C8B
:10D290008093201C2DB73EB7295F3F4F3EBF2DBF67
:10D2A0008091201C9091211C0097D1F78AE08983FE
:10D2B0008DB79EB707979EBF8DBFEDB7FEB731966E
:10D2C0008FE6ADB7BEB711968C9382E0818381E083
:10D2D0008283CE0101969483838381E090E09683DC
:10D2E00085830E944AD383E090E09093211C809331
:10D2F000201C2DB73EB7295F3F4F3EBF2DBF809109
:10D30000201C9091211C0097D1F787E089838DB76D
:10D310009EB707979EBF8DBFEDB7FEB731968BE6E0
:10D32000ADB7BEB711968C93118281E08283CE0196
:10D3300001969483838381E090E0968385830E94A5
:10D340004AD38FE48093800588EC90E09093231C6F
:10D350008093221C1092180A2DB73EB7295F3F4FC9
:10D360003EBF2DBF2296E2E00C9467F2A2E0B0E04F
:10D37000ECEBF9E60C9445F294E59093800591E08E
:10D3800099832DB73EB7275030403EBF2DBFEDB734
:10D39000FEB7319624E7ADB7BEB711962C9322E0C5
:10D3A000218392839E012F5F3F4F3483238321E0AB
:10D3B00030E0368325838A830E944AD31092180A6C
:10D3C0008A8190E09093211C8093201CEDB7FEB7DA
:10D3D0003796FEBFEDBF8091201C9091211C0097D5
:10D3E000D1F78091180A882309F44BC00E943ED4DB
:10D3F00000911A0A10911B0AD8018D919C911197E6
:10D40000815D9740873C910508F03DC0F894F80194
:10D41000648170E080E090E020E13EE040E050E098
:10D420000E94ACF16B017C01D80115966C911597A7
:10D4300070E080E090E02CE330E040E050E00E94BB
:10D44000ACF1C60ED71EE81EF91EF8018681C80E83
:10D45000D11CE11CF11CC092241CD092251CE0922E
:10D46000261CF092271C83818093281C8281809344
:10D47000291C8081918190932B1C80932A1C789485
:10D4800002C080E001C081E090E02296E8E00C94C8
:10D4900061F2A0E0B0E0EFE4FAE60C943DF2E09136
:10D4A000D81BF091D91BED5BFF4FA08080912E1C03
:10D4B00090912F1C009769F484E158DF009719F4CC
:10D4C00082E390E002C080E797E190932F1C809365
:10D4D0002E1C8091371C9091381C009709F0ABC02E
:10D4E0008BE4809380051092180A84E190E0909379
:10D4F000211C8093201CBB2481E0A822BB2490C067
:10D500008091180A882309F48BC00E943ED4A09110
:10D510001A0AB0911B0ADC909D2D983008F07EC04D
:10D5200085E0989FF0011124EB5AF44E0D90019282
:10D530008150E1F70D2D10E0F801EE0FFF1FEE0F07
:10D54000FF1FE00FF11FEB5AF44E8481807F09F436
:10D5500065C0A114B10409F461C0E801CC0FDD1F5E
:10D56000C00FD11FCC0FDD1FC552D24FDE01A75116
:10D57000BB4FED90FC9011970894E11CF11CED92CB
:10D58000FC929CEE492E94E0592E4C0E5D1ED20169
:10D590006D907C90119788249924C1806C2D70E047
:10D5A00080E090E024E630E040E050E00E94ACF102
:10D5B0006619770988099909970140E050E00E94AF
:10D5C00020F2260D371D481D591DF201318320839D
:10D5D000C551DB4F88818C1508F4C882F801EE0F25
:10D5E000FF1FEE0FFF1FE00FF11FEB5AF44E828179
:10D5F000F801EE0FFF1FE00FF11FEE0FFF1FE753C3
:10D60000FD4E9081981708F480838091C31290E0BA
:10D61000081719071CF0D394D092C3121092180A5D
:10D620008091201C9091211C009709F069CF1092E5
:10D63000381C1092371C8FE4809380051092180AD2
:10D640008CE291E09093211C8093201CCDB7DEB733
:10D65000E0E10C9459F2E091D81BF091D91BDF0165
:10D66000AD5BBF4F8C9180FF6AC0DF01A65BBF4FEF
:10D670008C9181FF64C085A996A997FF29C010925B
:10D680008B0580918D058F5F80938D0590918C0522
:10D69000992399F490919201891778F08091570E0F
:10D6A000882339F48CE291E06FEF7FEF40E00E9435
:10D6B00029BB8091920180938D0580918C058F5FAD
:10D6C00080938C0590919101891711F410928C052B
:10D6D000E091D81BF091D91B85A996A9009719F460
:10D6E00010928D050895181619064CF510928C05A8
:10D6F00080918D058F5F80938D0590918B05992387
:10D7000099F490919201891778F08091570E8823AF
:10D7100039F484E690E06FEF7FEF40E00E9429BB90
:10D720008091920180938D0580918B058F5F80930E
:10D730008B0590919001891711F410928B05089533
:10D740005091DC0D523330F560919305633020F534
:10D7500082E080939105E091D81BF091D91B42E0C3
:10D760007BE20BC0A42FAF5F21AD30E0479FC0012B
:10D770001124281739071CF04A2F473098F340939B
:10D780009105459F402D1124409392056F5F609352
:10D79000930502C050939205E091D81BF091D91BDC
:10D7A00091AD809192059817A0F4809194058530F1
:10D7B00020F48F5F809394050895ED5BFF4F808187
:10D7C00080FF07C088EE93E060E270E041E00C94D7
:10D7D00029BB0895CF93DF93C091D81BD091D91B5B
:10D7E0008EAD9FADE8E6F1E0BF010E94EBF19C0138
:10D7F0008EA59FA5BF010E94EBF1281B390B37FFB7
:10D8000002C028593E4F3093DB1B2093DA1BDF9177
:10D81000CF9108959C01285130402C32310528F1D8
:10D820009C01245430402D32310508F19C012157D0
:10D8300030402D323105E8F09C012E5930402D3218
:10D840003105C8F09C012B5C30402D323105A8F029
:10D850009C01285F30402D32310588F0855291407F
:10D860008D32910570F486E0089580E0089581E09E
:10D87000089582E0089583E0089584E0089585E0A6
:10D88000089587E00895A0E0B0E0E9E4FCE60C9498
:10D8900043F2382FF62ECA01D22E102F66E170E027
:10D8A0000E94D7F16D5E70E0EB01249755E0A52E44
:10D8B000B12CA60EB71E01C03C2DC32EC394FE0191
:10D8C000EA5AFC4C4491832F6F2D20E00D2DE12E60
:10D8D0000E940E512196CA15DB0571F7CDB7DEB750
:10D8E000EAE00C945FF2A0E0B0E0E9E7FCE60C941B
:10D8F00044F2F82EE62ED42EC22EE801822F869511
:10D90000B62EB81A8F2D6B2D01E00E94F7521F2DF5
:10D910001F5F6B2D6F5F4D2D42502C2D2250812F9C
:10D9200000E00E94D9504D2D4F0D8F2D6E2D2E2DC4
:10D9300001E00E9441501C161D060CF04FC0CE01A4
:10D9400065E070E00E94EBF1FB016130710569F068
:10D9500062307105B9F02E2D21508F2D8C5F4F2D27
:10D960004A5F309721F5622F52C02E2D21504F2D46
:10D970004A5F8F2D8C5F622F01E00E9441506E2D17
:10D98000635054C02E2D21504F2D4A5F8F2D8C5F38
:10D99000622F01E00E9441506E2D63508F2D8D5FEC
:10D9A00044E021E00E94D9506E2D655057C0622F8F
:10D9B00001E00E9441506E2D63508F2D8D5F44E039
:10D9C00021E00E94D9506E2D65508F2D8E5F46E06C
:10D9D00021E00E94D9506E2D66505AC0209709F45C
:10D9E0005CC0CE016BEF7FEF0E94EBF1FB01613079
:10D9F000710581F062307105E9F08F2D8C5F4F2D3C
:10DA00004A5F2E2D2F5F309769F5622F01E00E944B
:10DA1000415043C02E2D2F5F4F2D4A5F8F2D8C5FBD
:10DA2000622F01E00E9441506E2D6E5F8F2D8D5F41
:10DA300044E030C02E2D2F5F4F2D4A5F8F2D8C5F1D
:10DA4000622F01E00E9441506E2D6E5F8F2D8D5F21
:10DA500044E021E00E94D9506E2D6C5F8F2D8E5FC7
:10DA600046E018C0622F01E00E9441506E2D6E5FAB
:10DA70008F2D8D5F44E021E00E94D9506E2D6C5FA8
:10DA80008F2D8E5F46E021E00E94D9506E2D6B5F96
:10DA9000812F48E021E00E94D950CDB7DEB7E9E000
:10DAA0000C9460F28F929F92AF92BF92CF92DF92CE
:10DAB000EF92FF920F931F93F62E182F110F180F4E
:10DAC000110FFF0CFF0CFF0CB7E0AB2EAF0CA3E067
:10DAD0009A2E9F0C812F692D41E00E94334FF6E072
:10DAE000BF2EBF0CD12ED394E2E08E2E8F0C8D2D45
:10DAF0006B2D4D2D282D01E00E944150EF2CE39419
:10DB0000812F8E5F6E2D41E00E94334F73E0C72E50
:10DB1000C10E8C2D6F2D41E00E94334F812F8C5F01
:10DB20006E2D41E00E94334F65E0E62EE10E8E2D12
:10DB30006B2D4E2D282D0E944150812F8A5F692D1B
:10DB400041E00E94334F8C2D6B2D41E00E94334FFA
:10DB50006F2D6B5F8C2D41E00E94334F8D2D6A2D10
:10DB60004E2D2A2D0E9441501F910F91FF90EF9052
:10DB7000DF90CF90BF90AF909F908F900895A0E0DE
:10DB8000B0E0E5ECFDE60C9445F2F62E182F110FEF
:10DB9000180F110FFF0CFF0CFF0C07E0E02EEF0C2D
:10DBA000C12FD0E02396CE2CDD248DEF9FEFC80E41
:10DBB000D91ECE01B60144E050E021E00E94355369
:10DBC0002F2D2C5F412F4A5F812F622F01E00E9491
:10DBD0004150412F4D5F2F2D2F5F842F6E2D0E94BE
:10DBE0004150CE01B60142E050E021E00E943553A1
:10DBF000CDB7DEB7E8E00C9461F28F929F92AF92BE
:10DC0000BF92CF92DF92EF92FF920F931F93982EC5
:10DC1000862ECA01B901D02EBE2CAC2C0E94D7EFA3
:10DC20007B018C0120E030E048E453E40E94C0F026
:10DC3000181654F0C801B70120E030E048E453EC76
:10DC40000E9435EF87FF17C0C801B70120E030E020
:10DC500040EA51E40E943CEF0E94A4EF9B01AC011A
:10DC6000892D682DA90124E030E000E0ED2CCB2CBB
:10DC70000E94675716C0C801B70120E030E040E0BD
:10DC80005FE30E94C4F00E94A4EF9B01AC01892DC8
:10DC9000682DA90123E030E000E0ED2CCB2C0E94A0
:10DCA00031581F910F91FF90EF90DF90CF90BF9070
:10DCB000AF909F908F90089521E335E1D901F9014C
:10DCC000719791E101900D929150E1F7215130400F
:10DCD00093E12E3E390791F78093EE13D901119607
:10DCE000E4E2FCE188E001900D928150E1F70895B3
:10DCF000CF92EF920F9382E790E00E94EA5DAC0131
:10DD000080E060E022E00E94635283E790E00E949E
:10DD1000EA5DAC0180E062E020E00E94635284E7AB
:10DD200090E00E94EA5DAC0180E063E020E00E94A8
:10DD300063528AE090E00E94EA5DAC0180E065E019
:10DD400020E00E94635220913C0E30913D0E4091A4
:10DD50003E0E50913F0E81E066E000E0EE24CC24C0
:10DD60000E9428592091380E3091390E40913A0E78
:10DD700050913B0E8CE066E00E9428590F91EF9085
:10DD8000CF9008951F93182F2CE231E03093211C7F
:10DD90002093201C109280058091D71B883229F097
:10DDA00088E28ADF88E28093D71B112371F080E03C
:10DDB00090E060E070E042E00E9429BB0E94C24E09
:10DDC0008AEF90E060E470E008C08091450E8130F9
:10DDD00039F488EC90E060E870E040E00E9429BBF4
:10DDE00087DF81E02ADA1F910895EF92FF920F9367
:10DDF0001F93CF93DF93EC01FB01122FCA01880F11
:10DE0000991F840F951F880F991F62E070E00E9490
:10DE1000EBF19B012296BE01660F771F6C0F7D1FF1
:10DE2000660F771F83E0EE0FFF1F8A95E1F76E5FA5
:10DE30007F4F802F992787FD90953B96FF24E7FC25
:10DE4000F094EE0DFF1DA901425050402550304086
:10DE5000860F971FBF01012F0E947454CDB7DEB704
:10DE6000E6E00C9463F2AF92CF92EF920F931F9380
:10DE7000CF93DF93FB01D901202F0296EC01CC0F49
:10DE8000DD1FC80FD91FCC0FDD1F73E0EE0FFF1F82
:10DE90007A95E1F7842F880F840F880F63E00E9442
:10DEA000CBF1280F22963B96AE0EAE014C0D842F7F
:10DEB0006A2D422F8D010E941654DF91CF911F9140
:10DEC0000F91EF90CF90AF900895DF92EF92FF9275
:10DED0000F931F93182FF62E95E0E92EE60E6E2D68
:10DEE0004AE028E001E00E94F75285E0D82ED10EEA
:10DEF0008D2D6F2D412F2E2D0E944150412F465FB9
:10DF00008D2D6F2D2E2D0E9441506F2D665F812F1C
:10DF10008C5F42E023E00E94F7521F910F91FF9027
:10DF2000EF90DF900895CF92DF92EF92FF920F93E0
:10DF30001F93182FF62E52E0E52EE60E6E2D44E0CC
:10DF400022E001E00E94F752812F885F6E2D44E0AD
:10DF500022E00E94F752812F8C5F6F2D44E026E073
:10DF60000E94F75246E0C42EC10E37E0D32EDF0CDC
:10DF70002BE0E22EEF0C412F4E5F8C2D6D2D2E2DC0
:10DF80000E944150412F465F8C2D6D2D2E2D0E94F9
:10DF900041502F2D245F412F455F812F8F5F622FCE
:10DFA0000E9441501F910F91FF90EF90DF90CF9012
:10DFB0000895FF920F931F93182FF62E8E5F42E065
:10DFC00022E001E00E94F7526F2D6E5F812F46E044
:10DFD0002FE00E94F7521F910F91FF900895EF924A
:10DFE000FF920F931F93062F182F110F180F110F69
:10DFF000000F000F000FF02EF394E12EE394602F3A
:10E000006B5F812F8C5F41E00E94334F202F2D5F8B
:10E01000412F4B5F812F8D5F622F01E00E944150A5
:10E02000412F4A5F8E2D8F5F6F2D2F2D0E94415003
:10E030001F910F91FF90EF900895ACE2B0E0E3E202
:10E04000F0E70C9445F2F82ED62EC42E322F102F66
:10E050008CEB94E39A83898389EB94E39C838B8391
:10E0600086EB94E39E838D8383EB94E398878F8381
:10E0700080EB94E39A8789878DEA94E39C878B876A
:10E080008AEA94E39E878D8787EA94E3988B8F874B
:10E0900084EA94E39A8B898B81EA94E39C8B8B8B43
:10E0A0008EE994E39E8B8D8B8BE994E3988F8F8B15
:10E0B00088E994E39A8F898F85E994E39C8F8B8F0D
:10E0C00082E994E39E8F8D8F8FE894E398A38F8FDE
:10E0D0008CE894E39AA389A389E894E39CA38BA397
:10E0E00086E894E39EA38DA383E894E398A78FA387
:10E0F00080E894E39AA789A78DE794E39CA78BA770
:10E10000662331F0660F660F660F615028E002C08B
:10E1100027E060E0FF2039F08F2D880F8F0D880FEA
:10E1200082504EE002C04CE080E0810F6E0D332340
:10E1300091F001E00E94D950EC2DF0E0EE0FFF1FAE
:10E14000EC0FFD1F418152818F2D6D2D22E0012F9B
:10E150000E94545203C000E00E94D950AC96E8E0FF
:10E160000C9461F2EF920F93922FE02EE42FF0E0E7
:10E17000E631F10508F05FC0E759FF4FA091D81BC9
:10E18000B091D91B0C9472F2A65BBF4F02C0AC5B7E
:10E19000BF4F2C91227050C0AC5BBF4F0EC0A65B2E
:10E1A000BF4F13C0A65BBF4F34C0A65BBF4F36C086
:10E1B000AD5BBF4F38C0AD5BBF4F2C9124703CC0EE
:10E1C000AD5BBF4F26C0AD5BBF4F2C91217034C0FB
:10E1D000AD5BBF4FDECFAD5BBF4F20C0A65BBF4F77
:10E1E000ECCFAC5BBF4F0DC0AC5BBF4F2C9120950B
:10E1F000221F2227221F20C0AD5BBF4F19C0AD5B7D
:10E20000BF4F2C91207818C0AC5BBF4FDECFAC5B0A
:10E21000BF4F2C91287010C0AC5BBF4F2C91207168
:10E220000BC0AC5BBF4F2C91207206C0AC5BBF4FE4
:10E230002C91207401C020E0092FFFDE0F91EF9098
:10E240000895A1E0B0E0E7E2F1E70C944AF2182F5C
:10E25000E091D81BF091D91BE65BFF4F808181FFD5
:10E2600003C085E990E002C084E990E069830E94E0
:10E27000EA5DAC01812F698120E00E946352219602
:10E28000E3E00C9466F2DF92EF92FF920F931F93FC
:10E29000142FF22E982F990F980F990F190F660FC0
:10E2A000660F660FF60E812F6F2D46E027E000E027
:10E2B0000E94D950E091D81BF091D91B05A8F6A96E
:10E2C000E02DE330F1059CF0A2E0DA2ED10EF2E071
:10E2D000EF2EEF0C8D2D6F2D412F2E2D01E00E9482
:10E2E0004150412F4C5F8D2D6F2D2E2D18C08FEF7B
:10E2F000EE3FF807B4F4E2E0DE2ED10E76E0E72E32
:10E30000EF0C84E0F80E8D2D6E2D412F2F2D01E0A6
:10E310000E944150412F4C5F8D2D6E2D2F2D0E945C
:10E3200041501F910F91FF90EF90DF900895BF92A1
:10E33000CF92DF92EF92FF920F931F93182FB62E7A
:10E34000423039F448E754E320E00E9463521C5FF6
:10E3500005C08B5F49E020E00E94A352E091D81BEA
:10E36000F091D91B63A974A9882777FD8095982F10
:10E370000E94D7EF6B017C0120E030E048E453E4D9
:10E380000E94C0F0181654F0C701B60120E030E03A
:10E3900048E453EC0E9435EF87FF16C0C701B60171
:10E3A00020E030E040EA51E40E943CEF0E94A4EFFC
:10E3B0009B01AC01812F6B2DA90124E030E000E02E
:10E3C000EE240E949D5715C0C701B60120E030E041
:10E3D00040E05FE30E94C4F00E94A4EF9B01AC0107
:10E3E000812F6B2DA90123E030E000E0EE240E9494
:10E3F0006958812F8C5F6B2D46E754E320E00E9423
:10E4000063521F910F91FF90EF90DF90CF90BF90DC
:10E410000895A0E0B0E0EFE0F2E70C9444F2182F8A
:10E42000B62EE091D81BF091D91B91AD8091920549
:10E43000981710F492E001C090E09093BB1B4091BC
:10E440009105442309F4CAC0812F8A5F6B2D50E0E7
:10E4500021E030E000E0E92E0E945B57812F895FC8
:10E460006B2D44E754E32091BB1B0E9463528091C3
:10E470009105833009F04EC0F12EFF0CF10EFF0C18
:10E48000EB2CEE0CEE0CEE0C8F2D6E2D4CE127E0FC
:10E4900001E00E94F7522091910530E030952195DE
:10E4A0003F4FF5E0220F331FFA95E1F7E091D81BBB
:10E4B000F091D91B81AD280F311DC901880F991F1B
:10E4C00073E0220F331F7A95E1F7820F931F6CE000
:10E4D00070E00E94EBF16B01EB01CB0101978B31F6
:10E4E000910540F46E2D6F5F8F2D8F5F4C2D25E0D1
:10E4F0000E94D9502BE1C216D10470F48C2DF394F4
:10E500006E2D6F5F4AE14C198F0D25E000E00E94EF
:10E51000D95002C0C0E0D0E0809191058450823093
:10E5200008F05CC0F12EFF0CF10EFF0CBB0CBB0C15
:10E53000BB0C8F2D6B2D4EE127E001E00E94F752BE
:10E54000809191058430A9F4E091D81BF091D91BFA
:10E5500021AD30E020583040C901880F991F53E0A9
:10E56000220F331F5A95E1F7820F931F6FE070E07F
:10E5700016C08530B9F4E091D81BF091D91B21ADBC
:10E5800030E0205A3040C901880F991FB3E0220FB4
:10E59000331FBA95E1F7820F931F63E170E00E9489
:10E5A000EBF1EB01CE0101978D31910548F46B2D14
:10E5B0006F5F8F2D8F5F4C2F25E001E00E94D950B7
:10E5C000CC31D10558F48C2FF3946B2D6F5F4CE157
:10E5D0004C1B8F0D25E000E00E94D950CDB7DEB76F
:10E5E000E9E00C9460F2AF92BF92CF92DF92EF928B
:10E5F000FF920F931F93F82EB62ED42E122FE09178
:10E60000D81BF091D91B41AD80919205481710F4A9
:10E6100092E001C090E09093BB1B8F2D6B2D50E0DA
:10E6200023E030E000E0E92ECD2CA12E0E94A95776
:10E630000D2D0F5F8F2D8C5F6B2D42E754E32091E2
:10E64000BB1BE12E0E9454524F2D440F4F0D440F1F
:10E65000485E6B2D660F660F660F262F295F01E05F
:10E660008091BB1B823009F000E0842F0E94415052
:10E670001F910F91FF90EF90DF90CF90BF90AF90E0
:10E680000895AF92CF92EF920F938091BC1B81308F
:10E6900079F581E260E041E229E001E00E94415029
:10E6A0008DE560E04DE529E00E94415080E06AE0A0
:10E6B0004FE72AE00E9441508CE060E041E154E3E2
:10E6C00020E00FEFEE240E94545280E06AE040E028
:10E6D0002FE301E00E9441508FE76AE04FE72FE30C
:10E6E0000E94415080E06FE34FE72FE30E944150CA
:10E6F00080E060E040E020E076DFE091D81BF09120
:10E70000D91BE05BFF4F4081518180914C0E90916D
:10E710004D0E8417950710F492E001C090E090939D
:10E72000BB1B87E060E025E030E000E0E92EADEFC4
:10E73000CA2EAA240E942557E091D81BF091D91B1C
:10E7400047A950AD80E160E020E002E0EE240E94A5
:10E75000755883E162E042E029EF0EEF03DD83E1CB
:10E7600064E040E029EF0BEFFDDC83E166E041E08F
:10E7700029EF08EFF7DC83E167E043E029EF0DEFD5
:10E78000F1DC80E162E046E022EF0EEFEBDC80E1BD
:10E7900064E04BE022EF0BEFE5DC80E166E042E174
:10E7A00022EF08EFDFDC80E167E04EE022EF0DEFC3
:10E7B000D9DC8CE062E047E021EF0EEFD3DC8CE0A7
:10E7C00064E048E021EF0BEFCDDC8CE066E049E04F
:10E7D00021EF08EFC7DC8CE067E04AE021EF0DEFA6
:10E7E000C1DC89E062E044E02BEE0EEFBBDC89E0A7
:10E7F00064E045E02BEE0BEFB5DC89E066E044E138
:10E800002BEE08EFAFDC89E067E045E12BEE0DEF82
:10E81000A9DC86E062E04FE025EE0EEFA3DC86E0A7
:10E8200064E040E125EE0BEF9DDC86E066E041E12F
:10E8300025EE08EF97DC86E067E043E125EE0DEF7B
:10E8400091DC0F91EF90CF90AF900895A1E0B0E0F0
:10E85000ECE2F4E70C943BF28091BC1B813071F543
:10E8600081E260E041E229E001E00E9441508DE553
:10E8700060E04DE529E00E94415080E069E04FE70B
:10E8800029E00E94415080E06AE040E02FE30E94CE
:10E8900041508FE76AE04FE72FE30E94415080E04C
:10E8A0006FE34FE72FE30E94415086E060E047E1CD
:10E8B00054E320E002E0EE240E94545280E060E045
:10E8C00040E020E090DE8CE060E04EE025E000E0FB
:10E8D00049DCE091D81BF091D91B47A950AD80E1EC
:10E8E00060E020E002E0EE240E9475585CEF652EA7
:10E8F00052E1752E42E0B42E9BE04424552439E1C8
:10E90000232E312C2CEFD22ED40C420180E0692F23
:10E910004FE727E001E099830E94D9500894411CF9
:10E92000511C80E06B2DA20121E030E000E092E07C
:10E93000E92E14E0C12EAD2C0E942557829CF001D7
:10E94000839CF00D929CF00D1124EC50FD4E84E060
:10E950006B2DE080F1800281138124813581468115
:10E960005781B2E0CB2EAA248D2C0E94CB5884E193
:10E970006B2D45E154E322E000E0ED2C0E9454525F
:10E98000F30120813181442737FD4095542F80E1E8
:10E990006B2D02E0EE24CD2C30D99981292F285FF0
:10E9A00081E0622F4DE700E00E9441501B2D1F5F68
:10E9B000F301208531854285538581E0612F0E94D6
:10E9C0002859F30124813581468157818CE0612FDC
:10E9D0000E94285999819F5EF2E0BF0E29E130E044
:10E9E000620E731E9E3309F08DCF2196E2E10C94E6
:10E9F00057F2EF92FF920F931F93182FF62EE0918C
:10EA0000D81BF091D91B21AD80919205281710F4E5
:10EA100092E001C090E09093BB1B423009F41D5F6F
:10EA2000812F6F2D422F50E023E030E000E0E92EEF
:10EA30000E94E157812F8C5F6F2D40E754E32091B6
:10EA4000BB1B0E9463521F910F91FF90EF9008959E
:10EA5000CF92DF92EF92FF920F931F93E82EF62E44
:10EA6000D42E122F60919105E42FF0E042E2649FD2
:10EA7000402D112450E0A091D81BB091D91BD996FC
:10EA80002C91D99730E0241B350BE29FC001E39F06
:10EA9000900DF29F900D11242AE2629F602D1124A7
:10EAA00070E0641B750B0E94EBF1C62E67FDCC2451
:10EAB0008C2D992787FD9095E817F9070CF4CD2C3C
:10EAC000113009F410E02D2D2C19013069F48E2D30
:10EAD0006F2D412F00E00E94D9506D2D6F0D6C19E4
:10EAE0008E2D412F2C2D0CC08C2D8E0D6F2D422F75
:10EAF000212F00E00E94D9508E2D6F2D4C2D212FFB
:10EB000001E00E94D9501F910F91FF90EF90DF908C
:10EB1000CF900895A0E0B0E0E0E9F5E70C9440F272
:10EB20008091BC1B813009F056C080E063E14FE763
:10EB300023E101E00E94415080E069E24FE729E2D1
:10EB40000E94415080E06FE34FE72FE30E94415065
:10EB500081E260E041E223E10E9441508DE560E006
:10EB60004DE523E10E94415080E063E140E020E474
:10EB70000E9441508FE763E14FE720E40E9441503B
:10EB80008CE060E04DE054E320E00FEFEE240E94C3
:10EB900054528CE061E04BE054E320E0E2E0EE2EE2
:10EBA0000E9454524091910583E161E050E021E0E0
:10EBB00030E000E0EE2472E0C72E92E0A92E0E9421
:10EBC000255784E161E049E054E320E002E012E0EF
:10EBD000E12E0E94545280E060E040E020E003DD3E
:10EBE00080E069E04EE121E002E032DFE091D81BF5
:10EBF000F091D91BE05BFF4F4081518180914C0E19
:10EC000090914D0E8417950710F492E001C090E0AA
:10EC10009093BB1B87E060E025E030E000E0E92E48
:10EC2000BDEFCB2EAA240E942557E091D81BF0916E
:10EC3000D91B47A950AD80E160E020E002E0EE245E
:10EC40000E947558E091D81BF091D91BE25BFF4FF1
:10EC50004081518187E061E024E030E000E0A2E003
:10EC6000AA2E0E94A95788249924F5E0DF2EBB2400
:10EC7000BB2019F4E7EFFE2E02C07DEFF72E7D2CAE
:10EC80007A94E401CC0FDD1FCC0FDD1FC80DD91D18
:10EC9000CA5AD44E11E08B81807F19F149814423F7
:10ECA000A1F0812F672D50E023E030E000E0EE245A
:10ECB000CC24AF2C0E942557812F8D5F672D4BE010
:10ECC00020E001E0EF2C0E940E514881812F6D2D34
:10ECD00050E023E030E000E0EE24CC24AF2C0E9492
:10ECE000A95725961B5F1531B1F6B39482E0D80E73
:10ECF00084E090E0880E991E9B2D923009F0B8CFE9
:10ED0000CDB7DEB7EDE00C945CF2AF92CF92EF920C
:10ED10000F93CF93DF938091BC1B813009F06DC0BE
:10ED200080E06CE14FE72CE101E00E94415080E07F
:10ED300063E34FE723E30E94415081E460E041E454
:10ED400022E30E94415080E064E033D987E062E032
:10ED50004DE354E320E000E032E0E32E0E94545201
:10ED60008CE060E048E354E320E0EE240E9454523B
:10ED70008CE061E043E354E320E0EE24E3940E945E
:10ED8000545284E161E04BE020E001E00E940E512A
:10ED90008CE062E04EE254E320E000E092E0E92EF5
:10EDA0000E94545284E162E041E420E002E00E94CB
:10EDB0000E5180E061E2B7D886E065E049E254E3B5
:10EDC00020E000E0EE24E3940E94545286E460E2E6
:10EDD0007CD884E164E04DE620E002E0EE240E946D
:10EDE0000E5184E165E04BE020E001E0EE24E39485
:10EDF0000E940E5184E167E0F2D882E068E04BE0C7
:10EE000022E001E025DE82E060E040E020E0EBDB94
:10EE100088E060E046E020E000E0A4D9E091D81B63
:10EE2000F091D91B47A950AD82E061E020E0EE24CB
:10EE3000E3940E947558E091D81BF091D91BE05BD8
:10EE4000FF4F4081518180914C0E90914D0E84175F
:10EE5000950710F492E001C090E09093BB1B82E014
:10EE600062E025E030E000E0E92ECC24B2E0AB2EF9
:10EE70000E942557E091D81BF091D91B23A934A9F2
:10EE8000442737FD4095542F80E160E0EE240E9436
:10EE9000FD6D84E160E042E020E0F5D9E091D81B0F
:10EEA000F091D91B86AD97AD68E671E00E94EBF159
:10EEB000AC0181E161E023E030E0AA24A3940E9448
:10EEC0002557E091D81BF091D91BE25BFF4F808161
:10EED0009181CAE0D0E0BE010E94D7F1AB0181E18F
:10EEE00062E023E030E0A2E0AA2E0E942557E091E4
:10EEF000D81BF091D91B42A984E064E050E022E0E5
:10EF000030E00E945B5788E064E04EE02FEF2AD9A2
:10EF1000E091D81BF091D91B22AD33AD40E050E019
:10EF2000CA01B901F3E0660F771F881F991FFA9590
:10EF3000D1F7620F731F841F951F2AEF30E040E066
:10EF400050E00E94FEF183E065E0A90123E030E09B
:10EF5000AA24A3940E942557E091D81BF091D91BB5
:10EF600084A595A5BE010E94D7F1AB0181E164E0C3
:10EF700023E030E00E945B574091DA1B5091DB1B8D
:10EF800080E165E024E030E00E94255781E067E001
:10EF900042E020E0E7D884E067E040E020E0E2D80B
:10EFA00087E067E041E020E0DDD88AE067E043E009
:10EFB00020E0D8D88DE067E04BE020E0D3D8E091A6
:10EFC000D81BF091D91BEE5BFF4F408181E167E0D8
:10EFD00050E023E030E00E945B57DF91CF910F912A
:10EFE000EF90CF90AF90089590914F0E992309F034
:10EFF00010CAFFCCEF92FF920F931F93F82E162F9B
:10F00000E091D81BF091D91BE05BFF4F408151810B
:10F0100080914C0E90914D0E8417950710F492E05C
:10F0200001C090E09093BB1B8F2D612F25E030E055
:10F0300000E0E92E0E945B578F2D8B5F612F4CE61D
:10F0400054E32091BB1B0E9463521F910F91FF90CC
:10F05000EF900895A1E0B0E0E0E3F8E70C944AF205
:10F06000182FE091D81BF091D91BE65BFF4F8081F0
:10F0700080FF03C027E930E002C026E930E0C90183
:10F0800069830E94EA5DAC01812F698120E00E94C2
:10F0900063522196E3E00C9466F2EF92FF920F9395
:10F0A0001F93182FF62E423018F0423059F515C034
:10F0B000E091D81BF091D91B86AD97AD68E671E061
:10F0C0000E94EBF1AC01812F6F2D23E030E000E0D6
:10F0D000EE240E945B571D5F15C0E091D81BF09194
:10F0E000D91B86AD97AD68E671E00E94EBF1AC01EB
:10F0F000812F8B5F6F2D23E030E000E0EE240E9433
:10F100005B57185F812F6F2D4EE120E00E94A352C4
:10F110001F910F91FF90EF9008950F931F93082F69
:10F12000162FE091D81BF091D91B86AD97AD68E6FC
:10F1300071E00E94EBF10E940A6CE82FF0E0EE0F04
:10F14000FF1FEA57FC4C25913491802F612FA901B4
:10F1500020E00E9463521F910F910895A0E0B0E05B
:10F16000E4EBF8E70C9444F2E091D81BF091D91B42
:10F1700086A597A588599E4F26AD37AD821B930B68
:10F18000C8E6D1E0BE010E94EBF1C82EB92E8AE19B
:10F1900060E244E620E201E00E9441508FE360E03B
:10F1A0004FE32FE30E9441508DE36BE041E42BE0FD
:10F1B0000E94415088E26EE148E222E20E94415002
:10F1C00086E56EE146E522E20E9441508DE365E36B
:10F1D00041E425E30E9441508BE690E00E94EA5D05
:10F1E000AC0189E060E020E00E9463528DE690E08F
:10F1F0000E94EA5DAC0183E063E020E00E9463527C
:10F200008EE690E00E94EA5DAC0181E163E020E0DF
:10F210000E9463528CE690E00E94EA5DAC0189E0B6
:10F2200067E020E00E9463528FE690E00E94EA5D72
:10F23000AC0180E060E020E00E946352E091D81BC6
:10F24000F091D91BE05CFF4F4081552747FD509559
:10F2500082E060E023E030E000E0EE240E949D5771
:10F2600085E060E04BE020E00E94A35280E790E060
:10F270000E94EA5DAC0180E067E020E00E946352FA
:10F28000E091D81BF091D91BEF5BFF4F40815527D0
:10F2900047FD509582E067E023E030E00E949D57F3
:10F2A00085E067E04BE020E00E94A35281E790E018
:10F2B0000E94EA5DAC018DE060E020E00E946352B4
:10F2C000E091D81BF091D91B86AD97ADBE010E948D
:10F2D000EBF1AC018FE060E023E030E00E945B578F
:10F2E00082E160E04BE020E00E94A35283E160E015
:10F2F00014DFE091D81BF091D91BDF01A05CBF4F58
:10F300008C91992787FD909522E030E0B9010E9409
:10F31000EBF1709561957F4F70E2F72EF60EEF5B83
:10F32000FF4F8081992787FD9095B9010E94EBF1ED
:10F33000709561957F4F5FE3D52ED60E609186055F
:10F340008091870590E070E049E050E028E030E0EF
:10F350000E94745400918805109189058091870559
:10F360006091860548E027E00E9416548D2D90E0BC
:10F370006F2D70E049E050E028E030E001E00E94AD
:10F3800074548D2D6F2D48E027E00C2D1B2DEE249D
:10F39000E3940E941654C0928805B0928905F092B9
:10F3A0008605D0928705CDB7DEB7E9E00C9460F210
:10F3B0000F931F93082F162FE091D81BF091D91BA4
:10F3C00026AD37ADC90168E671E00E94EBF1AC01F2
:10F3D000802F612F20E000E00E94436C1F910F916D
:10F3E0000895EF92FF920F931F93F82E162FE0913E
:10F3F000D81BF091D91BE25BFF4F4081518123E084
:10F4000030E000E0EE240E94E1578F2D8C5F612FE9
:10F410004AE654E320E00E9463521F910F91FF904F
:10F42000EF9008950F931F93082F162FE091D81B8C
:10F43000F091D91B47A950AD0E94C258802F8B5F15
:10F44000612F48E654E320E00E9463521F910F9120
:10F450000895EF92FF920F931F93F82E162FE091CD
:10F46000D81BF091D91B22AD33AD40E050E0CA016A
:10F47000B901E3E0660F771F881F991FEA95D1F75E
:10F48000620F731F841F951F2AEF30E040E050E0A9
:10F490000E94FEF18F2D612FA90123E030E000E0F2
:10F4A000EE240E945B578F2D8D5F612F44E654E35D
:10F4B00020E00E9463521F910F91FF90EF900895FA
:10F4C0008F929F92AF92BF92CF92DF92EF92FF9274
:10F4D0000F931F93B82E962E842ED22E102FFE2C13
:10F4E0000E94EA6B8B2D90E0692D70E0482D50E072
:10F4F00021E00E94F56E20918805309189052C54F9
:10F500003F4F8B2D90E0692D70E0482D0D2DEE249E
:10F51000C12EAF2C0E94336F2091DA1B3091DB1B80
:10F520002C543F4F8B2D90E0692D70E0482DEE2438
:10F53000E3940E94336F8091DA1B9091DB1B9093D0
:10F540008905809388051F910F91FF90EF90DF90C0
:10F55000CF90BF90AF909F908F9008958F929F9281
:10F56000AF92CF92EF920F931F93CF93DF9380913F
:10F57000BC1B813031F581E260E041E22BE001E02B
:10F580000E9441508FE560E04FE52BE00E94415022
:10F5900080E06CE04FE72CE00E94415080E062E0A8
:10F5A00044E254E320E000E0A2E0EA2E0E9454523C
:10F5B00080E065E04EE154E320E0F3E0EF2E0E94AE
:10F5C000545280E060E040E020E00DD880E069E047
:10F5D0004EE121E002E03CDAE091D81BF091D91B2A
:10F5E00086AD97ADE8E68E2EE1E09E2EB4010E9436
:10F5F000EBF1AC0186E060E022E000E00E94436CA9
:10F60000E091D81BF091D91B47A950AD80E160E093
:10F6100020E002E0EE240E947558E091D81BF091A2
:10F62000D91B23A934A9442737FD4095542F80E0E6
:10F6300063E000E073E0C72E0E94FD6D84E063E0AC
:10F6400041E023E00E944371E091D81BF091D91B67
:10F6500084A595A56AE070E00E94D7F1AB0180E037
:10F6600066E024E030E0CC2494E0A92E0E942557E7
:10F6700084E066E04CE154E320E002E014E0E12E97
:10F680000E94545288E063E049E024E0B3E0EB2EAE
:10F6900017DF85E361E246E12AE000E00E94D950ED
:10F6A00084E360E248E12CE001E00E94F7528FE33E
:10F6B0006CE342E022E00E94D950C091DA1BD09165
:10F6C000DB1BC43BD10534F0C4018C1B9D0BEC014A
:10F6D00010E001C011E089E064E0AE0123E030E019
:10F6E00000E0EE24A3E0CA2EF3E0AF2E0E942557DF
:10F6F000112349F0209739F086E366E247E326E2DA
:10F7000001E00E94415080E162E046E02DEF00E020
:10F710000E94B27083E162E042E020E00E94B27099
:10F7200083E164E040E020E00DEF0E94B27083E1ED
:10F7300066E041E020E00AEF0E94B27083E167E0FA
:10F7400043E020E00FEF0E94B27080E167E04EE0FE
:10F750002DEF0E94B270DF91CF911F910F91EF902A
:10F76000CF90AF909F908F900895EF92FF920F935C
:10F770001F93F82E162F4091DA1B5091DB1B23E0CC
:10F7800030E000E0EE240E945B578F2D8D5F612FEB
:10F790004EE120E00E94A3521F910F91FF90EF9045
:10F7A0000895EF92FF920F931F93F82E162F423079
:10F7B00020F0423009F042C020C0E091D81BF09107
:10F7C000D91B84A595A56AE070E00E94D7F1AB0132
:10F7D0008F2D612F23E030E000E0EE240E945B5784
:10F7E0008F2D8D5F612F4DE620E00E94A3528F2D5B
:10F7F0008C5F612F0E94526D21C04FE554E320E0E1
:10F800000E946352E091D81BF091D91B84A595A565
:10F810006AE070E00E94D7F1AB018F2D8B5F612F02
:10F8200023E030E000E0EE240E945B578F2D885FDC
:10F83000612F4BE554E320E00E9463521F910F912A
:10F84000FF90EF9008950F931F93CF93DF93E09174
:10F85000D81BF091D91BE65BFF4F9081492321E033
:10F8600009F420E09091460E992311F091E02927A8
:10F8700006E0809F800111240B5F1F4FC62FD0E050
:10F88000B3E0CC0FDD1FBA95E1F723964091470E08
:10F89000C801BE0150E00E94AE53C801BE0143E062
:10F8A00050E021E00E943553DF91CF911F910F91DD
:10F8B000089548E0C8CF40E1C6CFA1E0B0E0E3E65C
:10F8C000FCE70C944AF2182FE091D81BF091D91B59
:10F8D000EC5BFF4F808180FF03C08BE990E009C0A3
:10F8E00081FF03C08CE990E004C082FF0BC08DE96A
:10F8F00090E069830E94EA5DAC01812F698120E07C
:10F900000E9463522196E3E00C9466F2EF92FF921C
:10F910000F931F93F82E162FE091D81BF091D91B4F
:10F92000EE5BFF4F408150E023E030E000E0EE244A
:10F930000E945B57E091D81BF091D91BEC5BFF4F05
:10F9400090818F2D8D5F94FF04C0612F48E554E3B3
:10F9500003C0612F45E554E320E00E94D0521F917F
:10F960000F91FF90EF900895EF92FF920F931F93E6
:10F97000F82E162FE091D81BF091D91BDF01AC5B5C
:10F98000BF4FEC90E094EE1CEE24EE1CEE0CE092E7
:10F99000BB1B423018F0423009F510C042A950E0BC
:10F9A00022E030E000E00E945B578F2D8E5F612FD8
:10F9B00048E02091BB1B0E94A35210C042A950E016
:10F9C00022E030E000E00E945B578F2D8E5F612FB8
:10F9D00040E554E32091BB1B0E9463521F910F919D
:10F9E000FF90EF900895A1E0B0E0E9EFFCE70C9400
:10F9F0004AF2182FE091D81BF091D91BED5BFF4F15
:10FA0000808182FF03C08FE990E01BC083FF03C0A9
:10FA100080EA90E016C080FF03C081EA90E011C048
:10FA200081FF03C082EA90E00CC084FF03C083EA38
:10FA300090E007C085FF03C084EA90E002C08EE931
:10FA400090E069830E94EA5DAC01812F698120E02A
:10FA50000E9463522196E3E00C9466F20F931F9389
:10FA6000660F660F660F982F990F980F695FE091E8
:10FA7000D81BF091D91B05A916A9892F880F4AE038
:10FA80002EE00E94736C1F910F910895EF92FF92E8
:10FA90000F931F93F82E162F423000F5E091D81BDC
:10FAA000F091D91B838D948D6AE070E00E94D7F1AC
:10FAB000AB018F2D612F23E030E000E0EE240E94A7
:10FAC0005B578F2D8D5F612F4DE620E00E94A35282
:10FAD0008F2D8C5F612F0E94BF6D21C04BE454E3DA
:10FAE00020E00E946352E091D81BF091D91B838DD6
:10FAF000948D6AE070E00E94D7F1AB018F2D8B5F8F
:10FB0000612F23E030E000E0EE240E945B578F2D50
:10FB1000885F612F47E454E320E00E9463521F9105
:10FB20000F91FF90EF900895EF92FF920F931F9324
:10FB3000182FF62EE091D81BF091D91B85A996A914
:10FB400097FF05C080959091490E981710F080E0BE
:10FB500001C082E08093BB1B80914A0E882311F084
:10FB60000E942B6B8091BB1B823059F48091570E01
:10FB7000882339F488EE93E060E670E040E00E946C
:10FB800029BBE091D81BF091D91B45A956A9812F1B
:10FB90006F2D23E030E000E0E090BB1B0E9469582D
:10FBA000812F8C5F6F2D44E454E32091BB1B0E9496
:10FBB000D0521F910F91FF90EF900895EF920F9305
:10FBC00081E061E041E00E94977180E067E041E000
:10FBD0000BDA8DE067E00EDA88E067E002DC8DE0AA
:10FBE00060E041E05ADA82E160E097DA8CE061E0BF
:10FBF000DFDB87E066E016DC80E060E02ADC81E0A5
:10FC000063E047E020E000E0EE245ADC88E063E0B7
:10FC1000ACDD87E062E041E0C4DD88E065E04DDE18
:10FC20008FE066E073DE8FE062E07EDF88E064E014
:10FC300041E09ADE89E060E011DF0F91EF900895D6
:10FC4000EF92FF920F931F93F82E162FE091D81B7F
:10FC5000F091D91B40A981E090E020918E052223EC
:10FC600011F080E090E0242F30E08217930729F410
:10FC700040938E0581E080938F0580918F058130C0
:10FC800071F4EC5BFF4F808185FF09C084EF91E048
:10FC900060E870E040E00E9429BB10928F05E0917F
:10FCA000D81BF091D91B40A98F2D8E5F612F50E09A
:10FCB00022E030E000E0EE240E945B578F2D612FA0
:10FCC00041E454E320E00E9463521F910F91FF90A2
:10FCD000EF900895EF920F9380E063E00E9421710E
:10FCE0008BE063E040E00E94977180E067E040E0D5
:10FCF0007BD98DE067E07ED988E067E072DB80E049
:10FD000065E0A8D98DE060E040E0C7D982E160E01D
:10FD100004DA8CE061E04CDB80E061E083DB80E0D2
:10FD200060E097DB80E164E045E020E000E0EE2465
:10FD3000C7DB8CE064E019DD8AE065E040E031DD9E
:10FD40008AE066E040E0A2DE85E066E079DF80E000
:10FD500066E0AFDD83E066E0AEDD80E064E0ADDD6F
:10FD60008CE062E0E1DE82E162E040E0FDDD80E027
:10FD700062E039DE89E060E071DE0F91EF90089576
:10FD8000EF92FF920F931F93F82E162FE091D81B3E
:10FD9000F091D91B858D968D6AE070E00E94EBF1A1
:10FDA000AB018F2D612F23E030E000E0EE240E94B4
:10FDB0005B578F2D8D5F612F4EE120E00E94A35293
:10FDC0001F910F91FF90EF900895EF920F9380E0B5
:10FDD00061E00E94217180E064E042E00E9497713E
:10FDE0008DE067E042E000D980E067E003D988E079
:10FDF00067E0F7DA80E063E02DD98CE063E042E071
:10FE00004CD98FE065E00EDB80E160E045E020E06A
:10FE100000E0EE2455DB8BE065E0A7DC80E065E0E8
:10FE200042E0BFDC80E066E042E030DE8BE066E08E
:10FE3000A7DF8CE062E03DDD8EE062E03CDD80E04B
:10FE400062E03BDD8FE064E06FDE8AE060E042E08C
:10FE50008BDD80E060E0C7DD0F91EF900895EF92B9
:10FE60000F93DF93CF93CDB7DEB76897DEBFCDBFDB
:10FE70001A82198283E00E94C16887E062E045ED42
:10FE800053E320E00EEFEE240E94545285E066E03A
:10FE90004AEC53E322E002E078EFE72E0E9454524E
:10FEA0008FEFBE016F5F7F4F40E00E941D5E882391
:10FEB00059F486E067E040EC53E322E00FEF3CEFBB
:10FEC000E32E0E94545260C0909183059E012D5FE5
:10FED0003F4F992309F14DB75EB7475050405EBF81
:10FEE0004DBFEDB7FEB73196ADB7BEB712963C9396
:10FEF0002E93119796E1928323E831E03483238394
:10FF0000858316820E9458E24DB75EB7495F5F4F06
:10FF10005EBF4DBF06E023C0ADB7BEB71997BEBFE9
:10FF2000ADBFEDB7FEB7319612963C932E93119765
:10FF300096E1928328E831E0348323838583168217
:10FF400089819A818C589F4F908787830E9458E2BD
:10FF50004DB75EB7475F5F4F5EBF4DBF00E0AE017C
:10FF60004D5F5F4FFA0101900020E9F73197E41BE4
:10FF7000F50BF695E79502508AE08E1B67E022E0CC
:10FF80009CEFE92E0E940E528FEF0E94F3BA8AEF87
:10FF900090E09093211C8093201C8091201C9091D4
:10FFA000211C009729F08FEF0E94F3BA8823A9F350
:10FFB00080EF0E94F3BA0E94C24E6896DEBFCDBFAA
:10FFC000CF91DF910F91EF900895AF92CF92EF9282
:10FFD0000F931F93CF93DF93182F83E00E94C16884
:10FFE00082E066E04EEA53E322E002E039EFE32EDE
:10FFF0000E945452C12FD0E08EE066E0AE0122E0B4
:020000021000EC
:1000000030E001E092E0E92E12E0C12EB9EFAB2E14
:100010000E942557FE01EE0FFF1FEC5FFC4C25915F
:10002000349181E067E0A90122E000E0EEEFEE2EDE
:100030000E945452DF91CF911F910F91EF90CF907A
:10004000AF900895AF92CF92EF920F931F93CF93FB
:10005000DF93182FEB0185E00E94C16883E061E225
:100060004CE721E200E00E94415083E065E34CE769
:1000700025E30E94415080E063E0412F50E022E000
:1000800030E001E0F2E0EF2EE5E0CE2EAA24AA94C3
:100090000E94255782E063E04CEA53E322E005E04A
:1000A000EE24EA940E94545285E063E0AE0122E01F
:1000B0000CEF0E94545280E064E040EA53E322E0F7
:1000C00006E074E0E72E0E94545281E165E04BE9BE
:1000D00053E322E000E00E94545283E090E00E944B
:1000E000EA5DAC0180E067E022E00E94635281E1BA
:1000F00067E046E953E322E00E946352DF91CF912B
:100100001F910F91EF90CF90AF900895CF93DF9311
:10011000FC01A091D81BB091D91BD3968D919C91D5
:10012000D497918780879C968D919C919D9793877A
:100130008287EF012C9611968DE00D9009928150E7
:10014000E1F7A4E2BCE188E00D9001928150E1F773
:10015000DF91CF9108958AEFE4EFF2E1DF011D9284
:100160008A95E9F70895E091D81BF091D91BEC5BD3
:10017000FF4F808187FF15C085ED93E1DC01FC0115
:10018000799729E101900D922150E1F7499722E1F9
:10019000843F920799F7BADF80EA90E06FEF7FEF34
:1001A00004C088E592E06FE070E040E00C9429BB69
:1001B000A3E0B0E0EEEDF0E80C943BF20E94C24EFA
:1001C000809181058230B9F480E990E00E94EA5D77
:1001D000AC0180E063E020E00E94635284E690E09E
:1001E0009093211C8093201C8091201C9091211CB5
:1001F0000097D1F706C38091E40D882309F02FDE24
:1002000081E00E941D6911E010938A051092930508
:10021000109291051092940510928E0510928F0500
:100220001092D71B1092BD1B0E94E26681EE90E0F7
:100230000E94EA5DBC0180E045E856E70E94E7665F
:1002400082EE90E00E94EA5DBC0181E04EEA5AE74E
:100250000E94E76683EE90E00E94EA5DBC0182E0C6
:100260004AE855E70E94E76684EE90E00E94EA5D66
:10027000BC0183E041E453E70E94E76685EE90E02D
:100280000E94EA5DBC0184E046E254E70E94E76612
:1002900086EE90E00E94EA5DBC0185E04EEA58E7F8
:1002A0000E94E76687EE90E00E94EA5DBC0186E06E
:1002B00049E857E60E94E76688EE90E00E94EA5D12
:1002C000BC0187E04AE65EE70E94E76689EE90E0BF
:1002D0000E94EA5DBC0188E04EED5DE70E94E766A2
:1002E0008AEE90E00E94EA5DBC0189E045EE5EE79F
:1002F0000E94E76680914E0E0E9429671093BC1BF6
:100300008CE291E09093211C8093201C8DE290E080
:1003100090933A1C8093391C1092381C1092371C11
:1003200010923E1C10923D1C10922F1C10922E1CFD
:1003300010E0EE2490E02CE2622E21E0722E01E02B
:1003400080E9482E81E0582EBCEB2B2EB2E03B2EEC
:100350008091180A882309F41BC20E943ED4E091C0
:100360001A0AF0911B0AF093D91BE093D81B8091D5
:1003700091058823B9F482E08093910542E00CC096
:10038000542F5F5F21AD30E06BE2469FC001112426
:10039000281739071CF0452F473090F340939105FB
:1003A0004093C2120E94EA6B8EEB9BE1AFDE80911C
:1003B000CE1B9091CF1BA091D01BB091D11B8093ED
:1003C0003C0E90933D0EA0933E0EB0933F0E809155
:1003D000CA1B9091CB1BA091CC1BB091CD1B8093DD
:1003E000380E9093390EA0933A0EB0933B0E809145
:1003F000D71B883211F41092D71B8091D81B909193
:10040000D91B9B838A83FC01ED5BFF4F808180FFBA
:10041000F6C080912A1C90912B1C009799F0809136
:10042000911290919212009769F4ABE8B2E1E4E284
:10043000FCE188E02A813B8101900D928150E1F737
:100440003B832A83EA81FB8187A990AD90939E121A
:1004500080939D12E0909F12F090A0120894E11CEE
:10046000F11CF092A012E0929F128090B512909031
:10047000B612AA24BB24E25BFF4FC080D180B60134
:1004800080E090E024E630E040E050E00E94ACF1F3
:10049000681979098A099B09970140E050E00E9498
:1004A00020F2280D391D4A1D5B1D3093B612209392
:1004B000B512EA81FB8183A994A92091A3123091FE
:1004C000A4122817390724F49093A4128093A3123E
:1004D000EA81FB8182AD93AD2091A9123091AA12DD
:1004E0002817390720F49093AA128093A912EA8161
:1004F000FB8184A595A52091AF123091B0122817E9
:10050000390720F49093B0128093AF128091B31208
:100510009091B4128C159D0520F4D092B412C09223
:10052000B312EA81FB81E05BFF4F808191812091D2
:10053000BB123091BC122817390720F49093BC12DB
:100540008093BB12EA81FB8181AD9091C112891722
:1005500010F48093C112EA81FB81E95BFF4F808137
:1005600091812091AD123091AE122817390724F4F1
:100570009093AE128093AD12EA81FB81EE5BFF4F48
:1005800080819091B712981710F48093B712EA8186
:10059000FB81EE5BFF4F80819091B812891710F4B8
:1005A0008093B812EA81FB81E05CFF4F80819091DB
:1005B000BE12891714F48093BE12EA81FB81E05CBD
:1005C000FF4F80819091BD12981714F48093BD1253
:1005D000EA81FB81EF5BFF4F80819091C012891708
:1005E00014F48093C012EA81FB81EF5BFF4F80819E
:1005F0009091BF129817B4F48093BF1213C0EE20ED
:1006000099F080912A1C90912B1C009769F0A3E926
:10061000B2E1E4E2FCE188E001900D928150E1F763
:10062000EE2402C0EE24E3940E94A06B1123C1F4D7
:100630008091391C90913A1C009721F08091BC1B4D
:10064000813071F48091BC1B813011F40E94C24E44
:100650000E944E678DE290E090933A1C8093391C83
:100660001092BC1BE091D81BF091D91BEB5BFF4FA4
:1006700080819091BD1B891739F1833228F5882339
:10068000B9F00E945C6EE091D81BF091D91BEB5B36
:10069000FF4F80819ADC88EE93E06FE070E040E0ED
:1006A0000E9429BB30922D1C20922C1C12E003C00A
:1006B0000093BC1B10E0E091D81BF091D91BEB5BC1
:1006C000FF4F80818093BD1B80E20E9412BBC82E29
:1006D00080E10E9412BB882329F491E0CC2021F410
:1006E00090E002C040DD91E080E199830E94FDBA74
:1006F00099818823B9F01123A1F480917D1BE82F03
:10070000F0E0EE0FFF1FEE0FFF1FE358F44E628183
:10071000738198DC50922D1C40922C1C11E090E0CB
:1007200001C091E080E899830E94F3BA99818823FF
:1007300019F00E94416791E080E499830E94F3BA26
:100740009981882319F00E94326791E0112331F0DA
:10075000992309F44EC00093BC1B09C0992339F4B6
:1007600003C00093BC1B10E00E94496A03C01092B2
:10077000180A10E08091221C9091231C009719F414
:1007800082E00E941D697092211C6092201C91E001
:100790002091201C3091211C2115310551F4892F05
:1007A0000E94C26E7092211C6092201C0093BC1BA0
:1007B00090E080917D1B80934E0E80E299830E9491
:1007C000FDBA9981882309F4C3CDEE2079F0809198
:1007D0002A1C90912B1C009749F0A3E9B2E1E4E2B6
:1007E000FCE188E001900D928150E1F710928A05BA
:1007F00008C080912C1C90912D1C009709F4B1CF5A
:10080000B3CF2396E2E10C9457F2FF920F931F931C
:10081000182F8CE390E06FEF7FEF40E00E9429BB40
:100820000E94C24E80E06AE04FE722E201E00E94AF
:10083000F752133091F0143028F4113041F0123097
:10084000E1F408C0143061F01530B9F40CC086ED45
:1008500090E00BC087ED90E008C088ED90E005C007
:1008600089ED90E002C08AED90E00E94EA5DAC0163
:1008700082E062E020E00E9463528BED90E00E94F3
:10088000EA5DAC0186E064E020E00E9463528BE008
:1008900090E00E94EA5DAC0180E067E020E00E9409
:1008A00063528EE190E00E94EA5DAC018CE067E06B
:1008B00020E00E9463528CE067E046E35AE320E0C8
:1008C0000E9463520E94519CF82E80E80E94F3BA65
:1008D000882311F402E001C001E080E10E94F3BA34
:1008E000882331F4023031F4FF2009F099CFEACFA8
:1008F00010E001C011E080EF0E94F3BA812F1F9138
:100900000F91FF90089585E080DF8823A1F00E9479
:1009100000690E9412691FDC60E070E0CB0120E0FA
:1009200030E0A9010E94AB4780E991E06FEF7FEFD3
:1009300040E00C9429BB0895CF92EF920F931F9340
:100940000E94C24E89E090E00E94EA5DAC0180E026
:1009500060E022E00E9463528CE090E00E94EA5D39
:10096000AC0180E061E022E00E9463528AE090E006
:100970000E94EA5DAC0180E062E022E00E946352E6
:1009800084E090E00E94EA5DAC018CE067E020E04A
:100990000E94635282E167E04FE857E320E00E9443
:1009A000635220913C0E30913D0E40913E0E50918D
:1009B0003F0E81E064E000E0EE24CC240E94285940
:1009C0002091380E3091390E40913A0E50913B0EE5
:1009D0008CE064E00E9428590E94519C182F80E20C
:1009E0000E94F3BA8823E9F480E10E94F3BA8823D5
:1009F00021F4112309F0A4CFEFCF84E006DF882390
:100A000009F49ECF80E991E06FEF7FEF40E00E9414
:100A100029BB60E070E0CB0120E030E0A9010E943A
:100A2000AB471F910F91EF90CF9008951F93162F12
:100A3000882371F400D00F92EDB7FEB7118226E241
:100A40003AE3338322830E9482DE0F900F900F904F
:100A500084E063E971E00E9494DE0E944DDF8430FF
:100A6000F1F4812FD2DE8823A9F0123039F013304F
:100A700041F0113039F40E94006904C00E941269EB
:100A800001C069DB80E991E06FEF7FEF40E00E94F9
:100A900029BB07C00E94C24E0E94A9DEDECF882378
:100AA000E1F61F910895A9E0B0E0E9E5F5E80C94BE
:100AB0003BF20E94C24E83E50E94EFDD882309F4D9
:100AC000C3C000D00F9282E0ADB7BEB711968C9331
:100AD000119782EC97E313969C938E9312970E9442
:100AE00082DE3EEEC32E33E1D32E0F900F900F9097
:100AF000EE24FF2480E01E010894211C311C2CE30D
:100B0000422E512C612C712CF6019081992309F40D
:100B100087C00E9435DEB70194E0660F771F9A9573
:100B2000E1F76E0D7F1D61517C4EC1010E949FE275
:100B300089809A80AB80BC802DB73EB72F50304063
:100B40003EBF2DBF0DB71EB70F5F1F4FADB7BEB76E
:100B500011961C9223EA37E3F80132832183C50101
:100B6000B40120E13EE040E050E00E94FEF1D801F7
:100B700014963C932E931397C501B401A3019201DF
:100B80000E94FEF14B015C01CA01B901A30192016F
:100B90000E94FEF1F80176836583908687828D81BD
:100BA000818712868E81838714868F8198859687A8
:100BB00085870E9482DE2DB73EB7265F3F4F3EBF3E
:100BC0002DBFEDB7FEB73196ADB7BEB711961C92EB
:100BD00028E937E332832183D6018C918383148201
:100BE0000E9482DED601EC91F0E0EE0FFF1FEC5F79
:100BF000FC4C85919491EDB7FEB73196ADB7BEB779
:100C000011961C9223E937E33283218383839483F3
:100C10000E9482DE0F900F900F900F900F9081E056
:100C20000894E11CF11CA1E1B0E0CA0EDB1EB4E1A6
:100C3000EB16F10409F068CF89870E9435DE8985BB
:100C400062E0F4DE0E9428DE2996E2E10C9457F27D
:100C5000A9E0B0E0EEE2F6E80C943BF20E94C24E4E
:100C60008DE20E94EFDD882309F4F7C000D00F92D7
:100C700082E0EDB7FEB7818388E098E393838283B7
:100C80000E9482DE5CEFE52E52E1F52E0F900F9070
:100C90000F908824992480E01E010894211C311CA7
:100CA0004CE3442E512C612C712C8701F8012085D6
:100CB000318542855385211531054105510509F4DA
:100CC000BAC00E9435DE89E190E0889EB001899E1D
:100CD000700D989E700D11246C507D4EC1010E94C4
:100CE0009FE2A980BA80CB80DC80EDB7FEB73F974A
:100CF000FEBFEDBFEDB6FEB60894E11CF11C1182FB
:100D000089EE97E3F701928381838D818383148237
:100D10008E81858316828F81988590878783C6010F
:100D2000B50120E13EE040E050E00E94FEF1F70115
:100D300032872187C601B501A30192010E94FEF10D
:100D40005B016C01CA01B901A30192010E94FEF18D
:100D5000F70174876387B686A5860E9482DE0F90AE
:100D60000F900F900F90EDB6FEB60894E11CF11CA9
:100D7000EDB7FEB711828AED97E3F7019283818385
:100D8000F801648575858685978528EE33E040E017
:100D900050E00E9420F2F701238334834583568379
:100DA000F80160817181882777FD8095982F0E94D6
:100DB000D7EF20E030E040E05FE30E94C4F0F701AD
:100DC00067837087818792870E9482DEEDB6FEB6C8
:100DD0000894E11CF11CEDB7FEB711828DEC97E38E
:100DE000F70192838183F8016085718582859385FF
:100DF0002AE030E040E050E00E9420F2F701238337
:100E0000348345835683F801648175818681978197
:100E10002AE030E040E050E00E9420F2F701278312
:100E20003087418752870E9482DE8DB79EB70B962E
:100E30009EBF8DBF81E00894811C911C075E1F4FEF
:100E40009AE08916910409F031CF89870E9435DE36
:100E5000898563E0EBDD0E9428DE2996E2E10C94AF
:100E600057F2A8E0B0E0E7E3F7E80C943DF27BE846
:100E7000672E72E1772E2E010894411C511CC2018D
:100E8000B3010E949FE2C980DA80EB80FC808DB7BD
:100E90009EB70B979EBF8DBF0DB71EB70F5F1F4F3D
:100EA000EDB7FEB7118289E09AE3F801928381835E
:100EB000C701B60120E13EE040E050E00E94FEF1B3
:100EC000F801348323836CE3862E912CA12CB12C62
:100ED000C701B601A50194010E94FEF1CA01B90142
:100EE000A50194010E94FEF1F801768365838D814E
:100EF000878310868E81818712860E9482DE8DB75D
:100F00009EB70B969EBF8DBFB301685F7F4FC20136
:100F10000E949FE2C980DA80EB80FC80EDB7FEB7CB
:100F20003B97FEBFEDBF0DB71EB70F5F1F4F11827E
:100F30008CEE99E3F80192838183C701B60120E129
:100F40003EE040E050E00E94FEF1F801348323834C
:100F5000C701B601A50194010E94FEF1CA01B901C1
:100F6000A50194010E94FEF1F801768365838D81CD
:100F7000878310868E81818712860E9482DE8DB7DC
:100F80009EB70B969EBF8DBF0E9435DE2896E0E18E
:100F90000C9459F22F923F924F925F926F927F92F0
:100FA0008F929F92BF92CF92DF92EF92FF920F9318
:100FB0001F93DF93CF9300D000D0CDB7DEB70E9450
:100FC000C24E8091C312880F880F865F0E94EFDDAA
:100FD000882309F420C1CE0101960E945C6700D0ED
:100FE0000F9242E0E42EADB7BEB71196EC92119786
:100FF00083EA98E313969C938E9312970E9482DE65
:101000000F900F900F902DDFEDB7FEB73797FEBF13
:10101000EDBF3196ADB7BEB711961C9282E998E349
:10102000928381830DE010E0148303838091B312D7
:101030009091B412968385830E9482DEEDB7FEB74D
:101040003196ADB7BEB711961C9281E898E39283B2
:1010500081838AE090E0948383838091B51290919C
:10106000B61264E670E00E94D7F1658316820E9492
:1010700082DE00D0EDB7FEB73196ADB7BEB71196A0
:101080001C928AE698E39283818314830383898187
:1010900090E00196968385838A81878310860E94DB
:1010A00082DE00D0EDB7FEB73196ADB7BEB7119670
:1010B0001C9284E598E392838183148303838B815C
:1010C00090E00196968385838C81878310868EE1DC
:1010D00090E0928781870E9482DEEDB7FEB73B9653
:1010E000FEBFEDBF0E9435DE8091C312882309F454
:1010F0008DC000D00F92ADB7BEB71196EC9211978C
:101100008BE498E313969C938E9312970E9482DE51
:101110000F900F900F90BB2436E3C32E38E3D32EED
:101120002DE0E22EF12C93E2892E98E3992E8AE0AD
:10113000682E712C04E6402E512C12E1212E18E36A
:10114000312E5FC08B2D90E0EDB7FEB73997FEBF13
:10115000EDBF3196ADB7BEB711961C92D282C18257
:101160009C012F5F3F4F34832383F682E5828C01FD
:10117000000F111F080F191F000F111F0552124FEA
:10118000D801A551BB4F8C91878310860E9482DEC7
:101190000F900F90EDB7FEB73196ADB7BEB7119671
:1011A0001C929282818274826382D801A451BB4FC7
:1011B0008D919C91B2010E94D7F1658316820E94A5
:1011C00082DE00D0EDB7FEB73196ADB7BEB711964F
:1011D0001C9232822182F482E382D801A251BB4F59
:1011E0008C91858316822EE130E0308727830E9420
:1011F00082DE8DB79EB709969EBF8DBF0E9435DEF9
:10120000B3948091C312B81608F49CCF81E061E0DA
:101210000DDC0E9428DE2496DEBFCDBFCF91DF918A
:101220001F910F91FF90EF90DF90CF90BF909F9014
:101230008F907F906F905F904F903F902F90089588
:10124000A4E0B0E0E6E2F9E80C9445F20E94C24E58
:1012500089E10E94EFDD882309F451C2CE01019695
:101260000E945C6700D00F9282E0ADB7BEB71196C6
:101270008C9311978DED99E313969C938E9312970F
:101280000E9482DE0F900F900F90EBDD80919D12F7
:1012900090919E12EDB7FEB73797FEBFEDBF319626
:1012A000ADB7BEB711961C9224EC39E3328321838B
:1012B0006CE370E00E94D7F1748363839683858327
:1012C0000E9482DEEDB6FEB60894E11CF11CEDB77B
:1012D000FEB7118284EB99E3D70112969C938E930B
:1012E00011970DE010E014961C930E9313976091E4
:1012F000A3127091A412882777FD8095982F0E94E1
:10130000D7EF20E030E040EA51E40E943CEF0E9439
:10131000A4EFF701768365830E9482DEEDB7FEB706
:101320003196ADB7BEB711961C9284EA99E39283C9
:101330008183148303838091AF129091B0126AE08D
:10134000C62ED12CB6010E94D7F1768365830E9408
:1013500082DEEDB6FEB60894E11CF11CEDB7FEB7D7
:1013600011828EE899E3D70112969C938E93119780
:1013700014961C930E9313976091A9127091AA1260
:1013800080E090E02AE530E040E050E00E94ACF1DF
:101390002AEF30E040E050E00E94FEF1F701368392
:1013A00025830E9482DE4091AD125091AE1224E25C
:1013B00030E0429FC001439F900D529F900D112439
:1013C000EDB7FEB73196ADB7BEB711961C9228E7C0
:1013D00039E3328321831483038354E6E52EF12C11
:1013E000B7010E94EBF1768365830E9482DEEDB740
:1013F000FEB73796FEBFEDBF0E9435DE00D000D0AD
:101400000F92EDB7FEB73196ADB7BEB711961C92ED
:1014100087E699E3928381838091BB129091BC12FD
:10142000948383830E9482DE00D0EDB7FEB73196AD
:10143000ADB7BEB711961C9286E599E3928381837E
:10144000148303838091B3129091B41296838583A1
:101450000E9482DEEDB7FEB73196ADB7BEB71196EA
:101460001C9285E499E392838183D482C382809124
:10147000B5129091B612B7010E94D7F1658316821A
:101480000E9482DE00D0EDB7FEB73196ADB7BEB791
:1014900011961C9280E399E39283818314830383E2
:1014A000898190E00196968385838A81878310865F
:1014B0000E9482DE00D0EDB7FEB73196ADB7BEB761
:1014C00011961C928AE199E39283818314830383AA
:1014D0008B8190E00196968385838C81878310862B
:1014E0008EE190E0928781870E9482DE8091C11216
:1014F000EDB7FEB73B96FEBFEDBF8F3F11F090E01A
:1015000002C080E090E02DB73EB7275030403EBF8C
:101510002DBFEDB7FEB73196ADB7BEB711961C9291
:1015200029E039E33283218320E130E034832383CF
:10153000968385830E9482DEEDB7FEB73796FEBFA5
:10154000EDBF0E9435DE2DB73EB7275030403EBF7D
:101550002DBFEDB7FEB73196ADB7BEB711961C9251
:1015600089EF98E3928381838DE090E09483838375
:101570008091B712858316820E9482DE8091B81214
:10158000EDB7FEB73796FEBFEDBF8F3F11F090E08D
:1015900002C080E090E02DB73EB7275030403EBFFC
:1015A0002DBFEDB7FEB73196ADB7BEB711961C9201
:1015B00029EE38E33283218320E130E03483238332
:1015C000968385830E9482DE00D0EDB7FEB7319608
:1015D000ADB7BEB711961C928BED98E392838183D1
:1015E0008DE090E0948383838091BD12992787FDDD
:1015F0009095968385838BE090E0908787830E9407
:1016000082DE8091BE12EDB7FEB73996FEBFEDBF08
:101610008E3721F0992787FD909502C080E090E0F9
:101620002DB73EB7295030403EBF2DBFEDB7FEB7B6
:101630003196ADB7BEB711961C922DEC38E33283CC
:10164000218320E130E034832383968385830BE07C
:1016500010E0108707830E9482DEEDB7FEB7319657
:10166000ADB7BEB711961C928FEB98E3928381833E
:101670008DE090E0948383838091BF12992787FD4A
:10168000909596838583108707830E9482DE8091E0
:10169000C012EDB7FEB73996FEBFEDBF8E3721F011
:1016A000992787FD909502C080E090E02DB73EB766
:1016B000295030403EBF2DBFEDB7FEB73196ADB7D4
:1016C000BEB711961C9221EB38E33283218320E1CF
:1016D00030E034832383968385838BE090E090878A
:1016E00087830E9482DEEDB7FEB73996FEBFEDBF5D
:1016F0000E9435DE81E061E099D90E9428DE2496BF
:10170000E8E00C9461F2EF92FF920F931F930E9416
:10171000DBD585E897E30E940FD61BEEE12E16E39A
:10172000F12E81E061E040E259E821EE36E38701E5
:101730000E94B5D7BEEFEB2EB6E3FB2E82E061E050
:101740004AEC57E824EF36E387010E94B5D7A7E1BA
:10175000EA2EA7E3FA2E83E061E043E555E827E0AF
:1017600037E387010E94B5D7F8E3EF2EF7E3FF2EAA
:1017700084E061E048E256E826E237E387010E9410
:10178000B5D7E5E5EE2EE7E3FE2E85E061E04CE916
:1017900054E825E437E387010E94B5D775E7E72EC3
:1017A00077E3F72E86E061E043E854E823E637E389
:1017B00087010E94B5D780E00E9435DB0E9402D6E7
:1017C0001F910F91FF90EF900895A6E0B0E0EBEE2F
:1017D000FBE80C943BF2082F0E94C24E402E552489
:1017E00053E0440C551C5A95E1F7F201E45DF64ACA
:1017F000149180E890E00E94EA5DAC0180E060E036
:1018000022E00E94635281E090E00E94EA5DAC0118
:1018100080E067E020E00E946352163009F4B4C310
:101820004DE2049FA00111249091DE0D8FE0989F5E
:10183000C0011124480F591F4F54534C80E062E0FF
:1018400020E00E946352112309F0D9C084E064E0D3
:101850004AEB50E620E00E9463528CE066E045EBE4
:1018600050E620E00E94635282E090E00E94EA5D30
:10187000AC0180E067E020E00E946352F201E35D8A
:10188000F64AC490F201E25DF64AF4904FE2642E0B
:1018900049E5742E640C751CF3018491E091DC1B06
:1018A000F091DD1BE80FF11D808080919905920178
:1018B000280F311DC901815D964AFC01949085E095
:1018C00064E04C2D50E023E030E000E0EE240E9484
:1018D0005B5789E064E04F2D50E023E030E00E9448
:1018E0005B5781E164E0492D50E023E030E00E9445
:1018F0005B57182D4F2C5524AC2CBB2480E064E0A2
:10190000412F50E023E030E000E0EE240E945B57DE
:10191000C12EDD24C6019695982F88279795879527
:10192000B2010E94EBF1462F80E068E226E001E080
:101930000E94D950FF2DF233A8F080E40E94F3BA40
:10194000082F80E463E00E941DBB802B21F0C414AB
:10195000D5040CF41F5F80E80E94F3BA082F80E8DA
:1019600063E014C080E40E94F3BA082F80E462E0D0
:101970000E941DBB802B21F0C414D5040CF41F5F02
:1019800080E80E94F3BA082F80E862E00E941DBB45
:10199000802BB1F0812F90E0A816B9068CF4019746
:1019A0009695982F882797958795B2010E94EBF11D
:1019B000862F68E240E826E000E00E94D9501150EE
:1019C00080E20E9412BB882341F080E068E240E898
:1019D00026E000E00E94D950192D80E10E94FDBA56
:1019E000882331F0181509F4EDC5F3016490BCC3E8
:1019F00080E20E94FDBA882309F480CFE3C511304C
:101A000009F006C184E064E043EA50E620E00E9469
:101A100063528CE066E04EE950E620E00E9463529B
:101A200082E090E00E94EA5DAC0180E067E020E0A7
:101A30000E946352F201E35DF64AC490F201E25D56
:101A4000F64AA4909201215D364A3A832983F9012E
:101A50008491E091DC1BF091DD1BE80FF11D90807B
:101A6000809199059201280F311DC901815D964A27
:101A7000FC01F490FF2DF83F80F081E164E049E93A
:101A800050E620E00E94635240E051E04F195109B6
:101A900083E164E021E030E006C081E164E04F2DA5
:101AA00050E023E030E000E0EE240E945B57192D67
:101AB000BB242C2C3324612C91E0792E8FEF482EFF
:101AC000512CC12EDD24183F08F40DC680E064E0DF
:101AD00046E950E620E00E94635293012C193D092B
:101AE0003C832B8382E064E0A90121E030E000E048
:101AF000EE240E945B574B814295407F80E068E274
:101B000026E001E00E94D95080E40E94F3BA082F39
:101B100080E461E00E941DBB802B81F534C0CA14B3
:101B2000DB045CF41F5F183F41F480E068E240E8AA
:101B300026E000E00E94D9501FEF80E80E94F3BA2F
:101B4000082F80E863E00E941DBB802BD1F1812F1C
:101B500090E028163906ACF501979695982F8827BE
:101B600097958795B5010E94EBF1862F68E240E8D2
:101B700026E000E00E94D950115023C038EFC31670
:101B8000D10409F0115080E80E94F3BA082F80E8D0
:101B900061E00E941DBB802BA1F0C201811B910955
:101BA0008295807F68E240E826E000E00E94D950FC
:101BB0001F5F39F480E068E240E826E00E94D950D7
:101BC00017EF80E20E9412BB882341F080E068E2B8
:101BD00040E826E000E00E94D9501F2D80E10E94DD
:101BE000FDBA882371F0191509F4ECC4E981FA8172
:101BF0008491E091DC1BF091DD1BE80FF11D108357
:101C0000D7C480E20E94FDBA882309F45ACFDAC40F
